:1000000000800020BD01000079CA000035CA000050
:1000100035CA000035CA000035CA000035CA0000E4
:1000200035CA000035CA000035CA000079CA000090
:1000300079CA000035CA0000EDBE0000F1BE000024
:1000400079CA000079CA000079CA000079CA0000A4
:1000500079CA000079CA000079CA000079CA000094
:1000600079CA000079CA000079CA000079CA000084
:1000700079CA000079CA000079CA000079CA000074
:1000800079CA000079CA000079CA000079CA000064
:1000900079CA00000D8BFF1F79CA000079CA0000E1
:1000A00031AE00003DAE000079CA000079CA000000
:1000B00079CA000079CA000079CA000079CA000034
:1000C00079CA000079CA000079CA000079CA000024
:1000D00079CA000079CA000079CA000079CA000014
:1000E00079CA000079CA000079CA000079CA000004
:1000F00079CA000051DA000079CA0000A1E30000CB
:1001000079CA000079CA000079CA000079CA0000E3
:1001100079CA000079CA000079CA000079CA0000D3
:1001200079CA000079CA000079CA000079CA0000C3
:1001300079CA000079CA000079CA000079CA0000B3
:1001400079CA000079CA000079CA000079CA0000A3
:1001500065C200007DC2000095C20000ADC2000073
:1001600079CA000001E7000079CA000079CA0000DE
:1001700079CA000079CA000079CA000079CA000073
:1001800079CA000079CA000079CA000079CA000063
:1001900079CA000079CA000079CA000079CA000053
:1001A00079CA000079CA000079CA000079CA000043
:1001B00079CA000079CA000079CA0000574B4CF296
:1001C000205210B5DA814DF62812DA8100BF00BF47
:1001D0000BF0F6F8524B4FF010621A63514A9A63D3
:1001E000514ADA63514A136913F4807303D153619E
:1001F0004FF4A85313614E4B9A78110703D59A78A0
:1002000042F008029A704B4B4B482A221A704B4B13
:10021000DA1C121AC11E22F00302994288BF002282
:1002200047490CF033FB474B4748DA1C121AC11EF2
:1002300022F00302994288BF0022002114F03EFC04
:10024000424943484FF4DE720CF020FB414B424AD6
:10025000802103F8011B9342FBD14FF0E0233C4A7D
:10026000C3F8082D3D4B8A221A70A3F5805324222F
:100270005A70A0221A709A799207FCD59A79D406FE
:10028000FCD4374B9A7902F00C02082AFAD10322E7
:100290001A7140225A719A799006FCD5304A9379A6
:1002A0005906FCD51E4B2F4959640221996420211F
:1002B0001170917901F00C010C29FAD12A4A5A6087
:1002C0004FF0E023294A5A6100229A6107221A61FD
:1002D000274AC3F8202D62B60CF040FD134B5B6932
:1002E000DA0705D523480CF02DFD234B234ADA61AC
:1002F000234B1B785B0609D51F4C204BE2699A42C1
:1003000004D11C480CF01EFD0023E3610CF0B8FB87
:1003100014F02CFC0CF0B2FAFEE700BF0020054000
:1003200000800440823F04000100002B00D0034005
:1003300000D0074000E007402089FF1FF09CFF1F0E
:10034000684A020064A6FF1FF09CFF1F0000000027
:100350000084FF1F00E400E05FE400E0005006407E
:100360000040064000000301C0100500FF760100B8
:10037000000020204C6A5F6400E00340A5C3945A4B
:1003800000F00740FFFFFFFFFFFFFFFFFFFFFFFF42
:10039000FFFFFFFFFFFFFFFFFFFFFFFFFFFFFFFF6D
:1003A000FFFFFFFFFFFFFFFFFFFFFFFFFFFFFFFF5D
:1003B000FFFFFFFFFFFFFFFFFFFFFFFFFFFFFFFF4D
:1003C000FFFFFFFFFFFFFFFFFFFFFFFFFFFFFFFF3D
:1003D000FFFFFFFFFFFFFFFFFFFFFFFFFFFFFFFF2D
:1003E000FFFFFFFFFFFFFFFFFFFFFFFFFFFFFFFF1D
:1003F000FFFFFFFFFFFFFFFFFFFFFFFFFFFFFFFF0D
:10040000FFFFFFFFFFFFFFFFFFFFFFFFDEF9FFFF23
:100410000548064B1B1AD90F01EBA301491002D066
:10042000034B03B118477047F09CFF1FF09CFF1F60
:100430000000000008B5054B1BB105490548AFF3A6
:100440000080BDE80840FFF7E3BF00BF00000000E8
:10045000F09CFF1F604A0200012108B528200CF023
:100460008DFE0C200CF0DEFD002128200CF0C8FCD5
:10047000F8B5431E092B24D8124C07460E461A2005
:1004800004F1090501E014F8010F00210CF076FEDB
:10049000AC42F8D12EB931462820BDE8F8400CF026
:1004A000AFBC094BDC5D012120460CF067FE204605
:1004B00000210CF02FFE31462820BDE8F8400CF05A
:1004C0009FBCF8BDE1BF0100E0BF0100704700BF65
:1004D00000207047014B01221A707047448EFF1FA5
:1004E00038B51A4C25683DB3284608F00BF820684B
:1004F000174907F06BFF2068164907F08BFF20684B
:10050000002107F0F3FF20684FF4004108F022F8C3
:10051000206847F6FF7108F02DF82068022108F0E6
:1005200039F8206808F00CF8206807F013FFBDE8E0
:1005300038400C200CF076BD10200CF0EFFA064A83
:100540000649054607F0FCFE2560CDE7089DFF1F24
:100550000000164400002041DD9800001D990000B5
:1005600008B5024B186810F0C5FA08BD349EFF1F8D
:100570002DE9F84F5949DFF868815A4EDFF8689144
:10058000022200200CF020FBFFF7AAFF05F020FF5D
:1005900006F036F8A6240A21404606F0C5F80028E1
:1005A00072D102200CF046FEB4F5805FA8BF002493
:1005B000214628200CF024FC02200CF03BFE33786E
:1005C000002B63D0494D02200CF034FE286807F060
:1005D000F9FF0028DFD002200CF02CFE286807F07D
:1005E000AFFF01232868337008F004F80746286835
:1005F00008F016F88346286808F028F8824628682C
:1006000008F03AF8054602200CF014FE384805F0D0
:10061000EDFF384805F0EAFF584605F0CDFF3648B3
:1006200005F002FF504605F0C7FF344805F0FCFE18
:10063000284605F0C1FF314805F0F6FE384605F0C2
:10064000BBFF2F4805F0F0FE204605F0A5FF2D4822
:1006500005F0EAFE384610F02FF8494610F084F80D
:1006600010F048FA05F098FF8A2F2BD9932F11D854
:100670008C3F062F16D8244805F0D6FE0A214046A6
:1006800006F052F800288CD0BDE8F88F1F4805F01E
:10069000ADFF80E7013C282021460CF0B1FB0A2089
:1006A0000CF0C8FD1A4805F0BFFE1A4805F0BCFE64
:1006B000932005F071FF184805F0B6FE8B2005F079
:1006C0006BFF68E70134214628200CF099FB204697
:1006D00005F096FF0A200CF0ADFDE3E7D50400001D
:1006E000A8C00100448EFF1F3333333F089DFF1F16
:1006F000ECBF010004C0010038C001003CC0010093
:1007000044C001004CC0010054C0010098C0010069
:1007100064C0010078C0010088C0010038B58F496D
:100720000822044612F080F8A0B18D49204614F04A
:100730006BFA10B98B4B186838BD8B49204614F002
:1007400063FAA0B18949204614F05EFAA0B9884B3B
:10075000186838BD04F1080015F046F9452809D895
:10076000844B1B68BC3003EB8003586838BD824B58
:10077000186838BD814838BD8149204614F044FAD4
:1007800038B12578722D07D163782BB97D4B186865
:1007900038BD7D4B186838BD7C49204614F034FACA
:1007A00010B97B4B186838BD672D04D1637813B935
:1007B000784B186838BD7849204614F025FA10B9EE
:1007C000764B186838BD622D04D1637813B9744B29
:1007D000186838BD7349204614F016FA10B9724BE8
:1007E000186838BD7149204614F00EFA10B9704BE4
:1007F000186838BD6F49204614F006FA10B96E4BE0
:10080000186838BD6D49204614F0FEF910B96C4BDC
:10081000186838BD6B49204614F0F6F910B96A4BD8
:10082000186838BD6949204614F0EEF910B9684BD4
:10083000186838BD6749204614F0E6F910B9664BD0
:10084000186838BD6549204614F0DEF910B9644BCC
:10085000186838BD6349204614F0D6F910B9624BC8
:10086000186838BD6149204614F0CEF910B9604BC4
:10087000186838BD5F49204614F0C6F910B95E4BC0
:10088000186838BD5D49204614F0BEF920B95C4BAC
:1008900018680FF015FF38BD5A49204614F0B4F916
:1008A00010B9594B186838BD5849204614F0ACF9B6
:1008B00010B9574B186838BD5649204614F0A4F9B2
:1008C00010B9554B186838BD5449204614F09CF9AE
:1008D00010B9534B186838BD5249204614F094F9AA
:1008E00010B9514B186838BD5049204614F08CF9A6
:1008F00010B94F4B186838BD4E49204614F084F9A2
:1009000010B94D4B186838BD4C49204614F07CF99D
:1009100010B94B4B186838BD4A49204614F074F999
:1009200010B9494B186838BD4849204614F06CF995
:1009300010B9474B186838BD4649204614F064F991
:1009400010B9454B186838BD4449204614F05CF98D
:10095000002840F08780424B186838BDACC00100C9
:10096000B8C00100349EFF1FC8C00100E4C00100F0
:100970003C9EFF1F4C8EFF1F389EFF1F0000C07F54
:10098000F8C001004C9EFF1F409EFF1F18C10100D0
:10099000509EFF1F249EFF1F24C10100289EFF1FA1
:1009A000749DFF1F30C10100789DFF1F3CC10100F5
:1009B000049EFF1F4CC10100089EFF1F64C101007F
:1009C0000C9EFF1F74C10100109EFF1F8CC101000F
:1009D000149EFF1F9CC10100189EFF1FB4C101009F
:1009E000FC9DFF1FC8C10100009EFF1FE4C1010064
:1009F0005C9EFF1FF0C10100609EFF1F04C201004A
:100A0000649EFF1F14C20100689EFF1F2CC20100DC
:100A1000549EFF1F38C201002C9EFF1F44C20100DC
:100A2000449EFF1F50C201006C9EFF1F54C2010074
:100A3000589EFF1F6CC20100309EFF1F80C2010044
:100A4000489EFF1F94C20100709EFF1FA4C20100B8
:100A5000F49DFF1FA8C20100F89DFF1FB8C201004E
:100A60005C9DFF1FB849204614F0CEF810B9B74B73
:100A7000186838BDB649204614F0C6F810B9B54B11
:100A8000186838BDB449204614F0BEF810B9B34B0D
:100A9000186838BDB249204614F0B6F810B9B14B09
:100AA000186838BDB049204614F0AEF810B9AF4B05
:100AB000186838BDAE49204614F0A6F810B9AD4B01
:100AC000186838BDAC49204614F09EF810B9AB4BFD
:100AD000186838BDAA49204614F096F810B9A94BF9
:100AE000186838BDA849204614F08EF810B9A74BF5
:100AF000186838BDA6491622204611F095FE002838
:100B000000F09080A3491522204611F08DFE0028A8
:100B100000F0BA81A0490822204611F085FE002885
:100B200000F0A3819D490722204611F07DFE002898
:100B300000F08E819A490922204611F075FE0028A6
:100B400000F0778197490822204611F06DFE0028B9
:100B500000F0618194490F22204611F065FE0028C3
:100B600000F04A8191490E22204611F05DFE0028D6
:100B700000F034818E491022204611F055FE0028E5
:100B800000F0D3808B490F22204611F04DFE002843
:100B900000F0BD8088490922204611F045FE00285A
:100BA00000F0A68085490A22204611F03DFE00286B
:100BB00000F0908082490922204611F035FE00287D
:100BC00079D080490922204611F02EFE002864D0F9
:100BD0007D490922204611F027FE00284ED07B498E
:100BE0001022204611F020FE002839D0784910222A
:100BF000204611F019FE20B376491022204611F04C
:100C000013FE00287FF4B6AD04F1100014F0ECFEE2
:100C10000A2803463FF6AEAD6F4AB233126852F867
:100C2000230038BD04F1160014F0DEFE032803464D
:100C30003FF6A0AD684A1268023302EB830358689E
:100C400038BD04F1100014F0CFFE0A2803463FF629
:100C500091AD614A1268A63302EB8303586838BD30
:100C600004F1100014F0C0FE0A2803463FF682ADDE
:100C7000594A9C33126852F8230038BD04F1090028
:100C800014F0B2FE0A2803463FF674AD524A1268C9
:100C9000903302EB8303586838BD04F1090014F067
:100CA000A3FE0A2803463FF665AD4B4A8633126819
:100CB00052F8230038BD04F1090014F095FE0A280B
:100CC00003463FF657AD444A12687A3302EB83037A
:100CD000586838BD04F10A0014F086FE0A2803465D
:100CE0003FF648AD3C4A7033126852F8230038BDD5
:100CF00004F1090014F078FE0A2803463FF63AADE5
:100D0000354A1268643302EB8303586838BD04F136
:100D10000F0014F069FE0A2803463FF62BAD2E4A59
:100D20005A33126852F8230038BD04F1100014F051
:100D30005BFE0A2803463FF61DAD274A12684E3374
:100D400002EB8303586838BDC4C20100609DFF1FD9
:100D5000DCC201001C9EFF1FECC20100209EFF1F91
:100D600004C30100449DFF1F10C30100589DFF1FD5
:100D700024C30100489DFF1F30C301004C9DFF1F8D
:100D800044C30100509DFF1F50C30100549DFF1F2D
:100D900064C301007CC3010094C30100A0C301002F
:100DA000A8C30100B4C30100C0C30100D0C3010047
:100DB000E0C30100F4C3010004C4010010C4010039
:100DC0001CC4010028C4010034C4010040C4010057
:100DD00054C4010068C401004C8EFF1F04F10E00D2
:100DE00014F002FE0A2803463FF6C4AC2E4A2E3306
:100DF000126852F8230038BD04F10F0014F0F4FD1E
:100E00000A2803463FF6B6AC274A1268223302EBA3
:100E10008303586838BD04F1080014F0E5FD0A2882
:100E200003463FF6A7AC204A4433126852F8230029
:100E300038BD04F1090014F0D7FD0A2803463FF637
:100E400099AC194A1268383302EB8303586838BDED
:100E5000E01D14F0C9FD0A2803463FF68BAC124A88
:100E60001833126852F8230038BD04F1080014F05A
:100E7000BBFD0A2803463FF67DAC0B4A12680C33D3
:100E800002EB8303586838BD04F1150014F0ACFD83
:100E9000032803463FF66EAC034A1268063302EBA2
:100EA0008303586838BD00BF4C8EFF1F2DE9F04307
:100EB000DFF81481D8F8009009F10106C8F8006045
:100EC00099F80040282C8FB070D0A4F12B03DBB22E
:100ED0000E2B1CD847F6ED7222FA03F3DA072ED553
:100EE0004146484610F0D6FF0FF0E0FAD8F800600F
:100EF0000446731CC8F8003033782A2B14D02F2BEB
:100F000049D02046C8F800600FB0BDE8F083204605
:100F100011F082FCC0B95F2C16D02C4C731CC8F8A1
:100F2000003033782A2BEAD1FFF7C0FF0146204674
:100F30000FF01AFC044620460FB0BDE8F0832046AF
:100F400011F06AFC0028E8D0C8F800903546152753
:100F50002E4615F8014B204611F056FC5B3CE4B2DE
:100F600027FA04F30028F3D1042C01D8DB07EFD4CF
:100F7000A6EB09042246494601A811F09BFC04F1A6
:100F800038030DEB0304002304F8343C01A8FFF7F9
:100F9000C5FB0446ADE7FFF789FF014620460FF089
:100FA00097FC044620460FB0BDE8F08300F010F82F
:100FB000D8F800305E1CC8F800601B78292B044666
:100FC00097D0024CAAE700BF0C9DFF1F0000C07F16
:100FD00010B5FFF76BFF0F4B1A68511C19601178A1
:100FE0002D29044604D02B290BD01A60204610BDB1
:100FF000FFF7EEFF014620460FF0ACFA044620460C
:1010000010BDFFF7E5FF014620460FF0A5FA0446A4
:10101000204610BD0C9DFF1F38B5114D2860FFF70D
:1010200045FF2B685A1C2A601A782D2A044604D0E2
:101030002B2A0BD02B60204638BDFFF7C9FF014695
:1010400020460FF087FA0446204638BDFFF7C0FF60
:10105000014620460FF080FA0446204638BD00BF06
:101060000C9DFF1F38B50D4D4FF40034234620462C
:1010700004F50064A34208D21A68013203F10403A4
:10108000F8D0002123F0D8FC18B9B4F57E3FEDD19B
:1010900038BD0146284605F035FAF6E77CC4010064
:1010A0002DE9F04100241C6090F800C0BCF13A0F1B
:1010B00084B011D11F4605468846164615F080F9C2
:1010C0000A2803D8204604B0BDE8F081294901AAC6
:1010D000681C11F031FC18B9002004B0BDE8F081A3
:1010E000284615F06DF9019B5B000B339842F3D352
:1010F00021493246E81C11F01FFC0028ECD00A9A66
:101100001C49E81D11F018FC0028E5D00A9A019945
:1011100014783368174E54FA81F454FA83F4C3F305
:1011200007231C4409353B6812E03146023511F0B3
:1011300003FC0028D0D03B68039A08F803203B68E2
:1011400018F803200133FF2B14443B60C4D80199E5
:101150008B42284603AAE8D1064902AA11F0ECFB0B
:101160000028B9D0029B1C44E4B2B4FA84F04009D0
:10117000B3E700BF94C401009CC401002DE9F04F07
:101180000223A149A148DBB04FF4807205F0BAF9FF
:10119000FFF768FF9E4BB3F5802F38D39D4BB3F517
:1011A000802F34D39C4BB3F5802F30D34FF40034D1
:1011B00002E0043C00F00F8123680133F9D0974826
:1011C000211D05F09FF9B4F5FC3F00F3FA80944827
:1011D000DFF850B2944CDFF854A2DFF85492954FE8
:1011E00005F090F9944805F08DF9002505F0C8F850
:1011F0000028FBD005F062F80A2805F5B4730CD07E
:101200000D280AD06B44013503F8C80CEEE78B4873
:101210005BB0BDE8F04F05F075B90DEB0305002399
:1012200005F8C83C9DF8A0303A2B4BD1DBF80030D4
:10123000002B47D1824907AA28A811F07DFB01287D
:1012400019D107992268914240F0C1807D4B1B68FB
:10125000002B00F0BC80D9F80010DAF800207A48A2
:1012600005F050F964200BF0E5FFDAF80010D9F82A
:10127000000023F0DDFB06AB0093236801332360FD
:101280003A4605AB08A928A8FFF70AFF002800F096
:10129000A7806E4B3A681B68059D02931A4450194B
:1012A000B0F5FC3F00F2A480069904296AD8DFE873
:1012B00001F03D130B690300BDF82030634A5BBAAF
:1012C0001B041360002591E7BDF820305F4A5BBA2C
:1012D0009BB21B011360F5E74FF47A700BF0AAFF85
:1012E0002168DAF80030D9F800205948009105F05B
:1012F00009F9DAF80060D9F8005006F5FF3606F56E
:10130000FA7605F50035B54257D2DFF8FC8001E0EA
:10131000AE4252D928460C224146013511F084FADA
:101320000028F5D1474A01231360CBE702F50038C6
:1013300045EA08018B0762D1002D31DD6E1E26F0D3
:10134000030608F10402B31808AE039535461E469D
:1013500001E0B0451ED0404655F8041B08F10408D2
:1013600023F062FB0028F4D001463A48039D05F0C3
:10137000C9F83A683848294605F0C4F80423CBF880
:1013800000309FE7354828AA05F0BCF80323CBF8C6
:10139000003097E73A68029B039D13441A46E81809
:1013A000DAF80030834201D2CAF80000D9F80030E0
:1013B000934288BFC9F8002084E7294805F0A2F8C5
:1013C00080E728485BB0BDE8F04F05F09BB82648A1
:1013D00005F098F876E71148042105F093F8F6E651
:1013E000224828A905F08EF80123CBF8003069E7E0
:1013F0001F4805F087F80223CBF8003062E71D484C
:1014000005F080F8B5E700BFA4C40100B4C4010032
:101410002189FF1FC589FF1F358AFF1FF0C4010006
:1014200020C50100249DFF1F149DFF1F189DFF1F55
:10143000488EFF1F289DFF1F44C50100D8C401002E
:1014400064C50100209DFF1F70C501001C9DFF1F8A
:10145000D8C5010050C601006CC6010018C60100C5
:1014600088C6010008C5010088C50100B0C501009B
:10147000C4C5010034C6010010B504460AF0CCFE14
:10148000204610BD0D4A1368B3B90D4B10B419882E
:1014900072B60C484FF480244FF4A0734464013BAF
:1014A000FDD11023C0F8C8304B0109B1013BFDD17B
:1014B000012310BC13607047704700BF309DFF1FB1
:1014C0002C9DFF1F00F00F40F8B5457804462DB95C
:1014D000207844F2AE3505FB00F0F8BD86783EB1C9
:1014E000C77877B944F2AE3707FB06F6013601E05C
:1014F00044F2AE36207806FB05F5013505FB00F019
:10150000F8BD03793BB10430FFF7DEFF013000FB8B
:1015100007F70137E8E744F2AE30F8E72DE9F84382
:101520002B4CDFF8B0902C4FDFF8B08076210646C8
:10153000204606F0E3FB204606F0C4FCC9F8000094
:10154000204606F0CBFC3860204606F0C1FC24495A
:101550000FF0BEF9C8F80000204606F0C5FC0FF0F9
:10156000ABF820490FF0B4F91F4B05461D6030461B
:101570000FF0A6F80446D9F80000DFF870901C4E72
:1015800021460FF0A5F9D9F800100EF0E5FF21462D
:10159000C9F800003868174F0FF09AF931680EF05B
:1015A000DBFF21463060D8F80000134E0FF090F9B1
:1015B00039680EF0D1FF034621463B6028460FF004
:1015C00087F931680EF0C8FF3060BDE8F88300BFCE
:1015D0007C9DFF1F549EFF1F2C9EFF1F449EFF1FDC
:1015E0000000C84200007A446C9EFF1F589EFF1FF7
:1015F000309EFF1F489EFF1F709EFF1F2DE9F04F7A
:101600008346ADF54D7D4000073000AF20F0070068
:10161000ADEB000D7960084611461E46FEF728FF27
:10162000FEF754FF05F07EFC0120C7F80CD00BF04C
:1016300001FEBBF1000F41DDD7F85833DFF8BC9055
:10164000C7F808B000245B014FF07C58A3469A46C7
:1016500072B61322314607F110004FF4802505F0D1
:1016600063FD4FF4A072C9F84450013AFDD1132232
:10167000314607F5D07005F057FDC9F8485062B6FD
:101680001321424607F5D07005F0E6F942460546BB
:10169000132107F1100005F0DFF9FB682D1A23F87C
:1016A0001B50BAF1000F02D05346013BFDD1BB687D
:1016B0000134A4B29C42A346CADB9B467868002151
:1016C000FEF7D6FEFC684FF07C525946204605F0E6
:1016D000DBF901460A4804F015FF5946204605F09B
:1016E000EBF90EF093FB02460B46064804F00AFFA6
:1016F00007F54D77BD46BDE8F08F00BF00F00F4005
:10170000A8C60100B0C601002DE9F04FA7B002AF96
:10171000D7E92E458A4690469B46FA6005F05AF96D
:1017200064200BF087FD680151464900F8616001B3
:101730005A4C3860C81D7960B8600FCC07F12C0C8A
:10174000C7F818C0ACE80F002368CCF80030C7F821
:1017500024A005F0E7FB52495248CDF800B04346BB
:101760005246514D4FF07C5907F140060AF0FEFDFC
:10177000BA694E4852F8043B3B611C461946BA61AF
:10178000C7F814D004F0BEFEF9682046FEF770FEDC
:10179000BB6823F00703ADEB030D7B6A002B0DF153
:1017A000080A73DD0024C7F820A0D7F800A0A046DF
:1017B0004FF48023FA690AB1013AFDD172B64FF4B1
:1017C000A0726B64013AFDD11022C5F8C820BAF1AD
:1017D000000F02D05246013AFDD1AB6462B614222A
:1017E0005946304605F0A0FC4A461421304605F023
:1017F00033F93B6A013423F818007B6A24B21022C3
:101800009C42C5F8C420A0464FF48023D2DB38693F
:10181000D7F820A00021FEF72BFE254804F004FE97
:101820007B68C7F820A09C1E0AEB0403AAF10208FB
:10183000204CC24698463AF9021F204604F062FE48
:10184000C245F8D1D7F820A07C6A4A4621465046C6
:1018500005F01AF90146184804F054FE2146504696
:1018600005F02AF90EF0D2FA02460B46134804F0AE
:1018700049FE134804F0BAFEBB69D7F814D0B3424E
:101880007FF476AF9437BD46BDE8F08F386900210C
:10189000FEF7EEFD064804F0C7FDD5E7D0D2010003
:1018A000D8C601007095FF1F00F00F4014C701005B
:1018B0005CC7010020C7010024C7010040C7010028
:1018C000ACC6010070B50546002006F051FC044688
:1018D000002006F04DFC014620460EF03DFE044679
:1018E000002006F045FC014620460EF035FE0A4970
:1018F0000A4E0EF0EDFF0A4B04461C6028460EF01F
:10190000DFFE014620460EF0E3FF31680EF024FEB4
:101910003060204670BD00BF00004040009EFF1FA9
:10192000FC9DFF1F2DE9F04FA1B008AE86E8030033
:1019300031B3DFF8748215461F460024CB68A342FA
:101940001EDD224631460FA806F060FB00210FA8DD
:1019500006F07AFB01460BA80AF070FD41460BA881
:101960000AF0F0FD78B12846FFF7D8FD6B1EBB42A8
:1019700067D00BA80AF026FD099901340029DDD1B2
:1019800021B0BDE8F08F89490BA80AF0DBFD90B1CA
:101990002846FFF797FF6B1EBB42EAD12A9B002B1C
:1019A000E7D1834B18680EF031FA02460B468148A6
:1019B00004F0A8FDDDE780490BA80AF0C3FD00286C
:1019C00060D0224631460FA806F020FB01210FA867
:1019D00006F030FB2246824631460FA806F016FB81
:1019E00002210FA806F026FB2246834631460FA8A7
:1019F00006F00CFB03210FA806F01CFB22468146D3
:101A000031460FA806F002FB04210FA806F012FBD6
:101A1000009001204B4601905A4651462846FFF758
:101A2000EDFD6B1EBB42A4D12A9B002BA1D1634BC1
:101A300018680EF0EBF902460B46614804F062FDAF
:101A400097E72A9B002B94D15E4B18680EF0DEF9C5
:101A50005D4B824618688B460EF0D8F9CDE904013B
:101A60005A4B18680EF0D2F9CDE90201584B1868AC
:101A70000EF0CCF95246CDE900015B46554804F022
:101A800041FD76E754490BA80AF05CFD002841D0DF
:101A9000224631460FA806F0B9FA01210FA806F038
:101AA000C9FA2246824631460FA806F0AFFA022153
:101AB0000FA806F0BFFA2246834631460FA806F06B
:101AC000A5FA03210FA806F0B5FA22468146314651
:101AD0000FA806F09BFA04210FA806F0ABFA0090BD
:101AE00002204B4601905A4651462846FFF786FD94
:101AF0006B1EBB427FF43DAF2A9B002B7FF439AFB6
:101B0000364B18680EF082F902460B46344804F052
:101B1000F9FC2EE733490BA80AF014FD8146002892
:101B200066D0224631460FA806F070FA01210FA8B0
:101B300006F080FA2246824631460FA806F066FA81
:101B400002210FA806F076FA2246834631460FA8F6
:101B500006F05CFA03210FA806F06CFA22468146D3
:101B600031460FA806F052FA04210FA806F062FAD7
:101B7000009003204B4601905A4651462846FFF7F5
:101B80003DFD6B1EBB427FF4F4AE2A9B002B7FF41D
:101B9000F0AE154B18680EF039F902460B461348A3
:101BA00004F0B0FCE5E600BF68C70100B4C1010065
:101BB000009EFF1FC4C701003CC10100089EFF1F1B
:101BC000E0C70100589EFF1F709EFF1F489EFF1F29
:101BD000309EFF1F8CC7010064C10100109EFF1FD3
:101BE000F8C701008CC10100189EFF1F10C801003A
:101BF000BD490BA80AF0A6FC00283ED0224631467B
:101C00000FA806F003FA0FA8012106F013FA4FF40B
:101C10007A7A5FFA80FB58460AF06AFDBAF1010A47
:101C20008144F8D1B14BDFF8C8B283FB09204FEAF9
:101C3000E973C3EBA0100EF043FDAE4B8246186073
:101C400028460EF03DFD014650460EF041FEDBF801
:101C500000100EF081FC6B1EBB42CBF800007FF43D
:101C600088AE2A9B002B7FF484AE0EF0CFF802469C
:101C70000B46A14804F046FC7BE6A0490BA80AF0FD
:101C800061FC78B3224631460FA806F0BFF9012166
:101C90000FA806F0CFF9C0B20BF062FA0EF00CFDFF
:101CA000974BDFF860B21860824628460EF008FDB8
:101CB000014650460EF00CFEDBF800100EF04CFC16
:101CC0006B1EBB42CBF800007FF453AE2A9B002B67
:101CD0007FF44FAE0EF09AF802460B468A4804F0A5
:101CE00011FC46E689490BA80AF02CFC002835D1E6
:101CF00087490BA80AF026FC00285CD02246314612
:101D00000FA806F083F901210FA806F093F903301C
:101D100005F07CFE0EF0D0FC7E4BDFF8FCB11860C5
:101D2000824628460EF0CCFC014650460EF0D0FD0F
:101D3000DBF800100EF010FC6B1EBB42CBF800006D
:101D40007FF417AE2A9B002B7FF413AE0EF05EF8E3
:101D500002460B46714804F0D5FB0AE64FF4FA60E0
:101D600005F0AEFC0EF0A8FCDFF8B4A1CAF8000044
:101D700064200BF05FFA28460EF0A2FC0146DAF868
:101D80000000DFF8A0A10EF0A3FDDAF800100EF0BD
:101D9000E3FB6B1EBB42CAF800007FF4EAAD2A9B4E
:101DA000002B7FF4E6AD0EF031F802460B465E489C
:101DB00004F0A8FBDDE55D490BA80AF0C3FB78B38E
:101DC000224631460FA806F021F901210FA806F09E
:101DD00031F9033005F01AFE0EF06EFC544BDFF8BB
:101DE00054B11860824628460EF06AFC01465046FF
:101DF0000EF06EFDDBF800100EF0AEFB6B1EBB426A
:101E0000CBF800007FF4B5AD2A9B002B7FF4B1AD79
:101E10000DF0FCFF02460B46474804F073FBA8E5B3
:101E200046490BA80AF08EFB78B3224631460FA82C
:101E300006F0ECF801210FA806F0FCF8033005F0DD
:101E4000E5FD0EF039FC3E4BDFF8F8B01860824635
:101E500028460EF035FC014650460EF039FDDBF801
:101E600000100EF079FB6B1EBB42CBF800007FF434
:101E700080AD2A9B002B7FF47CAD0DF0C7FF02469E
:101E80000B46314804F03EFB73E530490BA80AF0DD
:101E900059FB069000285DD0224631460FA806F077
:101EA000B5F801210FA806F0C5F822465FFA80FABE
:101EB00031460FA806F0AAF802210FA806F0BAF8DA
:101EC000834604F02FFA012150460BF057F95FFAD0
:101ED0008BF3002B00F098801D4B53F83A30012211
:101EE00083F8802045E500BFB8C20100D34D6210E1
:101EF000609DFF1F5C9DFF1F28C80100DCC2010020
:101F00001C9EFF1F209EFF1F3CC80100A4C20100B1
:101F100004C30100449DFF1F589DFF1F5CC80100C2
:101F2000F49DFF1FF89DFF1F50C8010024C301004E
:101F3000489DFF1F4C9DFF1F6CC8010044C301005A
:101F4000509DFF1F549DFF1F7CC801008CC80100DD
:101F5000BCD8010030490BA80AF0F4FA00283FF47D
:101F600008AD224631460FA806F050F801210FA80F
:101F700006F060F822465FFA80FA31460FA806F0B4
:101F800045F802210FA806F055F80FAB224681460E
:101F90003146184606F03AF80FAB0321184606F012
:101FA00049F80FAB834622463146184606F02EF814
:101FB0000FAB0421184606F03DF80FAA0346174957
:101FC0000793104644220AF061FC504601210BF0B1
:101FD000D5F820AB03EB8B02504652F8441C0BF0B3
:101FE0002FF858460BF01EF8494650460AF008FFF5
:101FF000079B18460BF01EF9504606990AF000FFA1
:102000000C200BF00FF8B4E4054B53F83A300122E2
:1020100083F80021ADE400BF9CC80100E4D20100B8
:10202000BCD8010070B5002086B005F041F8092841
:10203000014640F34D82C64D2A6813681068146843
:10204000166892680592C0F30740C4F30724CDE9EF
:102050000004F6B2BF4CC04AC04803911B0EC049F1
:102060000296049404F04EFABE48BF4E04F0DCF928
:1020700000242B6804F10C0203EB8203013458683E
:102080000DF0C4FE02460B46304604F03BFA0A2C23
:10209000EFD12B68B44ED86D0DF0B8FE02460B465A
:1020A000B24804F02FFAB248002404F0BDF92B68BE
:1020B00004F11802013453F822000DF0A7FE024685
:1020C0000B46304604F01EFA0A2CF0D12B68A64EBF
:1020D000D3F888000DF09AFE02460B46A34804F0A0
:1020E00011FAA448002404F09FF92B6804F1380287
:1020F00003EB8203013458680DF088FE02460B465C
:10210000304604F0FFF90A2CEFD12B68964ED3F835
:102110000C010DF07BFE02460B46944804F0F2F9E8
:102120009548002404F080F92B6804F1440201343E
:1021300053F822000DF06AFE02460B46304604F0CA
:10214000E1F90A2CF0D12B68874ED3F838010DF055
:102150005DFE02460B46854804F0D4F9874800240A
:1021600004F062F92B6804F1220203EB82030134CC
:1021700058680DF04BFE02460B46304604F0C2F99B
:102180000A2CEFD12B68784ED3F8B4000DF03EFE48
:1021900002460B46754804F0B5F97948002404F06E
:1021A00043F92B6804F12E02013453F822000DF09C
:1021B0002DFE02460B46304604F0A4F90A2CF0D15D
:1021C0002B68694ED3F8E0000DF020FE02460B4666
:1021D000664804F097F96B48002404F025F92B6851
:1021E00004F14E0203EB8203013458680DF00EFE39
:1021F00002460B46304604F085F90A2CEFD12B68D5
:10220000594ED3F864010DF001FE02460B465748C3
:1022100004F078F95C48002404F006F92B6804F116
:102220005A02013453F822000DF0F0FD02460B462D
:10223000304604F067F90A2CF0D12B684A4ED3F8E7
:1022400090010DF0E3FD02460B46484804F05AF9B0
:102250004E48002404F0E8F82B6804F1640203EB14
:102260008203013458680DF0D1FD02460B4630461A
:1022700004F048F90A2CEFD12B683B4ED3F8BC018F
:102280000DF0C4FD02460B46384804F03BF94048C7
:10229000002404F0C9F82B6804F17002013453F8EB
:1022A00022000DF0B3FD02460B46304604F02AF939
:1022B0000A2CF0D12B682C4ED3F8E8010DF0A6FDC6
:1022C00002460B46294804F01DF93248002404F068
:1022D000ABF82B6804F17A0203EB820301345868EF
:1022E0000DF094FD02460B46304604F00BF90A2C23
:1022F000EFD12B681C4ED3F814020DF087FD024677
:102300000B461A4804F0FEF82348002404F08CF829
:102310002B6804F18602013453F822000DF076FD9B
:1023200002460B46304604F0EDF80A2CF0D12B683B
:102330000D4ED3F840020DF069FD02460B460B48E6
:1023400004F0E0F81548002404F06EF828E000BF1F
:102350004C8EFF1FB4C9010010C9010028C901003B
:1023600018C90100BCC90100CCC90100D4C90100D1
:10237000DCC90100E8C90100F8C9010008CA010070
:102380001CCA010030CA010048CA01005CCA010031
:102390006CCA01007CCA01008CCA01009CCA010001
:1023A0002B6804F1900203EB8203013458680DF0AE
:1023B0002DFD02460B46304604F0A4F80A2CEFD15E
:1023C0002B68484ED3F86C020DF020FD02460B46F8
:1023D000454804F097F84548002404F025F82B6898
:1023E00004F19C02013453F822000DF00FFD024667
:1023F0000B46304604F086F80A2CF0D12B68394E93
:10240000D3F898020DF002FD02460B46364804F060
:1024100079F83748002404F007F82B6804F1A60285
:1024200003EB8203013458680DF0F0FC02460B46C2
:10243000304604F067F80A2CEFD12B68294ED3F808
:10244000C4020DF0E3FC02460B46274804F05AF89C
:102450002848002403F0E8FF2B6804F1B20201349D
:1024600053F822000DF0D2FC02460B46304604F031
:1024700049F80A2CF0D12B681F4ED3F8F0020DF06A
:10248000C5FC02460B461848002404F03BF82B68B4
:1024900004F1BC0203EB820358680DF0B7FC02465E
:1024A0000B4630462146013404F02CF8452CEED181
:1024B0002B68D3F808040DF0A9FC02460B460F4820
:1024C000214604F01FF806B0BDE8704004F0AEB835
:1024D0000B4804F017F804F0A9F806B0BDE8704006
:1024E00004F026B8CCC90100D4C90100ACCA01006F
:1024F000C4CA0100DCCA0100F4CA010008CB010013
:10250000ACC8010070B50D4604463549284612F0A6
:102510007BFB48B9334B34483449354A84E80F00D3
:1025200004236361204670BD324E2846314612F0C6
:102530006BFB20B9012326606361204670BD2E4EDF
:102540002846314612F060FB0028F3D02B4E284677
:10255000314612F059FB0028ECD0294E284631466E
:1025600012F052FB0028E5D0264E2846314612F0E4
:102570004BFB0028DED0244E2846314612F044FBA7
:102580000028D7D02149284612F03EFB28B9204B1D
:10259000204AC4E900230223C3E71F4E28463146E0
:1025A00012F032FB0028C5D01C49284612F02CFB43
:1025B00018B91A4B23600123B3E7194E2846314658
:1025C00012F022FB0028B5D0164E2846314612F0F4
:1025D0001BFB0028AED0144B23600123A1E700BFF2
:1025E00068C7010050C201002CC2010038C20100BE
:1025F00044C20100B8C2010004C3010024C30100A9
:1026000044C30100A4C20100B4C101001CCB0100FD
:1026100028CB010030CB0100DCC201003CC101002D
:1026200064C101008CC1010038CB01002DE9F04FDD
:10263000ADF54E5D89B006AF2822002107F5E670A2
:1026400012F03CFA07F55F7507F523742046002168
:10265000103409F0F3FEAC42F8D1234E07F5237491
:1026600020463146103409F0FDFEA542F8D11F493D
:1026700041F664134FF4FA7207F5956004F002F81E
:1026800007F5956004F09EFA002801F06C8607F5C6
:10269000956013F095FE012403464FF0000807F5FE
:1026A000956500E00134A34222D9295D7B29F9D147
:1026B00007F5237303EB081907F595631E194846C0
:1026C00009F030FF16F8011F7D2904F10104F6D14D
:1026D000484609F027FF07F5956013F071FE08F1F1
:1026E00001080346DEE700BFACC6010048CB01008D
:1026F0000020C7F8408004F0DBFC0928014641F3C4
:102700000D86CE4BCE4E1868CE4A03680568046825
:1027100000680391C0B2C4F30724C5F30745CA4952
:1027200002901B0EC94801940496009503F0EAFE3E
:10273000C74803F079FEC74B1022C3F8C4200A2013
:102740000AF078FD00230122FB64C7F894301C4690
:10275000BA647B6704F0E6FB3B6C002B01F0CF8290
:1027600000237B65786DBC4AC7F810D007F562730B
:1027700003EB0013002453F8F49C53F8FC1C09F1FC
:10278000080323F00703ADEB030D06AD07F1DC03EF
:10279000002908BF11464FEA00184A461C605C60D9
:1027A00028461E4610F086F807F523734046AB49CD
:1027B00005F80940184409F055FE07F55F7007F069
:1027C00009F807F5956240F2EE23294607F55F7098
:1027D00006F070FE07F59563A04229460CBF1A4625
:1027E000224607F55F7005F039FC07F55F7393E843
:1027F000030086E80300002800F0F885002900F0B7
:10280000F5853B6C3C65013BBB61954907F1DC00FC
:1028100005F06AFC934983B207F1DC00FB6605F022
:1028200063FC9149824607F1DC0005F05DFC8F4AAC
:1028300083B207F1DC0107F1E400C7F8D03005F0FE
:1028400043FC8B4A07F1DC0107F1EC0005F03CFC8E
:10285000884A07F1DC0107F1F40005F035FC864AEF
:1028600007F1DC0107F1FC0005F02EFC834A07F1BB
:10287000DC0107F5827005F027FC814907F1DC00D7
:1028800005F032FC7F4907F1DC0005F02DFC7E4AA3
:1028900083B207F1DC0107F58670C7F8803005F0D8
:1028A00013FC7A4907F1DC0005F028FC014607F526
:1028B000C67009F0C3FD764907F1DC0005F014FC91
:1028C000744907F1DC0005F00FFC031E08BF01236B
:1028D00071497B6607F1DC0005F006FC6F49786101
:1028E00007F1DC0005F000FC6D49B86407F1DC007D
:1028F00005F0FAFB6B49F86007F1DC0005F0F4FB2A
:10290000031E08BF01236849FB6307F1DC0005F0E3
:10291000EBFB6649786007F1DC0005F0E5FB1FFA88
:102920008AF3C7F808D0C7F8C830B863002841F068
:10293000C7845F4A07F1DC0107F58A7005F0C4FB24
:102940005C4A07F1DC0107F58E7005F0BDFB5A4AC1
:1029500007F1DC0107F5927005F0B6FB574A07F165
:10296000DC0107F5967005F0AFFB554A07F1DC0175
:1029700007F59A7005F0A8FB524A07F1DC0107F54C
:102980009E7005F0A1FB504A07F1DC0107F5A2702B
:1029900005F09AFB4D4A07F1DC0107F5A67005F03A
:1029A00093FB4B4A07F5AA7007F1DC0105F08CFB9D
:1029B000484A07F1DC0107F5AE7005F085FB07F525
:1029C0005F75444A07F1DC0107F5FA7005F07CFBFE
:1029D000002207F5FA71284605F018FB0021284669
:1029E00005F032FB3C4A386307F1DC0107F5B270B1
:1029F00005F06AFB394A07F1DC0107F5B67005F00E
:102A000063FB374A07F1DC0107F5BA7005F05CFBA0
:102A1000344A07F1DC0107F5BE7005F055FB324A78
:102A200007F1DC0107F5C27005F04EFBD7F8102165
:102A300007F58673002A01F0298257E04C8EFF1FAC
:102A4000B4C9010010C9010018C9010094CB0100EC
:102A500010CC010000F00F4068D80100ACC60100A6
:102A60003CCC010050CC01004CCC01005CCC0100FE
:102A700068CC010070CC010078CC010088CC01004A
:102A800094CC0100A0CC0100ACCC0100B4CC01007E
:102A9000C0CC0100D0CC0100DCCC0100ECCC0100AA
:102AA000FCCC010010CD01001CCD01002CCD01009B
:102AB00044CD010054CD010064CD010078CD01006A
:102AC00094CD0100B0CD0100BCCD0100CCCD010002
:102AD000D4CD0100E4CD0100F8CD010000CE01000D
:102AE0000CCE010018CE010020CE01004FF0000BEB
:102AF000594607F58679C7F884B0C7F8D4A0DA46F6
:102B0000CB468946D268524547DD5146584605F0C6
:102B100091FA07F5A276524604463146284605F05A
:102B200075FAD7F8802332B1D7F88430D26802FB27
:102B30000433C7F884300024A0460DE0DB689C42D3
:102B400016DA05F063FA2146284605F073FA0028E4
:102B5000C8BF08F10108013452463146284605F045
:102B600055FAD7F88033524631462846002BE5D136
:102B7000514607F5B27005F05DFA012851465846F6
:102B800000F05D8705F056FA08FB009907F586729C
:102B90000AF1010A5268002AB4D14B469B0009F1A0
:102BA000FF32C0487B62D7F8D4A0C7F82890FA62F9
:102BB00003F03AFCD7F8C8304D46002B41F077813E
:102BC000D7F8D030012B01F07C817B6A073323F0EA
:102BD0000703ADEB030D06AAADEB030D06AB7B645B
:102BE000BB6ABA66002B0BDDBB6AB86E9C0022463E
:102BF000002111F063FF786C2246002111F05EFF86
:102C0000D7F860C107F5AE73BCF1000F01F0508337
:102C10000026B046324607F5FA74DCF80C309A42CA
:102C200007F5AE7120461ADA05F0F0F9002107F534
:102C3000FA7005F009FA014607F55F70FFF762FCCC
:102C4000D7F89033D7F860C101364344B6B207F5E0
:102C5000AE721FFA83F83246BCF1000FDDD1C7F81F
:102C60007880BA6F134605FB03F39B00073323F00C
:102C70000703ADEB030D06AEC7F8C4601346002A88
:102C800041F0FB827C6E012C08DD874803F0CCFB11
:102C9000204603F081FC854803F0C6FB844A854941
:102CA00000231360844A1360844A1360844A1360CB
:102CB000844A1360844A1360844A1360844A136010
:102CC000844A1360844A1360844A1360844A136000
:102CD000844A1360844A1360844A1360844A1360F0
:102CE000844A1360844A1360844A1360844A1360E0
:102CF000844A1360844A1360844A1360844A1360D0
:102D0000844A1360844A1360844A1360844A07F13A
:102D1000DC00136005F0E8F9012801F0FB8281492D
:102D200007F1DC0005F0E0F9002841F09D827B6EA0
:102D3000002B40F3A9827B6A9B08FB6197F838302F
:102D40003B6200233B6703F01BFB002840F05386E7
:102D50003B6B002B00F06386D7F88430002B40F3E8
:102D600055820023C7F8B430BB657B63C7F8883051
:102D7000C7F8D4309B46C7F8D03007F5A273C7F820
:102D8000AC3007F1FC03FB6707F5CE73C7F8A03042
:102D900007F5D673C7F8A43000240023C7E92E3402
:102DA000614E07F5FA7AD7F8D430C7F89CD0002BDB
:102DB00000F01885D7F89490F86F594605F03AF965
:102DC0005A46D7F8AC100546504605F01FF9D7F81B
:102DD000D030B3FBF9F809FB1838414607F5FA7013
:102DE00005F028F9514BDFF8489118705A4607F55D
:102DF0009A71504605F00AF9414607F5FA7005F058
:102E000023F90146D7F8A00009F018FBD7F89C0178
:102E1000002808BF484607F5CE73FEF7FDF85A466E
:102E200007F59E710446504605F0F0F8414607F557
:102E3000FA7005F0FFF85A46C7F8C00007F582712E
:102E4000504605F0E3F8414607F5FA7005F0F2F850
:102E50005A4683B207F58E715046C7F8983005F090
:102E6000D5F8414607F5FA7005F0EEF80146D7F8B7
:102E7000A40009F0E3FAD7F8AC01002808BF4846DF
:102E800007F5D673FEF7C8F80DF05AFE294B1880E7
:102E9000ABB2002B00F0E48299469B00C7F8A83043
:102EA0004AE000BF30CE010050CE0100D0C9010081
:102EB000009EFF1F5CCE0100FC9DFF1F6C9EFF1F4C
:102EC000449EFF1F2C9EFF1F549EFF1F709EFF1FDE
:102ED000489EFF1F309EFF1F589EFF1FF89DFF1F3B
:102EE000F49DFF1F089EFF1F049EFF1F109EFF1FE3
:102EF0000C9EFF1F189EFF1F149EFF1F509DFF1F5B
:102F0000489DFF1F449DFF1F1C9EFF1F5C9DFF1FD0
:102F1000549DFF1F4C9DFF1F589DFF1F209EFF1FAC
:102F2000609DFF1F70CE0100389DFF1F349DFF1F65
:102F300068D801002C9DFF1FD7F89420D7F8D43013
:102F40009A420ADD002B00F03D8320460DF0F8FD8B
:102F5000C14B81B21878FDF78BFA03F011FA002803
:102F600040F0AC82D7F8A830073323F00703ADEB6D
:102F7000030D06AAC7F8C820B84AADEB030D00231D
:102F8000136006ABC7F8B030B44B1B68002BFBD006
:102F9000B7F8C050D7F8C8004A46294604F0C4F82C
:102FA000002333600F24152009F0A2FB3368013C95
:102FB0001844A4B23060002CF5D1A94BA3FB00301B
:102FC000D7F8D430C008022B306000F33E820CF0FA
:102FD000FBFEC7E92E01DFF88C824FF48023C8F88E
:102FE00048302023013BFDD1D7F8B00029464A469E
:102FF00004F09AF862B61023C8F8C430BB6F002BF7
:1030000040F05583D7F88030012B00F03F834946CC
:10301000D7F8C8004FF07C5203F01EFD5946804699
:1030200007F1E40005F006F8002840F03682D7F8F2
:10303000D430022B00F31A82D7E92E34C7E9323498
:10304000854B1A78884B1B68D7E9324503EB82031E
:103050002046D3F84422D3F81812D3F8EC31C7F83D
:10306000A820C7F890102246C7F88C3029462B4676
:103070000CF024FF0446D7F8A8000D460CF0C6FE5D
:1030800002460B46204629460CF018FF774B0022DB
:103090000DF03EF8002200230CF05AFD0446D7F84C
:1030A00090000D460CF0B2FED7E932230CF006FF7B
:1030B00002460B46204629460CF04AFD0446D7F846
:1030C0008C000D460CF0A2FE02460B462046294617
:1030D0000CF03EFD02460B46002065490DF018F845
:1030E000044640460D460CF07FFE02460B46204645
:1030F00029460CF0E3FE0DF091F98046D7F89830A0
:10310000002B00F0C181544B1B78002B44D07B6F07
:10311000A8EB03000DF0D4FA002104460DF0C2FC28
:10312000002840F0E181534920460DF0D9FC0028E9
:1031300040F0D083204650490DF016FB0446594616
:1031400007F1E40004F076FF002840F0D681B7F8DC
:10315000C030002B00F0DE81012B00F0D583D7F8C2
:1031600088502146BC6E54F825000DF0F5F9FB6E31
:1031700044F82500012B0AD130680DF09DFA7C6CD3
:10318000014654F825000DF0E7F944F82500D7F87A
:1031900088300133C7F88830D7F8D4300133C7F806
:1031A000D430D7F8D0305946013307F58670C7F8C8
:1031B000D03004F03FFFD7F8AC1004465A465046D2
:1031C00004F024FFDAF8043013B1DB6804FB03F3E6
:1031D000D7F8D420934204D100230BF1010BC7F898
:1031E000D430D7F8B430D7F8A40001331C46C7F860
:1031F000B43009F0E7F8D7F8A00009F0E3F8D7F801
:103200008430D7F89CD09C42FFF6CDAD1B4CBD6BF3
:1032100007F5E67307F5FA71012053F8042B954280
:1032200005D0A25C164E56F8322082F800018B427F
:10323000F3D13A6A124B3C6F53F8323011480122F5
:10324000013483F800213C6708F0E6FF7B6EA3425F
:1032500000F3C48318E000BF349DFF1F309DFF1FA3
:103260008988888800F00F404C8EFF1F00408F40F7
:103270000000F03F00FF7F4700401C4680D3010064
:10328000BCD801003C9DFF1F07F1F40393E8030045
:1032900007F1EC0207F5CE7383E8030092E8030020
:1032A00007F5D67282E803005B68002900F0D48736
:1032B000D1F80CB0002B01F03A80DB68C7F8D430AD
:1032C000BBF1000F4FDDB64D4FF0000807F5DE7A79
:1032D00007F5D67607F5FA7907E008F1010807F552
:1032E000FA7009F06FF8C3453DDD42463146484665
:1032F00004F08CFE002107F5FA7004F09BFE4246B4
:103300000446314607F5DE7004F080FE0121504688
:1033100004F09AFE014607F5FA7009F08FF8462C82
:10332000DBD8A04BD9F80000002808BF1846FDF7ED
:1033300073FE9D4BC7F8C8001B6803EB8404D4F8E8
:10334000F4120DF0A5FB18B9D7F8C830C4F8F43260
:103350006B78DB07FCD508F1010807F5FA7009F076
:1033600031F8C345C1DCD7F8D440002C00F30C85FC
:1033700007F5AE735B68002B00F0F7837A6AD7F825
:10338000C4A0D7F82C80BE6A9208C7F8B8200022E3
:10339000C7F8C020C7F8D020DB689A4280F2E583E6
:1033A00007F5AE7107F5DE7004F030FE002107F579
:1033B000DE7004F049FE07F5FA7401462046FFF777
:1033C000A1F86369C7F8C430002B40F3C28300231F
:1033D000C7F8C830D7F8C820042A00F27483DFE8A1
:1033E00012F00A043B04120402046B036F4803F05A
:1033F0001BF8284603F018F8D7F810D06C4803F0F3
:1034000013F803F013F903F093F86A4B1A2203F14F
:103410000900012101E013F8012F674C54F8322014
:10342000834282F80011F6D107F55B74204608F05C
:10343000C9FF07F52372A242A4F11004F6D107F5E3
:103440004E570C37BD46BDE8F08F0CF0BDFC024670
:103450000B46D7E92E010CF07BFBC7E92E01BAE53C
:103460002423C7F8A8304FF0090965E5D7F8D43010
:10347000581E0CF0B9FC02460B46D7E92E010CF0A1
:1034800047FEC7E93201DBE5D7F8B00049464FF007
:103490007C5203F0E1FA786735E6594607F1E4001B
:1034A00004F0C8FD01283FF4C2AD594607F1E4001D
:1034B00004F0C0FD02287FF421AEB8E53F480121A9
:1034C00003F032F901307FF44DADBB6C013BFB647E
:1034D000FB6B013B3B65D7F88430C7F8B4307B6E9B
:1034E0003B673B6C7B653DE5594607F1E4000024F2
:1034F00004F0A0FD00283FF42AAE594607F1E4008D
:1035000004F098FD01287FF42AAEB7F8C030002BF4
:103510007FF422AE2A4B1A78234B1B6803EB8203FD
:103520002046196ED3F834901A6EC7F8C820D3F825
:103530008C800DF00FF80CF069FCD7F8C820044619
:103540000D46484611460DF005F80CF05FFC0246AA
:103550000B46204629460CF0DBFD044640460D464E
:103560000CF054FC02460B46204629460CF0A6FC03
:103570000CF09CFF5946044607F1E40004F05AFDA4
:1035800001287FF4ECAD0E4B1A78074B1B686432B0
:1035900003EB8203204659680CF0DCFF0446DEE5AD
:1035A0000000024068D801004C8EFF1F1CCC0100B7
:1035B00084D1010081D30100BCD80100A8C0010062
:1035C000349DFF1F5A4607F5A671504604F01EFDB4
:1035D000D7F8D41007F5FA7004F036FD07F5DE7859
:1035E0000146404608F02AFFBB49404608F0AAFFC2
:1035F000002843D13B6F002B40D17B6B002B00F0A8
:103600005182B64802F010FF07F5DE731868B44B1C
:10361000002808BF184602F007FFB24802F004FF76
:10362000B14802F001FF5A4607F5A671504604F072
:10363000EDFC012107F5FA7004F006FD02F0F4FE3E
:10364000A84802F0F1FEA949404608F07BFF054674
:10365000002800F00282A64802F0E6FE07F5867315
:103660005B68002B00F0F381DB68013B5B4540F0B9
:10367000EE81A04802F0D8FE01237B634FF4C853CB
:10368000013BFDD1404608F09DFE5EE4D7F8C8300E
:10369000D7F8A82003EB4202043A043B07F55F7118
:1036A00053F8040F21F8020B9342F9D1AFE4012340
:1036B000009307F5AE753B6F7A6E95E80300FEF751
:1036C00031F96B68002B3FF49DAC002507F5DE71E6
:1036D000C7F860B0C7F85C90D7F8B4B0D7F81C90C2
:1036E000C7F890102A46DB689A4229DAD7F890008A
:1036F00007F5AE7104F08AFC002107F5DE7004F0D6
:10370000A3FC01465046FEF7FDFEDAF80000DAF8A9
:103710001480FDF781FC04FB09B3D7F8C420B8F18D
:10372000010F42F8230004F101039BB20DDC1C469B
:1037300007F5AE7301355B68ADB22A46002BD2D1D6
:10374000D7F860B0D7F85C905CE4DAF80400C7F80A
:103750008C30FDF761FCD7F88C30D7F8C42003FB20
:1037600009B3B8F1020F42F8230004F102039BB23F
:10377000DDD0DAF80800C7F88C30FDF74DFCD7F83B
:103780008C30D7F8C42003FB09B3B8F1030F42F81B
:10379000230004F103039BB2C9D0DAF80C00C7F888
:1037A0008C30FDF739FCD7F88C30D7F8C42003FBF8
:1037B00009B3B8F1040F42F8230004F104039BB2EB
:1037C000B5D0DAF81000C7F88C30FDF725FCD7F833
:1037D0008C30D7F8C42003FB09B3053442F823002A
:1037E000A4B2A5E7D7F8AC105A46504604F00EFC38
:1037F000DAF80430002B00F01D81DB68C7F8943044
:10380000994607F5DE78C7F8C89007F5E6750024F5
:10381000C1465A4607F59271504604F0F7FB21461F
:1038200007F5FA7004F006FC5A4645F8040B07F554
:103830009671404604F0EAFB2146484604F004FC39
:10384000014607F5FA7008F0F9FD254BDAF800009B
:10385000002808BF1846FDF7DFFB013407F5FA70B2
:1038600008F0B0FD0A2CD4D1D7F8C890BBF1000FF6
:1038700000F09280594607F58A7004F0E5FB014696
:1038800007F5FA7008F0DAFDDAF80000002800F019
:103890000D81FDF7C1FB0DF053F9BB6D98420FD0C0
:1038A000154B421E9A4200F2FB8000EB40021201CF
:1038B000013A232AB86503D91049114808F062FC7F
:1038C00007F5FA7008F07EFD00240023C7E92E34C6
:1038D000FFF772BA0B4C32E4ACC601008CCE01008B
:1038E00068D8010090CE01004CD5010014C9010038
:1038F00094CE01004CCE01005755550585140000AB
:103900003C9DFF1F643F1C4EC34B1A78C34B1B6882
:1039100003EB82032046D3F81011D3F8E490D3F8D8
:103920001021C7F8C820D3F83C810CF013FE0CF02E
:103930006DFAD7F8C82004460D46484611460CF0EB
:1039400009FE0CF063FA02460B46204629460CF0AD
:10395000DFFB044640460D460CF058FA02460B4683
:10396000204629460CF0AAFA0CF0A0FD5946044660
:1039700007F1E40004F05EFB01287FF4F0ABA64BF6
:10398000A64A1B7812687033204652F823100CF0B8
:10399000E1FD0446FFF7E3BB594607F58A7004F0E2
:1039A00053FB014607F5FA7008F048FDDAF800000D
:1039B000002800F0B581FDF72FFB0DF0C1F8B865C8
:1039C000B96D974B4A1E9A423FF67AAF01EB41021E
:1039D0001201013A232A7FF673AF6DE77B69002B52
:1039E0007FF7B1A919468F4802F09EFE02F0C8FC8D
:1039F00000283FF4ADA98B48012102F095FE01306B
:103A00007FF4A6A9BB6C013BFB647B6E3B67FB6B41
:103A10003B65BB697B653B6B002B7FF49DA90093E5
:103A200007F5AA7393E803007A6E3B6FFDF77AFF00
:103A3000FFF792B9D7F8D490C7F89490E1E604F074
:103A4000F9FA08FB00F209EB0229FFF79FB8764864
:103A500002F0EAFC01237B6310E67449404608F05B
:103A600071FD002800F06E81714808F0D5FB6D48AB
:103A7000294602F059FE6F4802F0D6FCB96D684B3A
:103A80004A1E9A423FF6EAAD01EB41021201013AA9
:103A9000232A7FF6E3AD6849654808F073FBDDE54E
:103AA000B8650DE7654802F0BFFCAAE56448FDF77C
:103AB000B3FA0DF045F8F0E66248D7F8041207F5BE
:103AC000FA7302F01FFD002E32DDD7F8D030D7F8A0
:103AD000B820DFF874B1DFF8749102FB03F500241D
:103AE00005EB08022346C7F8D4200DE05AF822005F
:103AF0000CF08CF9013402460B46A4B2484602F0A1
:103B000001FDA642234613DD984505EB0302EDD1E6
:103B1000D7F8D4305AF823000CF078F90134024673
:103B20000B46A4B2584602F0EDFCA6422346EBDC5D
:103B3000D7F8D030D7F8C82001339BB20132C7F88C
:103B4000D030D7F8C43092B29A42C7F8C820FFF6F6
:103B500041ACD7F8C03001339AB207F5AE73C7F85D
:103B6000C0205B68002B7FF417AC394802F05CFC86
:103B7000D7F88030002B77D1BB6A002B40F3E0836D
:103B8000BA6ED7F88040334EDFF89C80D7F8649047
:103B9000151F9B4613E00CF093FD014650460CF0B8
:103BA00097FE002102F0E4FCFB6AA342404601D0EC
:103BB00002F03AFC631C9B4500F020811C4655F83E
:103BC00004AF314650460CF08BFF02464846002AAF
:103BD000E1D10CF075FD014650460CF079FE042150
:103BE00002F0C6FCE0E71748D7F8001207F5FA73B1
:103BF00002F088FC67E71348D7F8F41107F5FA7369
:103C000002F080FC5FE70F48D7F8FC1107F5FA7364
:103C100002F078FC57E700BF349DFF1F4C8EFF1F5A
:103C200057555505A8C00100D0C9010098CE010024
:103C30003C9DFF1FA0CE01008514000080CE010036
:103C400068D80100F0CE010048CE0100CCC90100C7
:103C5000E0CE0100000048437E48D7F8F81107F590
:103C6000FA7302F04FFC2EE7DFF8EC8107F55F7680
:103C7000002407F1FC050EE036F8020B02F08CFC84
:103C80000021284604F0D6F9431EA342404601D045
:103C900002F0CAFB01340021284604F0CBF9A0420F
:103CA000EADC6E4802F0C0FBBB697A6D93423EDCF1
:103CB000FB6B3A6D013B934239DCBA69796D8A42FC
:103CC00000F049833C6D28220134002107F5E6709D
:103CD0003C6510F0F3FE07F5C67008F073FBFB6B54
:103CE000D7F808D0A3423EF790AD7B6D01337B65DA
:103CF0003A6CD7F810D09A423EF734ADFC6802F027
:103D000011FBBB6CFA6C013B934200F33C83FB6CF0
:103D1000BA6C01339A42FB647FF770ABFEF71ABDB1
:103D20004F48FDF779F90CF00BFFB86548E64A48B3
:103D300002F07AFB7B68002BC4DD1946494802F08B
:103D4000F3FCBFE74849404608F0FCFB0546002865
:103D500040F0BE824549404608F0F4FB00283FF49D
:103D60007DAC434808F058FA3E492A46962307F5A9
:103D7000FA7002F087FC3F4802F056FB07F5FA7034
:103D800002F052FB3C4877E63C48DFF8D490DFF87D
:103D9000F080DFF8F0B002F047FB04F1FF3A0025B5
:103DA00007F5CE762946304604F04EF9014607F570
:103DB000FA7008F043FBD7F8F441002C08BF4C46DA
:103DC000204607F5FA73FDF727F90CF01FF80B46AC
:103DD00002462146404602F095FBAA451E4808BF10
:103DE000584602F021FB07F5FA7008F0EBFAD7F815
:103DF000D4300135AB42D5D1FFF7BABAFA2009F079
:103E000019FAFB6E012B7FF44CAF7B6C1E48DFF878
:103E100048801D1F02F008FB786E0CF051FC4FF03B
:103E20000009064600E0994655F8040F31460CF0AB
:103E30004FFD002102F09CFBFB6A4B45404601D040
:103E400002F0F2FAA14509F10103ECD1FA2009F0E0
:103E5000F1F926E7F0CE0100D0C9010050D10100F0
:103E600068D80100A8C00100A8CE0100BCCE0100A6
:103E70003C9DFF1F4CD50100C4CE0100C8CE0100FF
:103E8000D4CE0100DCCE0100F8CE010013467A62E8
:103E9000C348C7F8843015464FF0FF32BB62FA6260
:103EA00002F0C2FAD7F8C830002B3EF489AEBD4804
:103EB0001FFA8AF102F026FBD7F8D030012B7EF4EE
:103EC00084AEB948B94E02F0AFFA0024B84B1B6873
:103ED00004F10C0203EB8203013458680BF096FFE7
:103EE00002460B46304602F00DFB0A2CEED1B04BD9
:103EF000AE4E1B68D86D0BF089FF02460B46AD48ED
:103F000002F000FBAC4802F08FFA0024A84B04F149
:103F100018021B6853F822000BF078FF01340246A8
:103F20000B46304602F0EEFA0A2CEFD1A04B9F4E22
:103F30001B68D3F888000BF069FF02460B469D48CA
:103F400002F0E0FA9D4802F06FFA0024984B1B68DB
:103F500004F1380203EB8203013458680BF056FF7A
:103F600002460B46304602F0CDFA0A2CEED1904BB9
:103F70008E4E1B68D3F80C010BF048FF02460B462F
:103F80008C4802F0BFFA8E4802F04EFA0024884BAB
:103F900004F144021B6853F822000BF037FF013490
:103FA00002460B46304602F0ADFA0A2CEFD1804BA8
:103FB0007E4E1B68D3F838010BF028FF02460B46F3
:103FC0007C4802F09FFA7F4802F02EFA0024784BDA
:103FD0001B6804F1220203EB8203013458680BF0E2
:103FE00015FF02460B46304602F08CFA0A2CEED141
:103FF0006F4B6E4E1B68D3F8B4000BF007FF024600
:104000000B466C4802F07EFA6F4802F00DFA00246D
:10401000674B04F12E021B6853F822000BF0F6FEEA
:10402000013402460B46304602F06CFA0A2CEFD1FE
:104030005F4B5E4E1B68D3F8E0000BF0E7FE0246D4
:104040000B465C4802F05EFA604802F0EDF900248D
:10405000574B1B6804F14E0203EB8203013458688E
:104060000BF0D4FE02460B46304602F04BFA0A2C07
:10407000EED14F4B4D4E1B68D3F864010BF0C6FEDA
:1040800002460B464B4802F03DFA514802F0CCF98B
:104090000024474B04F15A021B6853F822000BF02E
:1040A000B5FE013402460B46304602F02BFA0A2CCC
:1040B000EFD13F4B3D4E1B68D3F890010BF0A6FEAD
:1040C00002460B463B4802F01DFA424802F0ACF9AA
:1040D0000024374B1B6804F1640203EB82030134B4
:1040E00058680BF093FE02460B46304602F00AFA7F
:1040F0000A2CEED12E4B2D4E1B68D3F8BC010BF0D1
:1041000085FE02460B462B4802F0FCF9324802F0CD
:104110008BF90024264B04F170021B6853F822002F
:104120000BF074FE013402460B46304602F0EAF909
:104130000A2CEFD11E4B1D4E1B68D3F8E8010BF083
:1041400065FE02460B461B4802F0DCF9234802F0EC
:104150006BF90024164B1B6804F17A0203EB82030F
:10416000013458680BF052FE02460B46304602F00E
:10417000C9F90A2CEED10E4B0C4E1B68D3F8140271
:104180000BF044FE02460B460A4802F0BBF9144805
:1041900002F04AF90024064B04F186021B6821E074
:1041A00030CE010034CE0100BCC90100CCC90100F1
:1041B0004C8EFF1F48CE0100DCC90100E8C9010098
:1041C000F8C9010008CA01001CCA010030CA010078
:1041D00048CA01005CCA01006CCA01007CCA010027
:1041E0008CCA010053F822000BF010FE0134024685
:1041F0000B46304602F086F90A2CCCD1674B684E4C
:104200001B68D3F840020BF001FE02460B466548DE
:1042100002F078F9644802F007F900245F4B1B684C
:1042200004F1900203EB8203013458680BF0EEFDB9
:1042300002460B46304602F065F90A2CEED1574B88
:104240001B68D3F86C020BF0E1FD02460B465548A3
:1042500002F058F9FEF7B9BC002B3FF489A8DB68DF
:10426000C7F8D430FFF77FB8504907F1DC0003F0FE
:104270003BFF03F0BBF8FEF75ABD7A6AB96A9408AF
:1042800000209C4600290DDD00231A4600FB04F5A2
:1042900001332A449BB24FF0000E8B4246F822E0D5
:1042A0001A46F5DB013083B26345EBD3FEF7EABC77
:1042B00007F1D803C7F878C0C7F8C430FEF7E2BCEE
:1042C0003B4907F1DC0003F00FFFB863FEF731BB99
:1042D0003848394D07F0A0FF02E001333FF4CBAB83
:1042E0000021284602F020FA01280346F5D1334880
:1042F00002F09AF8BB6C013BFB64FB6B013B3B6536
:10430000D7F88430C7F8B4307B6E3B673B6C7B6575
:10431000FFF7B4BB03F07CF8FEF701BD284802F0BC
:10432000F1F802F083F902F003F9FFF77DB8BBF171
:10433000000FC8BFC7F8D4303EF7C5AFFFF718B8B5
:10434000FA2008F077FFFB6E012B7FF4AAAC1D4822
:1043500002F06AF87AE53A6D93427FF4B3AC1A48FA
:1043600002F062F8AEE4194802F05EF807F59560D5
:1043700002F05AF8164802F057F802F057F902F026
:10438000D7F8FFF751B8134802F04EF8002C3FF46D
:10439000BEAC2146084802F0C7F9B8E44C8EFF1FB6
:1043A000CCC9010048CE01009CCA010070CE0100BA
:1043B0002CCD01003C9DFF1FA8C00100B0CE010024
:1043C000ACC80100F8CE0100A4CE01004CCB010026
:1043D00088CB0100D0C9010030B5012887B030D0AA
:1043E000002002F065FE0928014620DD1C4B1A68FA
:1043F000136814681068156892680592C4F307443E
:104400000094C0F30720174C174A0391EDB21749E7
:1044100001901B0E16480295049402F073F815489B
:1044200002F002F807B0BDE8304002F0FFB81248D1
:1044300002F068F802F0FAF807B0BDE8304002F088
:1044400077B80E48002102F06FF9054B1B681A6817
:1044500082420B4A18BF18605378DB07FCD5BFE7D0
:104460004C8EFF1FB4C9010010C9010018C901001A
:104470000CCF010084D10100ACC80100A8C001002C
:104480000000024038B50D4D0D4C0021284607F0C4
:10449000D5FF22460B4928460BF04EFB4FF0FF316B
:1044A000094803F017FC09480949802300250371D6
:1044B00022460560BDE838400BF03EBB649DFF1FFF
:1044C000408EFF1FC5C300007C9DFF1F3C9DFF1F4A
:1044D000791400002DE9F04FC1B033AEC749312344
:1044E0004FF4FA72304602F0CDF8304611F068FF12
:1044F0003746054600240CE017F8010B0EF00CFAC5
:10450000034628B9304607F8013C11F059FF05462B
:104510000134AC42F0D3022D49D99DF8CC4020465D
:104520000EF072F9002800F01186A4F13003092B77
:1045300040D8304611F058FAB14B984201F025842A
:104540003FD8B04B984201F03C8440F2CF81AE4B53
:10455000984201F0DF8140F22481AC4B984201F097
:104560000C8240F28E80AA4B984200F0BA8703F189
:104570003E7303F54A7398421FD102F02BFAA54C03
:10458000A54802F033F84FF4802532210220FBF7D2
:104590006FFFFBF79BFF40F2EE20656408F04AFED8
:1045A00000210220A564FBF763FFFBF78FFF41B0FA
:1045B000BDE8F08F002C40F04185984801F0A2FF43
:1045C000F5E7974B984200F0E5813ED9954B98422C
:1045D00001F0B78240F26082934B984201F01C8355
:1045E00040F23F82914B984200F01686904B9842E1
:1045F00040F0A981814DDFF83CA28F4C0021284674
:1046000002F078F80BF00AFF461C0746CFD00021D5
:10461000284602F06FF8DAF8006006EB870680465D
:104620008946706B0BF0F2FB42464B460BF0AEFE38
:1046300020B9404649460BF039FF70636378D807CC
:10464000DCD46378D807F9D5D8E77C4B984201F0E1
:10465000588240F2C4837A4B984201F06E8240F255
:10466000A583784B984201F05F8003F18E5303F5E8
:10467000852303F23E53984240F06883FDF7D2FC55
:1046800095E7A3F1CE63A3F5CF33A03B984200F0AA
:10469000F9856D4B984240F0E5805848002102F0C2
:1046A00029F80BF0BBFEC4B20021204608F066FDDD
:1046B000204608F01DF801F0A3FFC82008F0BAFD5D
:1046C000204608F015F801F09BFFC82008F0B2FD65
:1046D000204608F00DF801F093FFC82008F0AAFD6D
:1046E000204608F005F801F08BFFC82008F0A2FD75
:1046F000204607F0FDFF01F083FFC82008F09AFD77
:10470000204607F0F5FF01F07BFFC82008F092FD7E
:10471000204607F0EDFF01F073FFC82008F08AFD86
:10472000204607F0E5FF01F06BFFC82008F082FD8E
:10473000204607F0DDFF01F063FFC82008F07AFD96
:10474000204607F0D5FF01F05BFFC82008F072FD9E
:10475000204607F0CDFF01F053FFC82008F06AFDA6
:10476000204607F0C5FF01F04BFFC82008F062FDAE
:10477000204607F0BDFF01F043FFC82008F05AFDB6
:10478000204607F0B5FF01F03BFFC82008F052FDBE
:10479000204607F0ADFF01F033FFC82008F04AFDC6
:1047A00005E72A4B984200F038861CD9284B9842DE
:1047B00000F01484274B98427FF4FFAE264801F0A6
:1047C00015FF0E48002101F095FF0BF027FE0A218E
:1047D000024601234FF47A70019000911846072198
:1047E000FCF792FFE3E61D4B984200F0B5841C4BAA
:1047F00098425CD102F03AFAD9E600BFA8C00100A5
:10480000EC767A6172F2602D72682150B6D60B5C3C
:10481000C40CD95C00F00F4010D20100B4D20100EA
:10482000467A9BB914E6E5D6EC9415F9A617FDFA7D
:10483000A699F4FF4C8EFF1F00000240EC80039409
:104840005E3A62A132EABEA526324A56B23CD33E57
:1048500032DE364EEA500A50BCD10100C60DA030FF
:1048600040FED935BB4B98427FF4A7AEBA4801F061
:10487000DBFD02F0AFF8002101220846FBF728FE1D
:10488000B64801F0D1FD002102220846FBF720FEC8
:10489000B34801F0C9FD002103220846FBF718FECA
:1048A000B04801F0A3FE0120FFF796FD7FE6AE4B76
:1048B00098427FF482AE02F08DF8AC4CAC4801F027
:1048C00095FE4FF480254B210920FBF7D1FDFBF726
:1048D000FDFD656440F2EE2008F0ACFC00210920EB
:1048E000A564FBF7C5FDFBF7F1FD60E6A14B98421F
:1048F00000F0548740F29A809F4B984200F0578511
:104900005ED99E4B984200F0F1839D4B984239D17D
:1049100002F060F8954C9B4801F068FE4FF480254A
:104920004B210420FBF7A4FDFBF7D0FD656440F2AA
:10493000EE2008F07FFC00210420A564FBF798FD21
:10494000FBF7C4FD33E6904B98427FF436AE02F09D
:1049500041F8864C8D4801F049FE4FF480254B21EB
:104960000620FBF785FDFBF7B1FD656440F2EE2004
:1049700008F060FC00210620A564FBF779FDFBF739
:10498000A5FD14E6A3F17373A3F5E333BE3B984290
:104990007FF413AE00217E4801F0C6FE7D49A0F5EC
:1049A0009C42213A8A4201F248827B4A7B4B126840
:1049B0009168814218BF90605A78D107FCD5F6E51E
:1049C000774B984200F0C685764B98427FF4F5AD60
:1049D0006F4DDFF8C4A1714C0021284601F08AFE1A
:1049E0000BF01CFD421C07463FF4E1AD00212846B8
:1049F00001F080FEDAF8006006EB87068046894603
:104A0000D6F8F4020BF002FA42464B460BF0BEFC1D
:104A100028B9404649460BF049FDC6F8F4026378D0
:104A2000DB07D9D46378DB07F9D5D5E740F24C43EF
:104A300098423FF4BCAD40F23C815B4B984200F0A1
:104A4000258340F22781594B98427FF4B6AD584BED
:104A500018680BF0DBF902460B46564801F052FD90
:104A6000A5E5554B984200F06486544B984240F0BF
:104A7000BB80534801F0D8FC0021524801F054FE9D
:104A800001460446504801F03DFD204601F008FC77
:104A90004E4801F0ABFD8AE54D4B984201F0158080
:104AA00035D94C4B984200F099854B4B98427FF496
:104AB00084AD374DDFF8E0A0384C0021284601F0E6
:104AC00019FE0BF0ABFC411C07463FF470AD002112
:104AD000284601F00FFEDAF8006006EB87068046F4
:104AE0008946D6F83C010BF091F942464B460BF053
:104AF0004DFC28B9404649460BF0D8FCC6F83C01AD
:104B00006378DA07D9D46378DA07F9D5D5E7334B78
:104B1000984200F05183324B984240F0848001F07B
:104B200059FF124C2F4801F061FD4FF480253221CE
:104B30000320FBF79DFCFBF7C9FC656440F2EE2007
:104B400008F078FB00210320A564FBF791FCFBF73C
:104B5000BDFC2CE512609552BCCF0100C4CF010012
:104B6000CCCF0100D4CF0100EC6CF12E00F00F404F
:104B700048D201004D4B6720C232F92332E2B72BF5
:104B8000EC05482D20D20100ECFBBEFA30D201002A
:104B9000A8C00100DE8E6D004C8EFF1F0000024099
:104BA000645AEC22DEFD7123A673000F7026571A9B
:104BB000349EFF1F8CD2010090D721F1C28D5CF38F
:104BC00058D2010068D201006CD2010080D20100ED
:104BD000ECF135C8B64ED9C9C2DCA8D6E2D765BC5F
:104BE000EC8A8CC618D20100C64B98427FF4E5AC23
:104BF00001F0F0FEC44CC54801F0F8FC4FF48025EC
:104C000032210A20FBF734FCFBF760FC656440F2BC
:104C1000EE2008F00FFB00210A20A564FBF728FC1A
:104C2000FBF754FCC3E4A3F14B63A3F57E23A3F687
:104C30002A2398427FF4C1ACB54DDFF8D8A2B64C18
:104C40000021284601F056FD0BF0E8FB431C074607
:104C50003FF4ADAC0021284601F04CFDDAF80060CD
:104C600006EB870680468946D6F810010BF0CEF891
:104C700042464B460BF08AFB28B9404649460BF0AA
:104C800015FCC6F810016378DE07D9D46378DE0717
:104C9000F9D5D5E7A14B984200F09C81A04B9842F2
:104CA0007FF48BAC9F4801F0BFFB9F4801F09EFC56
:104CB0007DE440F20543984200F28781B0F57A7FA7
:104CC000FFF47BACA0F57A701D283FF676AC01A30B
:104CD00053F820F0A54C0000BB450000BB45000088
:104CE000BB450000BB450000BB450000BB450000C4
:104CF0001F57000029570000BB450000BB450000BE
:104D0000BB450000BB450000BB450000BB450000A3
:104D1000BB450000BB450000BB450000BB45000093
:104D2000BB450000BB450000BB450000BB45000083
:104D3000BB450000BB450000BB450000BB45000073
:104D400033570000BB4500004F4A0000774B9842A4
:104D50007FF433AC764801F049FC40F6B83008F0F7
:104D600069FA01F05FFE734801F040FC40F6B8308C
:104D700008F060FA01F06CFE6F4801F037FC40F675
:104D8000B83008F057FA01F051FE6C4801F02EFCE3
:104D900040F6B83008F04EFA01F01CFE40F6B8308C
:104DA00008F048FA664801F021FC00E403F177437B
:104DB00003F56D0303F6FA33984200F0B08403F173
:104DC000F27303F5C6437033984261D101F002FEDD
:104DD0005C4801F029FBFBF7CBFBFFF7E8BB5A4B24
:104DE000984200F04D871BD9584B984200F04583FC
:104DF00003F13A6303F52F3303F2531398427FF420
:104E0000DCAB53484FF4165107F002F9514B93E8CD
:104E100003000B0C2990ADF8A8108DF8AA3024E1FE
:104E20004D4B984200F05E824C4B984240F0988087
:104E3000384C3748002101F05DFC256806460F46D6
:104E400068690AF0E3FF32463B460BF09FFA002800
:104E500001F00780304B5A78D007FCD52C48002150
:104E600001F048FC26680D460446706A0AF0CEFF41
:104E700022462B460BF08AFA20B9204629460BF031
:104E800015FB7062244B5A78D107FCD5FFF78FBB16
:104E9000A3F1B263A3F5AA33A3F5AB7398427FF4F1
:104EA0008CAB1C4C1A48002101F024FC25680646F6
:104EB0000F46A8690AF0AAFF32463B460BF066FA95
:104EC000002800F0C787144B5A78D207FCD5104849
:104ED000002101F00FFC26680D460446B06A0AF076
:104EE00095FF22462B460BF051FA20B92046294661
:104EF0000BF0DCFAB062084B5A78D707FCD5FFF705
:104F000056BB00BF6C5038EC00F00F4050D201008F
:104F1000A8C001004C8EFF1F00000240B5185A01C6
:104F200050662C0518C90100B4CF010073966DA21C
:104F3000FCCF01001CD0010040D0010060D0010076
:104F400080D00100DCCF0100E0DE087E271E1D823C
:104F50003494FF1F50D30100F27ACA7272DEE172FC
:104F6000A3F10B73A3F5886398427FF426ABC14D80
:104F7000DFF804A3C14C0021284601F0BBFB0BF075
:104F80004DFA411C07463FF412AB0021284601F0C0
:104F9000B1FBDAF8006006EB870680468946D6F852
:104FA00044020AF033FF42464B460BF0EFF928B9B2
:104FB000404649460BF07AFAC6F844026378DA07AD
:104FC000D9D46378DA07F9D5D5E740F23643984269
:104FD0007FF4F3AAFCF7D2F8FFF7E9BADFF894926E
:104FE000DFF894A2A54C0021484601F083FB0BF0AA
:104FF00015FAB0F1FF3F80463FF4D9AA0021484698
:1050000001F078FBDAF8005005EB880506460F46FC
:10501000D5F818020AF0FAFE32463B460BF0B6F914
:1050200028B9304639460BF041FAC5F818026378C2
:10503000D807D8D46378D807F9D5D4E79DF8CD2020
:10504000002A00F0E4819DF8CE50002D40F0378317
:1050500044F2AE3303FB02F00130DAE129A8072164
:1050600009F04EF8322008F0E5F809F0F5F80028CC
:10507000F4D00B2402E0322008F0DCF809F0ECF860
:10508000062800F35E83013CF5D156E3DFF8E49196
:10509000DFF8E4A1794C0021484601F02BFB0BF02E
:1050A000BDF9B0F1FF3F80463FF481AA0021484698
:1050B00001F020FBDAF8005005EB880506460F46A4
:1050C000D5F88C000AF0A2FE32463B460BF05EF9A2
:1050D00028B9304639460BF0E9F9C5F88C006378F9
:1050E000DD07D8D46378DD07F9D5D4E7DFF88491FC
:1050F000DFF884A1614C0021484601F0FBFA0BF077
:105100008DF9B0F1FF3F80463FF451AA0021484697
:1051100001F0F0FADAF8005005EB880506460F4674
:10512000D5F8EC010AF072FE32463B460BF02EF940
:1051300028B9304639460BF0B9F9C5F8EC01637867
:10514000DD07D8D46378DD07F9D5D4E74C4801F002
:10515000D9F941B0BDE8F08FDFF81891DFF818A158
:10516000464C0021484601F0C5FA0BF057F9B0F162
:10517000FF3F80463FF41BAA0021484601F0BAFADF
:10518000DAF8005005EB880506460F46D5F8B8005A
:105190000AF03CFE32463B460BF0F8F828B93046A0
:1051A00039460BF083F9C5F8B8006378D807D8D42E
:1051B0006378D807F9D5D4E7DFF8B890DFF8B8A05E
:1051C0002E4C0021484601F095FA0BF027F9B0F17A
:1051D000FF3F80463FF4EBA90021484601F08AFAE0
:1051E000DAF8005005EB880506460F46D5F8680149
:1051F0000AF00CFE32463B460BF0C8F828B93046A0
:1052000039460BF053F9C5F868016378DB07D8D449
:105210006378DB07F9D5D4E7DFF85890DFF858A0BA
:10522000164C0021484601F065FA0BF0F7F8B0F192
:10523000FF3F80463FF4BBA90021484601F05AFADF
:10524000DAF8005005EB880506460F46286E0AF08E
:10525000DDFD32463B460BF099F820B93046394621
:105260000BF024F928666378D907DAD46378D90774
:10527000F9D5D6E7A8C001004C8EFF1F0000024000
:1052800098CF0100DFF83093DFF830A3CC4C002139
:10529000484601F02FFA0BF0C1F8B0F1FF3F80460D
:1052A0003FF485A90021484601F024FADAF80050BD
:1052B00005EB880506460F46D5F894010AF0A6FDD1
:1052C00032463B460BF062F828B9304639460BF0BF
:1052D000EDF8C5F894016378DF07D8D46378DF0769
:1052E000F9D5D4E7B44DDFF8D482B54C0021284677
:1052F00001F000FA0BF092F8431C06463FF457A960
:105300000021284601F0F6F9D8F8007007EB86076F
:1053100082468B46D7F870020AF078FD52465B460B
:10532000B6000BF033F828B9504659460BF0BEF8DA
:10533000C7F870026378DF07FCD50021284601F02A
:10534000D9F9D8F80070374482468B46D7F89C02CA
:105350000AF05CFD52465B460BF018F828B950463F
:1053600059460BF0A3F8C7F89C026378D807FCD520
:105370000021284601F0BEF9D8F800301E448246CC
:105380008B46D6F8C8020AF041FD52465B460AF049
:10539000FDFF28B9504659460BF088F8C6F8C802F8
:1053A0006378D907A2D46378D907F9D59EE7DFF8E7
:1053B0000892DFF808A2824C0021484601F09AF9D1
:1053C0000BF02CF8B0F1FF3F80463FF4F0A800212D
:1053D000484601F08FF9DAF8005005EB88050646DB
:1053E0000F46D5F8E4000AF011FD32463B460AF0BC
:1053F000CDFF28B9304639460BF058F8C5F8E4001F
:105400006378DA07D8D46378DA07F9D5D4E744F2B9
:10541000AE3004FB00F0FFF78FB8DFF89C91DFF8A7
:105420009CA1674C0021484601F064F90AF0F6FFA0
:10543000B0F1FF3F80463FF4BAA80021484601F092
:1054400059F9DAF8005005EB880506460F46D5F8FD
:10545000C0010AF0DBFC32463B460AF097FF28B950
:10546000304639460BF022F8C5F8C0016378DE07F4
:10547000D8D46378DE07F9D5D4E701F0ABFA514808
:1054800001F0B4F84C48002101F034F904464E48CC
:105490000D4601F0ABF84848002101F02BF9064613
:1054A0000F46204629460AF0B9FF394604463046E1
:1054B0000AF0B4FF454D01464FF480262046FAF726
:1054C000D7FFFBF703F86E644FF47A7007F0B2FE73
:1054D00000212046AE64FAF7CBFFFAF7F7FFFFF79B
:1054E00066B801F077FADFF8E880384E05274FF408
:1054F0008025404600F098FF384601F081F80024EE
:10550000204601F07DF821463846FAF7B1FF0A340B
:10551000FAF7DCFF75644FF4487007F08BFEC82C77
:10552000B564EDD1204601F06BF821463846FAF714
:105530009FFF3234FAF7CAFF75644FF4487007F0E2
:1055400079FEB4F5FA6FB564ECD101370A2FD0D1EA
:10555000FFF72DB81F4DDFF88090DFF8708001F065
:1055600039FA0FCD29AC27460FC40FCD0FC495E8EB
:10557000030084E8030057F8044B4846214600F036
:10558000C1FF4FF4802532212046FAF771FFFAF768
:105590009DFF4FF4FA70C8F8445007F04BFE2046C8
:1055A0000021C8F84850FAF763FFFAF78FFFBE42B0
:1055B000E1D1FEF7FCBF00BFA8C001004C8EFF1F69
:1055C0000000024054D1010088D1010000F00F40DA
:1055D000F4D1010028D30100FCD1010001F0FAF957
:1055E000C24EC34C24AB9C46129329AB1F46139367
:1055F0000FCEACE80F0056F8043BCCF800300FCECD
:105600000FC733683B6001250E2001F0EFFEDDF887
:105610004890139F4FF0000859F8046B4FF0140B9B
:1056200059463046FAF724FFFAF750FF97F800A0E2
:1056300054F83A204FF4967082F8805007F0FAFD43
:105640000BF10A0B54F83A20BBF5827F82F8005127
:10565000E6D14FF4FA713046FAF70AFFFAF736FF4F
:1056600054F83A204FF4967082F8805007F0E2FD2B
:1056700054F83A204FF44871304682F80051FAF756
:10568000F7FEFAF723FF54F83A204FF4967082F8A9
:10569000805007F0CFFD54F83A300021304683F8AF
:1056A000005108F10108FAF7E3FEFAF70FFFB8F12D
:1056B000050F66D0B8F1040F68D00437ACE79DF849
:1056C000CF70002F00F00F819DF8D080B8F1000F4F
:1056D00000F006819DF8D190B9F1000F00F0AA8387
:1056E0009DF8D210002900F0A2839DF8D330002B42
:1056F00000F09A830DF1D300FBF7E6FE034603FBAF
:1057000001114B1C03FB09F3013303FB08F30133C5
:1057100007FB03F3013305FB03F301339AE4002095
:10572000FEF75AFEFEF743BF0120FEF755FEFEF7D7
:105730003EBF08F0E3FF08F0A3FD08F08DFD002850
:10574000F9D108F09DFD08F09BFD08F099FD08F0E7
:1057500097FD08F095FD08F093FD08F091FD9DF888
:10576000A7309DF8A8404FF47A7004EB032407F0AB
:1057700061FD6048214600F0C5FE08F013FBFEF70E
:1057800016BF41F2707007F055FD3DE74FF41670FB
:1057900007F050FD0E2001F029FE8EE729AB139390
:1057A00017AF24AB544D1293BB464FF47A71534854
:1057B00000F0BAFF14900120FAF7D2FE0AF080FF41
:1057C0000646002002F0D4FC0446002002F0D0FC83
:1057D000014620460AF0C0FE0446002002F0C8FC44
:1057E000014620460AF0B8FE45490BF071F8139ABD
:1057F000129907461FA802F007FD1BAA594616A8D2
:1058000003F0F0FFC82007F015FD4FF47A7800246C
:10581000112006F06DFFB8F101080444F8D1012011
:1058200007F008FD7621284602F068FA284602F0C3
:1058300049FB8046284602F051FB8146284602F08B
:1058400047FB8246284602F04FFB0346304615933D
:105850000AF0DCFA2B4B0A4601460E46384617463C
:1058600083FB0421E217C2EBA1120A921B9A109249
:10587000179A0F92169A0E92299A0D92249A0C92C8
:105880001F9A0B920AF0C2FA159BCDE9080118463F
:105890000AF012FF1C490BF01BF80AF0B7FACDE929
:1058A00006011A4950460BF013F80AF0AFFACDE999
:1058B000040148460AF0AAFACDE9020140460AF07E
:1058C000A5FA3B46CDE900013246114800F01AFE28
:1058D00000F0ACFE149B01337FF467AFFEF767BEA8
:1058E00044F2AE3314E744F2AE3314E758D3010068
:1058F000BCD80100A0D201007C9DFF1FA8C0010000
:1059000000004040D34D621000007A440000C842BD
:10591000B4D00100CE4CCF48002100F0EBFE25684A
:1059200006460F4628690AF071FA32463B460AF0ED
:105930002DFD20B9304639460AF0B8FD2861C64B26
:105940005A78D507FCD5C348002100F0D3FE26685D
:105950000D460446306A0AF059FA22462B460AF0F0
:1059600015FD20B9204629460AF0A0FD3062BA4B49
:105970005A78D407FCD5FEF71ABEB84CDFF8E0829F
:1059800001F028F80FCC1FAE0FC654F8043B33606B
:105990000FCC24AD0FC517AF23682B60002138460C
:1059A00006F04CFD40F2145007F044FC0DF1900A53
:1059B0001FABAC4C13930DF1A40BCDF848A0139B77
:1059C00053F804AB139314254FF0010929465046B0
:1059D000FAF74EFDFAF77AFD129B1E7854F836203E
:1059E0004FF4FA7382F8809041460022584600F046
:1059F00049FE0146384606F087FD4146384606F026
:105A000083FD0A3554F83630B5F5827F83F800916E
:105A1000DCD1129B4FF4FA71043350461293FAF71B
:105A200027FDFAF753FD54F83630002283F88090B2
:105A300041464FF4FA73584600F024FE01463846BA
:105A400006F062FD4146384606F05EFD54F83630F9
:105A50004FF4487183F800915046FAF709FDFAF7C0
:105A600035FD54F83630002283F8809041464FF4DB
:105A7000FA73584600F006FE0146384606F044FD2B
:105A80004146384606F040FD54F83630504683F81B
:105A900000910021FAF7ECFCFAF718FD724938463C
:105AA00006F032FD139B24AA934288D139461BA8E5
:105AB00006F06AFC1BA800F08FFD1BA806F082FC14
:105AC000384606F07FFCFEF772BD00F083FF674C9E
:105AD000674800F08BFD4FF480254B210820FAF732
:105AE000C7FCFAF7F3FC656440F2EE2007F0A2FB76
:105AF00000210820A564FAF7BBFCFAF7E7FCFEF7E3
:105B000056BD00F067FF594C5A4800F06FFD4FF446
:105B100080254B210520FAF7ABFCFAF7D7FC65642A
:105B200040F2EE2007F086FB00210520A564FAF77D
:105B30009FFCFAF7CBFCFEF73ABD01F08BFBFEF7BA
:105B400036BD00F047FFDFF83081484E01274FF4A3
:105B50008025404600F068FC384600F051FD0024E6
:105B6000204600F04DFD21463846FAF781FC053409
:105B7000FAF7ACFC75644FF47A7007F05BFB322CDB
:105B8000B564EDD1204600F03BFD21463846FAF7DA
:105B90006FFC0A34FAF79AFC75644FF47A7007F0D8
:105BA00049FBB4F5967FB564ECD10137052FD0D110
:105BB00031482E4E00F038FC0A2000F021FD002470
:105BC0004FF48025204600F01BFD21460A20FAF7FD
:105BD0004FFC0534FAF77AFC75644FF47A7007F0DD
:105BE00029FB322CB564EDD1204E4FF480252046A0
:105BF00000F006FD21460A20FAF73AFC0A34FAF7CB
:105C000065FC75644FF47A7007F014FBB4F5967F69
:105C1000B564ECD1FEF7CBBC00F0DCFE134C1748AA
:105C200000F0E4FC4FF4802532210120FAF720FC3B
:105C3000FAF74CFC656440F2EE2007F0FBFA002115
:105C40000120A564FAF714FCFAF740FCFEF7AFBC9C
:105C50004C8EFF1FA8C001000000024058D3010075
:105C6000D0C90100BCD8010048CB010000F00F40B2
:105C700040D2010028D20100F4D1010008D2010075
:105C80007B48002100F036FD0AF0C8FBC4B20021B9
:105C9000204607F073FA204607F062FA00F0B0FCE5
:105CA000C82007F0C7FA204607F05AFA00F0A8FC0F
:105CB000C82007F0BFFA204607F052FA00F0A0FC17
:105CC000C82007F0B7FA204607F04AFA00F098FC1F
:105CD000C82007F0AFFA204607F042FA00F090FC27
:105CE000C82007F0A7FA204607F03AFA00F088FC2F
:105CF000C82007F09FFA204607F032FA00F080FC37
:105D0000C82007F097FA204607F02AFA00F078FC3E
:105D1000C82007F08FFA204607F022FA00F070FC46
:105D2000C82007F087FA204607F01AFA00F068FC4E
:105D3000C82007F07FFA204607F012FA00F060FC56
:105D4000C82007F077FA204607F00AFA00F058FC5E
:105D5000C82007F06FFA204607F002FA00F050FC66
:105D6000C82007F067FA204607F0FAF900F048FC6F
:105D7000C82007F05FFA204607F0F2F900F040FC77
:105D8000C82007F057FAFEF712BC00F023FE394C8A
:105D9000394800F02BFC4FF480254B210720FAF7FF
:105DA00067FBFAF793FB656440F2EE2007F042FAD6
:105DB00000210720A564FAF75BFBFAF787FBFEF7E3
:105DC000F6BB2E4C2A48002100F094FC25680646BC
:105DD0000F46E8680AF01AF832463B460AF0D6FA4F
:105DE00020B9304639460AF061FBE860244B5A7806
:105DF000D707FCD51E48002100F07CFC26680D4624
:105E00000446F0690AF002F822462B460AF0BEFA70
:105E100020B9204629460AF049FBF061184B5A7810
:105E2000D607FCD5FEF7C3BB44F2AD3367E444F2BA
:105E3000AE3367E444F2AE3367E4104B114A1B689B
:105E40009968914218BF9A600D4B5A78D207FCD5D9
:105E5000FEF7ADBB304639460AF028FBA861FFF7D4
:105E600032B8304639460AF021FB6861FEF7F2BFCE
:105E7000A8C0010000F00F4038D201004C8EFF1F77
:105E800000000240A0680600174B1B68996844F6A2
:105E90001F62914210B517DD9968144A914213DCD4
:105EA00000F0D6FE01E001F0C5F800F091FA431CC5
:105EB0000446F8D003F0B6FA5B2C0FD0FEF70AFBCD
:105EC000BDE8104000F034BB094A9968914218BF00
:105ED0009A60084A5378D907FCD5E1E7FCF7A6FB9E
:105EE000BDE8104000F024BB4C8EFF1F00DD6D00AC
:105EF000A06806000000024038B5174C0D200121B3
:105F000007F03CF904F109051A2001E014F8010F2B
:105F1000002107F033F9AC42F8D10121062007F047
:105F20002DF90E4B1022C3F8C4200121202007F0C8
:105F300025F90021222007F021F90021232007F074
:105F40001DF90021242007F019F9BDE8384000218F
:105F5000252007F013B900BF8DD3010000F00F40DA
:105F600008B500F063FD1A4B1B6893F81024012A52
:105F700020D0042000F094F94FF4E13000F0E2FB6F
:105F800000F028FD41F2883007F054F9FFF7B4FF24
:105F9000104804F097FF06F03BFC06F0CDFE002110
:105FA00005F0BAF80C4800F03FFABDE808400B488D
:105FB00000F01CBB93F8102432B9094A5378DB0770
:105FC000FCD500F067FFD4E7002283F81024F4E743
:105FD0004C8EFF1F3CA0FF1F18C90100B4CF010069
:105FE0000000024010B50024E0B20021013407F0A7
:105FF000C5F8212CF8D110BD0278002A37D02DE940
:10600000F8431B4E1B4FDFF8709004464FF000081A
:1060100002E014F8012FD2B131684B1C142B7A54D2
:10602000336016D0D9F80050002DF2D1002BF0D0FB
:106030003846FD5410F0C4F90146384607F0B8FB65
:1060400007F03EFC14F8012F3560002AE4D1BDE8CA
:10605000F883384687F8148010F0B2F901463846C4
:1060600007F0A6FB07F02CFCC6F80080D1E77047CC
:10607000749FFF1F789FFF1F989FFF1F2DE9F04F10
:10608000644BD3F800808FB0B8F1000F00F0AA8005
:10609000614BDFF888911B6808F1010E41331EF057
:1060A000FF0009F8083000F0B080484449464FF638
:1060B000FF7211F8013B83EA122383EA131444EAC6
:1060C0000223620182EA04329BB2534081429AB2B7
:1060D000EFD1100BC2F30321C2F3031302F00F023E
:1060E00038336B444B4D0493DFF834C1DFF834A1EF
:1060F000DFF828B14C4F02F13803383038310DEB5E
:106100000304684408F10603694402900391019373
:106110002B60BCE80F00059409AC0FC40298DCF8B2
:1061200000302370039910F8143C09F80E3009EB85
:10613000080311F8142C9A70049A059C12F8142C78
:10614000DA704FF0040014F8142C1A715871019B86
:10615000364D4FF0000209F80320002601E007F059
:10616000E7FB07F0D1FB0028F9D1DAF800300BB1DA
:10617000002E45D05846FFF73FFF2D4B1B686BB1F3
:106180002C4A0024D454104610F01AF9014629482C
:1061900007F00EFB07F094FB254B1C602B68079360
:1061A000079C03E007F00AFC01301ED12B6808931E
:1061B000089B1B1BF92BF5D93B6801360133052ED3
:1061C0003B60CED1144C1C492368013381FB032171
:1061D000DA17C2EBE1021A2000FB12330D4A2360EA
:1061E000002111600FB0BDE8F08F07F0A1FB04465D
:1061F00007F0E4FB0130F8D1E4B2062CDCD1E1E792
:1062000009EB0800FFF7F8FEB7E70F221346114627
:10621000104665E7749EFF1F709FFF1F789EFF1F4B
:1062200098D30100548EFF1F6C9FFF1F00A1FF1F1A
:10623000749FFF1F789FFF1F4FECC44E03783BB342
:10624000F0B5144D144F154E83B0441C04E0EA2AF7
:1062500016D014F8013BCBB1042BFAD02968306872
:106260007B544A1C2A600028F1D0002201A88DF836
:1062700005208DF80430FFF7BFFE2A68EA2AE8D12E
:10628000FFF7FCFE14F8013B002BE5D103B0F0BD95
:10629000704700BF749EFF1F789EFF1F548EFF1F24
:1062A0000428044A044B12BF00210121032011607D
:1062B00018607047909FFF1F508EFF1F2DE9F0411F
:1062C000134D144EDFF85080144F07F01DFB0446A9
:1062D000B8B908F0E3FF2B78002BF6D03378DB0752
:1062E000F3D5D8F800303A689B1A0E2BEDD908F098
:1062F0009DFE0028E9D00A4B1C60BDE8F04108F083
:1063000059BE074B0122BDE8F0411A6007F010BBEF
:1063100010A3FF1F34A3FF1F00A1FF1F38A3FF1FFF
:10632000949FFF1F2DE9F041114D124EDFF8488078
:10633000124F01E0FFF7C2FF08F0B0FF2B7803F027
:10634000FF0473B1347814F001040AD0D8F8003097
:106350003A689B1A0E2B4FF0000402D908F066FE33
:10636000044607F0D1FAE042E4D1BDE8F08100BF75
:1063700010A3FF1F34A3FF1F00A1FF1F38A3FF1F9F
:1063800010B508F08BFF0E4B1B7803F0FF0473B1C0
:106390000C4B1C7814F0010409D00B4B0B4A1B6802
:1063A00012689B1A0E2B06D908F040FE044607F02F
:1063B000ABFA204410BD07F0A7FA0024204410BD1A
:1063C00010A3FF1F34A3FF1F00A1FF1F38A3FF1F4F
:1063D00008B507F099FA18B1BDE8084007F0EEBA21
:1063E00008F05CFF0C4B1B7853B10C4B1B78DB07A0
:1063F00006D50B4B0B4A1B6812689B1A0E2B02D852
:106400004FF0FF3008BD08F011FE0028F8D0BDE8BD
:10641000084008F0F3BD00BF10A3FF1F34A3FF1F07
:1064200000A1FF1F38A3FF1F38B52E4B1B68044681
:10643000002B2FD02C4B1B688BB12C4B1B6820469C
:1064400033B9FFF7D9FD2046BDE8384003F016B850
:10645000FFF7F4FE2046BDE8384003F00FB808F01F
:106460001DFF234B1B78002BEDD0224B1B78D80748
:10647000E9D5214B214A1B6812689B1A0E2BE2D9E1
:10648000002CE0D020460FF09BFF0146204608F08C
:10649000FFFDD8E708F002FF154B1B78C3B1154B81
:1064A0001B78D90714D5144B144A1B6812689B1A21
:1064B0000E2B0DD9124D2B68DA070BD554B120469F
:1064C0000FF07EFF0146204608F0E2FD2B6801E058
:1064D0000B4B1B689B07B6D5044B1B682046002B53
:1064E000AFD0B5E7909FFF1F949FFF1F989FFF1F9E
:1064F00010A3FF1F34A3FF1F00A1FF1F38A3FF1F1E
:10650000508EFF1F0FB400B5B5B036ABC82153F89D
:10651000042B009301A80DF009FF002301A88DF8BA
:10652000CC30FFF781FF35B05DF804EB04B0704765
:106530000C4B1B6870B58BB90B4C236803B970BD4D
:106540000A4D00262846EE540FF03AFF0146284631
:1065500007F02EF907F0B4F9266070BDFFF78EFD45
:10656000EAE700BF989FFF1F749FFF1F789FFF1FE0
:1065700010B590B00C4609F049FC064ACDE900017F
:106580002346322103A80FF0CDFF03A8FFF74CFFED
:1065900010B010BDACD3010000B58FB00346054A62
:1065A000322101A80FF0BEFF01A8FFF73DFF0FB099
:1065B0005DF804FBB4D3010000B58FB00346054A73
:1065C000322101A80FF0AEFF01A8FFF72DFF0FB099
:1065D0005DF804FBB8D30100034B0068002808BF36
:1065E0001846FFF721BF00BF68D8010008B5FFF7C4
:1065F0001BFFBDE808400148FFF716BF10C70100A8
:1066000000B58FB00346074A322101A80FF08AFF78
:1066100001A8FFF709FF0448FFF706FF0FB05DF878
:1066200004FB00BFB4D3010010C7010070B502F035
:1066300001FF02F0C5FEFFF7F7FE0E48FFF7F4FE7C
:106640000D4B1B689BB90D4C236863B10C4D0026A4
:106650002846EE540FF0B4FE0146284607F0A8F88D
:1066600007F02EF92660BDE8704002F0DBBEFFF7B0
:1066700005FDE8E710C70100989FFF1F749FFF1FEB
:10668000789FFF1F2DE9F04FDFF8648083B09946B3
:10669000D8F800300093009D82468B4617460024B0
:1066A000D8F800300193019E17B1731BBB4215D877
:1066B000FFF78EFE013018D0FFF700FEC5B2294665
:1066C00058460FF095F948B90AF804500134B9F169
:1066D000000F01D04C4501D23546E1E7002350467A
:1066E0000AF8043003B0BDE8F08F30BFD8E700BF30
:1066F00000A1FF1F00B589B00A461823014601A872
:10670000FFF7C0FF9DF8043023B90649002009B007
:106710005DF804FB01A800210BF0BCFB09B05DF89B
:1067200004FB00BF0000F87F00B589B00A461823BB
:10673000014601A8FFF7A6FF01A80FF0BFF909B0B5
:106740005DF804FB2DE9F047164D174C2E68174FE6
:10675000DFF85C90824640F2EE2808F09FFD237837
:1067600073B13B78DB070BD52B68D9F800209B1A57
:106770000E2B05D951460F48BDE8F04705F0D0BBB8
:106780002B6822789B1B2AB1B3F5FA6FF2D808F078
:1067900085FDE2E74345FAD951460648BDE8F04792
:1067A00005F0BEBB00A1FF1F10A3FF1F34A3FF1FF6
:1067B00038A3FF1F2094FF1FB0F90020B1F900306B
:1067C0009A4205D001DD012070474FF0FF3070473D
:1067D0000020704702680B689A4205D001DD012055
:1067E00070474FF0FF3070470020704790F9241039
:1067F000124B03604B1C1FD070B4114D55F8213063
:10680000834201D070BC70470E4E56F8213043B120
:106810004FEA810C002403EB0C0253685460002BF8
:10682000F9D1094A002346F8213045F82130137880
:10683000013B137070BC7047704700BF24D5010046
:10684000A8A0FF1F84A0FF1FA5A0FF1F704700BFC7
:1068500090F92430581C00F0B6802DE9F04F5A4AC8
:1068600085B052F8232000928A465849DBB20B705B
:10687000002A00F08B809B000293D346009A92F886
:106880002530002B7AD0136851491B688B4240F0A9
:10689000968092F92430591C70D04B4AD9B252F8E4
:1068A00023704A4B1970002F68D08B000193DA4691
:1068B00097F82530002B5BD03B68454A1B68934214
:1068C00079D197F92490B9F1FF3F51D03E4B53F85D
:1068D00029B03E4B5FFA89F983F80090BBF1000FB5
:1068E00046D003974FEA89095F4697F82530002B79
:1068F00037D03B68364A1B68934252D197F924300F
:106900005A1C2ED0304A5FFA83F852F823502F4B8E
:1069100083F800802DB34FEA880895F82530E3B15D
:106920002B682B4A1B68934233D195F92460731C62
:1069300013D0254B53F82640244BF6B21E7064B199
:10694000B60094F825302046514613B123681B68E1
:10695000984734446468002CF3D145446D68002D99
:10696000DBD107EB090BDBF80470002FBDD1039FCF
:10697000019B1F447F68002F9AD1D346009B029A47
:1069800013445B680093002B7FF478AF05B0BDE83B
:10699000F08F28464544514698476D68002DBCD17C
:1069A000DFE707EB090B384651469847DBF80470E0
:1069B000002F9AD1DBE7514638469847D8E7009830
:1069C00059469847DAE7704784A0FF1FA4A0FF1F2D
:1069D0005168000010B50121022006F0CFFB104ADB
:1069E000002001214FF4A074C2F8C4100023834298
:1069F00002D000BF0133FAE7C2F8C81020460138C0
:106A0000FDD1262B03F10200EED1C2F8C4104FF4E1
:106A10007A7006F00FFCBDE81040F9F71DBD00BF0D
:106A200000F00F400021022006F0A8BB08B51F208F
:106A3000012106F0A3FB054B0122C3F8C8204FF447
:106A40007A70BDE8084006F0F5BB00BF00F00F40CB
:106A500000211F2006F092BB70B50A4B0E4615466A
:106A6000042204460FF076F8304609F029FE294644
:106A700009F07AFE08F0ECFC0AF03CF854F820002B
:106A800070BD00BFD567000070B50A4B0E461546B5
:106A9000022204460FF05EF8304609F011FE294646
:106AA00009F062FE08F0D4FC0AF024F834F9100072
:106AB00070BD00BFB96700002DE9F04F87B00B1E15
:106AC00005936DDD4FF0000A4FF0000BA0F10208B6
:106AD000CDE900AB08EB4303994654465D46364B7F
:106AE00000225046594609F033F8824638F9020F21
:106AF0008B4609F079F902460B46CDE9022322467E
:106B00002B4609F023F852465B4606460F4609F02D
:106B1000FFFA02460B462046294609F019F80446BA
:106B20000D4622462B46DDE9020109F00FF83246F8
:106B30003B4609F0C3F902460B46DDE9000109F0C6
:106B400007F8C145CDE90001C9D1059B581E09F0E0
:106B50004BF902460B46DDE9000109F0D9FA08F0CD
:106B60009BFC02460B4604460D4608F0F1FF08F078
:106B7000A7FD0FA3D3E9002309F0CAFA02460B468A
:106B800000200E4908F0E2FF02460B460C48FFF7D2
:106B9000B9FC2046294609F089FC07B0BDE8F08F12
:106BA00000230024CDE90034CFE700BFAFF300801D
:106BB00000000000432EE63F0000F03F00002E40A2
:106BC000BCD3010070B503780446C3B1002102466E
:106BD0008C4606E05D2B08BF0CF1FF3C12F8013F2C
:106BE00053B17B2B1BD016D85B2BF3D112F8013F8E
:106BF0000CF1010C002BF4D15CEA010C11D15D21E8
:106C000020460BF00BFF054658B140780BF08CFE88
:106C100048B9012070BD7D2BE0D10139DEE701319B
:106C2000DCE7002070BD6E1C02F0FCFB311B20462F
:106C300002F006FC02F0FEFB02F0C2FB0822314625
:106C40000BF0F2FD0028ECD16870012070BD00BF90
:106C5000044A054B126882B00192019A1A6002B090
:106C6000704700BF00A1FF1F9C9FFF1F4FF0E02354
:106C7000014AC3F80C2D70470400FA05002900F002
:106C800083802DE9F04F4B4FDFF82C9181B0054602
:106C90009B460C4604EB82035E689300002E4AD0AC
:106CA000F118D1F80480B8F1000F32D008EB0301DD
:106CB000D1F804A0BAF1000F18D0534428465968FF
:106CC0005B46FFF7DBFF9AF825307BB1DAF800303E
:106CD0005B68BB4267D19AF92420531C06D059F84F
:106CE00022105046D2B25B46FFF7C8FF98F8253015
:106CF0007BB1D8F800305B68BB4250D198F92420B2
:106D0000551C06D059F822104046D2B25B46FFF718
:106D1000B5FF96F8253073B133685B68BB423AD152
:106D200096F92420501C06D059F822103046D2B2D1
:106D30005B46FFF7A3FF94F8253013B323685B6825
:106D4000BB4222D194F92420511C1AD059F8225068
:106D5000BDB1D2B205EB8203204659685B46FFF70E
:106D60008DFF95F8253063B12B685B68BB421ED15F
:106D700095F92420531C04D059F82240D2B2002C9B
:106D800088D101B0BDE8F08F70475946204601B068
:106D9000BDE8F04F1847304659469847CBE7404684
:106DA00059469847B5E75046594698479EE7594691
:106DB0002846ECE7BD6D000084A0FF1F90F9242059
:106DC000531C54D02DE9F041304E56F82250002D7E
:106DD0004BD0D2B205EB82030C465F6893008FB3B1
:106DE000F918D1F80480B8F1000F18D0434459685D
:106DF0002346FFF743FF98F8253083B1D8F80030D9
:106E0000234A5B6893423CD198F92420501C06D059
:106E100056F822104046D2B22346FFF72FFF97F8CC
:106E200025307BB13B681A4A5B68934225D197F9BC
:106E30002420511C06D056F822103846D2B22346E0
:106E4000FFF71CFF95F825307BB12B68104A5B6873
:106E500093420DD195F92420531C06D056F82210E8
:106E60002346D2B22846FFF709FFBDE8F0817047FC
:106E700021462846BDE8F041184738462146984744
:106E8000E0E7404621469847C9E700BF84A0FF1FBE
:106E9000BD6D0000014804F061B900BFA49FFF1F51
:106EA00070B58EB006F044FD041E28DD642006F0A7
:106EB000C1F90DF103050DF1290605F8014F06F0A2
:106EC00037FDB5420446F8D1002411498DF82A4017
:106ED000252201A80BF0A8FC10B901200EB070BD4E
:106EE0000C48FFF7A1FA0A48FFF79EFA0A48FFF795
:106EF0009BFA01A8FFF798FA20460EB070BD07482C
:106F0000FFF792FA0648FFF78FFA00200EB070BD27
:106F1000D0D30100F8D3010018D4010038D4010007
:106F20006CD4010010B5104C23680121D3F8840003
:106F300004F076FB23680121D3F8840004F0F8FD07
:106F400023681021D3F8840004F0B8FC23680321DF
:106F5000D3F8840004F09AFB23680321BDE81040B5
:106F6000D3F8840004F090BDA09FFF1F70B50121ED
:106F70000646212006F002F9294B102098600021D6
:106F800006F0FCF8FFF7CEFF4FF41653013BFDD19E
:106F900064240025102005F0ABFB013C0544F9D129
:106FA000D6B9204BA3FB05356C090021212006F042
:106FB000E5F8204609F080FB4FF05E5109F0D4FB64
:106FC000194909F0D1FB194909F0CEFB184909F01C
:106FD0007FFC09F08FFD70BD4FF496610920F9F731
:106FE00047FA012006F026F90D4A4FF480214FF4AC
:106FF0007A535164013BFDD16425102005F078FBE4
:10700000013D0444F9D1074B054A4FF48021A3FB0D
:107010000434916405202946C440F9F729FAC4E7ED
:1070200000F00F401F85EB51C3F5983F00007A44F4
:1070300013E9813E00B5184B18491B68184A0968C6
:10704000126883B00193019B5B1A93420BD8002016
:10705000FFF78CFF09F034FB124909F023FD10B94A
:1070600003B05DF804FB104803F06AFF06F060FA15
:107070000021022006F082F800211F2006F07EF891
:10708000FEF7B0FF4FF47A7006F0D4F8074803B06B
:107090005DF804EB04F062B800A1FF1F9C9FFF1F86
:1070A000F49FFF1F000060403CA0FF1FA49FFF1F34
:1070B00038B50446FFF75AFFF4B9164C164D09F0DF
:1070C000FFFA294609F046FA214609F001FC134966
:1070D00009F04AFB0021044609F0F8FC4FF07C510E
:1070E00068B1204609F038FA09F004FD6428A8BF09
:1070F000642020EAE07038BD094C0A4DDFE72046E5
:1071000009F028FA09F0F6FC6428A8BF642020EAF8
:10711000E07038BD00002F4400C05A450000C8424E
:107120000000484400805445F8B504461646C1B9ED
:10713000184F3B680D46D3F884002322222104F027
:107140007BFD002E0CDD043C3B682322D3F8840039
:10715000222104F071FD0135AE4244F8040FF3D151
:10716000F8BD0C4F3B682522D3F88400242104F09D
:1071700063FD002EF4DD043C00253B682522D3F896
:107180008400242104F058FD0135AE4244F8040F78
:10719000F3D1F8BDA09FFF1F2DE9F04F234B244EE4
:1071A0001A68244B92681B682349DFF890A0DFF827
:1071B0009090DFF8908083B030460193224B019C81
:1071C0001A604FF0200B0C605A46204C40F804AB7C
:1071D00000210DF073FC0025FF274A46414630464A
:1071E00086F8255086F8265086F8247008F0A4FC0E
:1071F00020465A46294640F804AB0DF05FFC4A464B
:10720000414684F8247084F8255084F8265020469E
:1072100008F092FC942005F081FC044604F0D2F9B9
:107220000B4B1C6003B0BDE8F08F00BF4C8EFF1FFE
:10723000A49FFF1F00A1FF1F9C9FFF1F24D50100DB
:10724000408EFF1FED670000F49FFF1FCC9FFF1FC4
:10725000A09FFF1F2DE9F0475248534D534C544F08
:10726000DFF85091CCB0FFF7DFF800234EF6602234
:10727000514901A8FFF706FA4EF660214E48FFF784
:1072800053FA012182460D2005F078FF2E6840F266
:10729000EE2808F003F82378002B71D03B78DB0749
:1072A0006ED52B68D9F800209B1A0E2B68D943485D
:1072B000514604F035FE01210D2005F02BFF4FF45F
:1072C0007A7005F0B7FF02213D4806F071FA4FF4DD
:1072D0007A7005F0AFFF0A213A4806F069FA4FF4D8
:1072E0007A7005F0A7FF0C21374807F0D1FE40F275
:1072F000D241364805F028F83548062106F058FAFC
:1073000040F2D2412D4805F01FF84FF47A7005F095
:1073100091FF0D212F4807F0BBFE01A80FF050F898
:10732000014601A807F0B4FE07212B4806F040FAF9
:1073300001A80FF045F8014601A806F039FA4FF40C
:107340007A7005F077FF1321244807F0A1FE244846
:10735000082106F02DFA4FF47A7005F06BFFFFF765
:107360009FFDD0B900210D2005F0D4FE1D48FFF788
:107370005BF8FFF75BF9FFF7DBF84CB0BDE8F0878F
:107380002B6822789B1B2AB1B3F5FA6F8FD807F0D0
:1073900085FF7EE74345FAD989E71348FFF744F8AC
:1073A000E0E700BF94D4010000A1FF1F10A3FF1F5E
:1073B00034A3FF1F38A3FF1FA8C001002094FF1FA4
:1073C000A4D40100A8D40100B4D401007095FF1F1B
:1073D000C4D40100CCD40100DCD40100E4D4010009
:1073E000F8D401000CC9010004D5010038B5C4B2BD
:1073F0000021204605F0C2FE4FF44865204605F006
:10740000AFFE2B46013BFDD10028F7D038BD00BFB1
:107410002DE9F04F0A2487B0112005F069F9013CED
:10742000112005F065F9A4B2112005F061F9002CD6
:10743000F2D1112005F05CF90446112005F058F94D
:10744000034611201C4405F053F9984B204483FB5C
:107450000023A3EBE07009F033F9954B1D68044657
:10746000D5F82C802F6BE86A296B09F039FB0028CE
:1074700040F089808F4EDFF840A233680293414686
:10748000384609F067F84FF07D51804609F06CF9F5
:10749000029B019307464FF0000925463AE005F0AC
:1074A00027F90546112005F023F9034611201D4454
:1074B00005F01EF97D4B284483FB0023A3EBE0700D
:1074C00009F0FEF80546962005F0B4FE2146284650
:1074D00009F040F851468346404609F045F9014617
:1074E000584609F0DFFA4946002845D1284609F0F8
:1074F000CFFA724900283FD1284609F0C9FA47F26D
:107500003052002838D133680593059B01995B1AE6
:10751000934231D82146284609F01CF839460546E1
:1075200009F0C0FA03461120002BB8D1394628468D
:1075300009F0D6FA00B3DFF87481112005F0D8F80D
:107540000546112005F0D4F80544112005F0D0F8C7
:1075500006463544962005F06DFE88FB0520A0EB1D
:10756000E57009F0ADF8214608F0F4FF0146384611
:1075700009F098FA0028E0D14FF4967007B0BDE802
:10758000F04F05F057BE4B4E296BE86A3368029303
:1075900008F0E0FF4FF07D51804609F0E5F8029BCE
:1075A000DFF814A1019307464FF0000925463AE0A1
:1075B00005F09EF80546112005F09AF803461120C3
:1075C0001D4405F095F8394B284483FB0023A3EBB9
:1075D000E07009F075F80546962005F02BFE294667
:1075E000204608F0B7FF51468346404609F0BCF8F4
:1075F0000146584609F056FA49460028BCD12846AB
:1076000009F046FA2D490028B6D1284609F040FA7B
:1076100047F230520028AFD133680393039B01999E
:107620005B1A9342A8D82946204608F093FF3946B2
:10763000054609F037FA03461120002BB8D1284639
:10764000394609F04DFA68B3DFF86090DDF804A020
:1076500047F230580BE0962005F0ECFD2946204615
:1076600008F078FF0146384609F01CFAD0B1112025
:1076700005F03EF80546112005F03AF805441120C2
:1076800005F036F8284489FB0023A3EBE07009F0ED
:1076900017F833680493049BA3EB0A03434505469C
:1076A000D9D969E707B0BDE8F08F00BF56555555E9
:1076B0004C8EFF1F00A1FF1FCDCC4CBE00FF7F47AB
:1076C00070B54FF4165188B004463148314D04F07E
:1076D0009FFC314B93E8030008330A0C0490ADF88B
:1076E000141093E803008DF816202A6802920B0C00
:1076F000029E8DF81E302B680193019B0690ADF819
:107700001C100AE006F0FCFC322005F093FD2B680B
:107710000393039B9B1BA34233DC06F09DFD0346B2
:10772000072104A8002BEDD003E00A2C24DC05F08F
:1077300081FD06F091FD062804F101044FF03200AE
:10774000F3DD0DF117040DF11E0506F099FD04F8A7
:10775000010FA542F9D19DF81B309DF81C4004EBA8
:10776000032406F01FFB204608F0A6FF09F0E8F905
:1077700008B070BD06F084FD06F06EFD0028F9D15A
:10778000DFE70648FEF750FE0548FEF74DFED0E75E
:107790003494FF1F00A1FF1F50D5010030D5010018
:1077A000D0C90100082870B504D840F097804FF484
:1077B000304301E04FF440434B4D4C4C2B800121B2
:1077C0000A2005F0DBFC4A4AE37A1268D3B172B6AC
:1077D000E37AD90708D54FF0E020E668D0F88011A9
:1077E0003140C0F88011A1619E0708D54FF0E0201C
:1077F0002669D0F884113140C0F88411E16158073E
:1078000062D462B62368D9688A4207D039491960C0
:10781000DA6042F08041384A19611A6000210A207A
:1078200005F078FC236829884FF00042DA620A0AE2
:107830005A63DA6A002AFCDA4FF00042C9B2986B48
:10784000DA625963DA6A002AFCDA01210A209B6BAA
:1078500005F060FCC023013BFDD100210A2005F0AA
:1078600059FC298823684FF000400A0AD8625A63FD
:10787000DA6A002AFCDA4FF00042C9B2986BDA6289
:107880005963DA6A002AFCDA01210A209B6B05F0B1
:1078900041FCC023013BFDD1E37AA3B1D90704D554
:1078A0004FF0E022A169C2F800119A0704D54FF009
:1078B000E022E169C2F804115B0704D54FF0E02330
:1078C000226AC3F8082170BD4FF0E0216069D1F849
:1078D000883103402362C1F8883192E7074B43EABD
:1078E00040239BB268E700BFFC9FFF1F3CA0FF1F27
:1078F000F89FFF1F01403F0000003F8000C0FFFFD6
:1079000030B4A023013BFDD13A493B4ACB7A1268FF
:10791000D3B172B6CB7ADC0708D54FF0E024CD683E
:10792000D4F8800128408861C4F88001980708D500
:107930004FF0E0240D69D4F884012840C861C4F8F0
:1079400084015D074BD462B60B68D868904207D0BB
:107950002A4D2B481D6042F08044DA601C6118609B
:10796000284A2948B2F800C01024C0F888404FEADD
:107970001C224FF00040D8625A63DA6A002AFCDA0F
:10798000986B4FF00044C0B25FFA8CF2DC620002E8
:107990005A63DA6A002AFCDA9B6B1B4ADBB21024BA
:1079A0001843C2F88440A023013BFDD1CB7AA3B198
:1079B000DC0704D54FF0E0228C69C2F800419A0739
:1079C00004D54FF0E022CC69C2F804415B0704D52E
:1079D0004FF0E0230A6AC3F8082130BC70474FF02B
:1079E000E0204C69D0F8883123400B62C0F8883120
:1079F000A9E700BF3CA0FF1FF89FFF1F01403F0009
:107A000000003F80FC9FFF1F00F00F4008B50021E1
:107A1000FFF7C8FE064A1021C2F888106023C2F89A
:107A20008410013BFDD1BDE80840FFF769BF00BFEE
:107A300000F00F40014B024A1A607047F89FFF1F89
:107A4000000001B805F0F6BB2DE9F0471E4E96F98F
:107A500000305A1C074628D0DFF870A0DFF870907D
:107A6000072500244FF0010801E096F90030D8B254
:107A7000002105F04FFB08FA05F19AF800003940A3
:107A800005F048FB3078012105F044FB640099F8CB
:107A90000000E4B2013D05F063FB08B144F00104CD
:107AA0006B1CE2D12046BDE8F0870A4A12684FF00D
:107AB0000043D3625063D36A002BFCDA946BE4B2C8
:107AC0002046BDE8F08700BF00A0FF1FFF9FFF1FFB
:107AD000FE9FFF1F3CA0FF1F2DE9F041DFF8E4806F
:107AE0000F4600211D460646144605F013FB98F983
:107AF0000030013316D03846FFF7A6FF3DB12544CC
:107B00000020FFF7A1FF04F8010BAC42F8D198F96F
:107B1000003001333BD03046012105F0FBFA002054
:107B2000BDE8F081284BDA7A1AB372B6DA7AD00758
:107B300008D54FF0E02CD868DCF88011014099613D
:107B4000CCF88011910708D54FF0E02C1869DCF8CB
:107B500084110140D961CCF88411520708D54FF047
:107B6000E0205969D0F888210A401A62C0F88821BB
:107B700062B61B68154AD9689142BCD01449196095
:107B8000DA6002F180421A61124A1A60B3E70E4BC2
:107B9000DA7A002ABFD0D00704D54FF0E0219869E7
:107BA000C1F80001910704D54FF0E021D869C1F870
:107BB00004015207AFD54FF0E0221B6AC2F808312A
:107BC000A9E700BF00A0FF1F3CA0FF1F0320033850
:107BD00001403F0000003F802DE9F041DFF8E080E8
:107BE0000F460021144606461D4605F093FA98F903
:107BF0000020013215D03846FFF726FF35B1254465
:107C000014F8010BFFF720FFAC42F9D198F90030CE
:107C100001333BD03046012105F07CFA0020BDE85D
:107C2000F081284BDA7A1AB372B6DA7AD00708D51F
:107C30004FF0E02CD868DCF8801101409961CCF855
:107C40008011910708D54FF0E02C1869DCF88411F9
:107C50000140D961CCF88411520708D54FF0E020DB
:107C60005969D0F888210A401A62C0F8882162B6A2
:107C70001B68154AD9689142BDD014491960DA6071
:107C800002F180421A61124A1A60B4E70D4BDA7AA7
:107C9000002ABFD0D00704D54FF0E0219869C1F881
:107CA0000001910704D54FF0E021D869C1F8040123
:107CB0005207AFD54FF0E0221B6AC2F80831A9E79E
:107CC00000A0FF1F3CA0FF1F0320033801403F001E
:107CD00000003F8010B4064C0177FF222270054956
:107CE000054C0A702270002210BC026102757047B8
:107CF000FF9FFF1F00A0FF1FFE9FFF1F70B50446E0
:107D000090F91C006175421C86B041D00121C0B2BF
:107D100005F000FA207F012105F030FA264B93F997
:107D20000000431C2DD00121C0B205F027FA234BDF
:107D30000121187805F022FA214B0021187805F06E
:107D40001DFA257F1F4820490023204AA06684F899
:107D5000215084F82230E166226704F1200000F00F
:107D6000BFFD90B91A491B4BA16501204FF00132AC
:107D700084F85E0022612075236684F8640006B0F2
:107D800070BD154803F09EF8DBE7002006B070BD1B
:107D9000124B0493124A002301260393029301938A
:107DA0000093059610690D46517B1A4602F0B0F813
:107DB0000C480D493346C8E700A0FF1FFF9FFF1F77
:107DC000FE9FFF1FD97A0000D97B0000457A000092
:107DD00002040302400196003CA0FF1FA0860100A0
:107DE00010A0FF1F457F0000F97E000030B5837CA6
:107DF00004460122407C84F8642087B00BB140F037
:107E00000400E37C0BB140F00200237C0BB140F096
:107E10001000237D0BB140F0C80004F12005294675
:107E200000F0E4FE18B10025284607B030BD284612
:107E300000F088FE0028F6D129460DF1020001F07D
:107E4000D7F8BDF80200400005F0F4F9294601A872
:107E500001F008F90028E6D1637C0BB3BDF90800F6
:107E600008F02EFC144908F033FDA37C2060EBB130
:107E7000049808F021FC114908F02AFDE37CA06079
:107E800093B1039808F018FC257D606055B19DF80A
:107E90000430DB060CD5059808F00EFCE060C3E763
:107EA0000748E2E70125BFE70548EDE70448E5E7B5
:107EB0000023E360B8E700BF0000C84200007A4436
:107EC0000000C07F10B50446FFF790FF206810BD8A
:107ED00010B50446FFF78AFF606810BD10B5044670
:107EE000FFF784FFA06810BD10B50446FFF77EFFC2
:107EF000E06808F025FE10BD70B5044682B0104859
:107F00000E4621461D46144602F008F90C4831463B
:107F100001F056FD45B10A4E254414F8011B3046C8
:107F200001F04EFDAC42F8D105480024427B0169C6
:107F30000094012302F0FCFB204602B070BD00BF9C
:107F400010A0FF1F2DE9F0411B4D82B08846064668
:107F5000014628461F46144602F0E0F841462846EE
:107F60004FF0000801F02CFD6A7B2969CDF80080F4
:107F70000123284602F0DCFBCDF804804FF0010815
:107F8000697B2869CDF800803246FBB202F0F2FB33
:107F9000C0B2B8420CD1261830B1286902F004FCF6
:107FA00004F8010BB442F8D1002002B0BDE8F08122
:107FB000404602B0BDE8F08110A0FF1FC0E90012EA
:107FC00012B11378022B02D0002303604360704784
:107FD00070B50468ACB144689CB100290E4612DB50
:107FE000E3688B420FDD002904F1100409DD002550
:107FF000204600F08DF801350130AE4204EB00144C
:10800000F6D1204670BD0024204670BD38B50B4621
:108010000446114618461D68FFF7DAFF25606060C8
:1080200010B10378022B02D0002323606360204646
:1080300038BD00BF10B50446FFF7CAFF0146204611
:10804000BDE8104000F076B810B50446FFF7C0FF59
:1080500001462046BDE8104000F078B8C0E90012A3
:1080600012B11378012B02D00023036043607047E4
:10807000F8B5036833B3446806461CB30F4609B32A
:10808000E368012B04F110041CDD00250BE000F077
:108090003FF87368DB6803EBD3730230B5EB630F13
:1080A00004EB00140EDA2146304600F04FF801468A
:1080B00038460CF0A9FD0346013504F11000002BF1
:1080C000E5D1F8BD0020F8BD38B50B460D68044673
:1080D00011461846FFF7CCFF294602462046FFF717
:1080E0006DFF204638BD00BF10B50446FFF7C0FF46
:1080F00001462046BDE8104000F01CB810B504460B
:10810000FFF7B6FF01462046BDE8104000F01EB85C
:1081100081684269914200F110034FF0000007DDD1
:108120005A698A4203F1100300F10100F8DB70473D
:10813000704700BF09B10A780AB1002070474B6848
:1081400000681146184409F055BF00BF21B10B78F3
:10815000012B03D9032B01D00020704702688B68E4
:108160004FF0000C02F803C000684B6818447047D9
:10817000F0B5214E214C3178054683B0204601F000
:10818000CDFF002D32D02621204601F019FC00271A
:10819000627B216900973B460125184802F0C8FA26
:1081A0003278617B20690223CDE9005702F0E2FAC0
:1081B000206902F0F9FA0646206902F0F5FA2B462A
:1081C0000546627B216900970C482D0202F0B0FA47
:1081D00005F4FE45F0B2284308F072FA084908F0A9
:1081E000C3FA084908F0B6F903B0F0BD27212046CC
:1081F00001F0E6FBCBE700BF588EFF1F10A0FF1F6A
:108200000AD7A33C339388432DE9F041354D82B022
:108210000E4607461D212846144601F07FFF002127
:10822000284601F0CDFB4FF47A7300936A7B2969ED
:108230000023284602F07CFA4023013BFDD10121B6
:108240000023CDE900131D22697B2869072302F072
:1082500091FA286902F0A8FA286902F0A5FA804686
:10826000286902F0A1FAC3B243EA08231BB2C3EBA8
:10827000431203EB8203DB0044BF03F57F533F331C
:108280009B133B60286902F08FFA0746286902F0C9
:108290008BFAC0B240EA072000B2C0EB401300EBFB
:1082A0008300C00044BF00F57F503F30831328692E
:1082B000336002F079FA034628691D4602F074FA29
:1082C000C0B240EA052000B2C0EB401300EB8300CF
:1082D000C00044BF00F57F503F308013206002B0E3
:1082E000BDE8F08110A0FF1F38B504469225292073
:1082F000A36820712246012125709847E368207900
:108300002246012198472378142B01D01D2B02D13E
:108310000120E07038BD3920A36820712246012178
:1083200025709847E36820792246012198472378F1
:10833000142BEDD01D2BEBD000232371E07838BD3A
:108340004FF0000C8160C26080F803C080F804C068
:10835000704700BFC37870B50446002B2FD080252E
:108360002079A36825702246012198472079E36887
:108370002246012198472378A6682079257043F08A
:108380000103224663700221B047032004F052FF2C
:108390002079A36825702246012198472079E36857
:1083A00022460121984723782079A668257043F05A
:1083B0000203637022460221B047012070BDFFF71F
:1083C00093FFE0780028CAD170BD00BFC378DBB14D
:1083D00010B5044608460D4908F0C6F908F0B0FB90
:1083E00041F6170398429DBF094BA3FB0030C0F331
:1083F00007100020812222706070A3682079224635
:108400000221BDE810401847704700BF000020411E
:10841000ABAAAAAAC378002B3DD070B50446084683
:108420002F4908F0A1F908F065FB1728054645DD3E
:10843000B0F5C05F30DC8D22A3682280207922460F
:1084400002219847274AEB1782FB0525C3EBA503BA
:10845000C3F5807383212079A5682170224663705B
:108460000221A84780252079A36825702246012192
:108470009847E36820792246012198472378A66827
:1084800043F00803637025702079224633460221A9
:10849000BDE870401847704740F28D22A3682280E3
:1084A00020792246022198470F4BB5F5903FA8BF8F
:1084B0004FF49035A3FB0535AB09C9E7802520793A
:1084C000A3682570224601219847E3682079224657
:1084D000012198472378A66803F0F703D2E700BF8D
:1084E00000002041ABAAAA2A398EE338C37802469D
:1084F00033B18F20107051709368107902211847A2
:10850000704700BFC37803B9704770B50446802533
:10851000A368024601210079257098472079E36815
:108520002246012198472378A668257043F010035E
:1085300063702079224633460221BDE87040184717
:10854000C37802462BB1E6210170836800790121CE
:1085500018477047C378024653B1A6204FEA112C42
:10856000107051709368107982F802C00321184787
:10857000704700BFC378024653B1A4204FEA112CC4
:10858000107051709368107982F802C00321184767
:10859000704700BFC37802468BB13C2907D90F2131
:1085A0008C201070517093681079022118470329AC
:1085B000F6D9034BA3FB013189080331F0E770477B
:1085C000CDCCCCCC10B50446C07800B910BD4FF06E
:1085D000930C2079A36884F800C0224601219847B3
:1085E0002079E368224601219847207800F00100B5
:1085F00010BD00BF10B50446C07800B910BD4FF0E3
:10860000B40C2079A36884F800C022460121984761
:108610002079E368224602219847208810BD00BFD8
:1086200010B50446C07800B910BD4FF0B60C2079E3
:10863000A36884F800C02246012198472079E368A6
:10864000224602219847208810BD00BF10B504467D
:10865000C07800B910BD4FF0B80C2079A36884F839
:1086600000C02246012198472079E3682246022172
:108670009847208810BD00BF10B50446C07800B9E7
:1086800010BD4FF0BA0C2079A36884F800C02246D0
:10869000012198472079E3682246022198472088E3
:1086A00010BD00BFCB78C043C0F3C010B3EB001FB8
:1086B00027D010B502010C46CA7082B04878D4F8B1
:1086C00048C001230DF10702F321E04784F854006C
:1086D000C8B99DF80730E2786078D4F84CC002F051
:1086E000100223F0100313438DF807300DF1070239
:1086F00001237321E04784F8540020B9002002B020
:1087000010BD002070476FF00100F8E7F0B130B500
:10871000856C83B004469DB1C36C8BB1036D7BB196
:10872000407801230DF10702F321A84784F8540093
:1087300048B99DF8073003F01003E37003B030BD73
:108740004FF0FF30FAE76FF00100F7E74FF0FF302E
:10875000704700BF2DE9F8431C469B78D4F8489039
:1087600005460E4617467BB14FF0000860783B4641
:1087700032462946C847002884F854000CBF4046BA
:108780006FF00100BDE8F883B9F1000F0DD0E36C84
:108790005BB1236D4BB12146FFF784FF804608B9DA
:1087A00045F08005D4F84890E0E74FF0FF38DDE76A
:1087B0002DE9F04300258BB01E46044688469146BD
:1087C0002946242201A800950CF078F9002E4AD001
:1087D000B36C002B47D0F36C002B44D0336D002BCF
:1087E00041D009F1FF33122B43D81FFA89F908F160
:1087F000FF380DF1010728460CE0237807F8013C0B
:108800000135ABB218F8012F07F8022B4B4504F1E4
:10881000010413D2B378002BEFD1B26C23782AB3C2
:10882000F26C1AB3326D0AB318463146FFF73AFFBD
:10883000237803F07F0307F8013CE1E780B94FEAB2
:108840004903013BF46C9DF8001070789BB20DF168
:108850000102A047002886F8540018BF6FF00100FD
:108860000BB0BDE8F0834FF0FF30F9E74FF0FF3079
:10887000DFE76FF00300F3E730B583B0E022B62303
:108880008DF806208DF8073038B3836C044623B387
:10889000C36C13B3036D03B383788BB123460122FA
:1088A0000DF107010DF10600FFF782FF236D05466C
:1088B0000A2098470DB9A37853B1284603B030BDBC
:1088C000FFF724FF05460028E8D0284603B030BD56
:1088D0002046FFF71BFF0546EFE74FF0FF35ECE7BB
:1088E000002800F0178130B5836C8DB00446002B52
:1088F00000F0BE80C36C002B00F0BA80036D002B2B
:1089000000F0B680FFF7B8FF034610B118460DB06F
:1089100030BDA36C002B00F0AB80E36C002B00F0AB
:10892000A780236D002B00F0A3802346012221465F
:10893000D020FFF70FFF03460028E7D12378612BF3
:1089400040F0938000252522294602A801950CF0CD
:10895000B5F8A36C8DF80350002B00F08980E36C10
:10896000002B00F08580236D002B00F081802346D2
:10897000192201A98920FFF7EDFE0346002800F027
:10898000BA809DF826009DF825109DF805209DF8D9
:108990000750A57641EA00219DF80600E18242EAEF
:1089A00000229DF809109DF80A00228341EA002167
:1089B0009DF80B209DF80C00A18342EA00229DF84F
:1089C0000F109DF810009DF80D5084F8205041EADA
:1089D00000219DF814509DF81200E28361849DF8F7
:1089E00011209DF8171084F826509DF8185042EA7F
:1089F000002241EA0521A28421859DF819209DF8D5
:108A00001A109DF8130084F8270042EA01226285BB
:108A10009DF81B1084F82C109DF828C09DF8271095
:108A20009DF81E209DF81D009DF81F5041EA0C2165
:108A3000618202F00F01120942EA001241EA0511B7
:108A400062819DF824200898218122749DF82910C4
:108A50009DF82A20E0606174227563B19DF80320BF
:108A600042F3031284F8362050E76FF002034DE71B
:108A70004FF0FF334AE7A36C002B4FD0E36C002B81
:108A80004CD0236D002B49D0234601220DF1030168
:108A90000220FFF75FFE9DF80320C2F30111034699
:108AA00084F834100028DBD1A36C002B42D0E36C97
:108AB000002B3FD0236D002B3CD0234601220DF12B
:108AC0000301FFF747FE9DF8032084F83520034695
:108AD0000028C5D1A36C93B3E36C83B3236D73B348
:108AE000234601220DF103010420FFF733FE9DF818
:108AF00003200346B4E7A36CCBB1E36CBBB1236D99
:108B0000ABB1234610220DF11D01E120FFF722FE3B
:108B1000034636E74FF0FF33184670479DF80320B1
:108B2000C2F301114FF0FF3384F8341098E74FF08F
:108B3000FF3326E784F835204FF0FF3390E74FF0FE
:108B4000FF338DE730B583B074238DF807300028EC
:108B500048D0836C0446002B44D0C26C002A41D01C
:108B6000026D002A3ED00025CBB3E36CBBB3236D6E
:108B7000ABB3234601220DF106017420FFF7EAFD95
:108B800010B1CDB1A36CEFE79DF8063013F00305EB
:108B90000FD023F0030C012223460DF106010DF145
:108BA00007008DF806C0FFF703FE236D0A209847E3
:108BB000E8E794F844200AB903B030BD23F003037A
:108BC00002F0030243EA020C0DF1060123460122E2
:108BD0000DF107008DF806C0FFF7EAFDECE74FF056
:108BE000FF30CEE74FF0FF30E6E700BFF0B58A6C0C
:108BF00091F8446089B000238DF807300493ADF8F4
:108C000014300693ADF81C30002A00F0D681CA6CEF
:108C10000C46002A00F0D1810A6D002A00F0CD81B7
:108C200010F00802054640F0428181F844202046B9
:108C3000FFF788FF15F0100731D094F83B30072B71
:108C400008D994F84630072243F0020384F83B2009
:108C500084F84630A36C002B00F0B481E36C002B49
:108C600000F0B081236D002B00F0AC81234601227F
:108C70000DF107017520FFF76DFD94F83B309DF86D
:108C800007209B0003F01C0322F01C0213438DF805
:108C900007308DF81830752301278DF81030AA069B
:108CA00034D594F83D30082B08D9082384F83D309A
:108CB00094F8463043F0020384F84630A36C002B4E
:108CC00000F08C81E36C002B00F08881236D002B79
:108CD00000F08481234601220DF107017020FFF787
:108CE00039FD9DF8073094F83D2023F0080302F089
:108CF0000802134307F120026A448DF8073002F896
:108D0000083C01377023FFB202F8103CAB0742D099
:108D100094F83930052B08D9052384F8393094F8B4
:108D2000463043F0020384F84630A36C002B00F079
:108D30005281E36C002B00F04E81236D002B00F07C
:108D40004A81234601220DF107017420FFF702FD3D
:108D5000E9079DF8073008D594F8392003F01F0380
:108D600043EA4213DBB28DF80730AA0709D594F81D
:108D70003A20920023F01C0302F01C0213438DF8EA
:108D8000073007F120026A44013702F8083C7423D7
:108D9000FFB202F8103C6B0734D594F83830052B3D
:108DA00008D9052384F8383094F8463043F002039C
:108DB00084F84630A36C002B00F00A81E36C002B92
:108DC00000F00681236D002B00F002812346012272
:108DD0000DF107017220FFF7BDFC9DF8073094F8F4
:108DE000382023F0070302F00702134307F12002A3
:108DF0006A448DF8073002F8083C01377223FFB24D
:108E000002F8103C15F0C00F45D094F83E30012B0D
:108E100008D9012384F83E3094F8463043F0020329
:108E200084F8463094F83C300A2B08D90A2384F899
:108E30003C3094F8463043F0020384F84630A36C8B
:108E4000002B00F0C280E36C002B00F0BE80236D8D
:108E5000002B00F0BA80234601220DF1070171209A
:108E6000FFF778FC69062AD49DF807302A0608D552
:108E700094F83C2023F00F0302F00F0213438DF807
:108E8000073007F120026A44013702F8083C7123D9
:108E9000FFB202F8103C18B184F8446009B0F0BD8C
:108EA00023463A4606A904A8FFF782FCF4E7012E00
:108EB000ADF80C3010D081F844300120BAE694F8B7
:108EC0003E309DF807201B0103F0100322F0100232
:108ED00013438DF80730C9E7B1F84020B1F91210FB
:108EE000B2F5C87F28BF4FF4C872C82A01F5163101
:108EF00038BFC82201F2991101FB02F23949A1FBE6
:108F00000202120902F54812A1FB0212D00894F9DC
:108F1000141094F9042012FB01F2334981FB027111
:108F200094F91170D217C2EBA11207F5447707FB31
:108F300000F0120294F9351002EB600294F834004C
:108F40000430B2FBF0F201EB811001EB400101F5BE
:108F50008031B2FBF1F2FA3A02EB021223495200DD
:108F6000323281FB0201D217C2EB61128DF80C2064
:108F700046F25A42ADF80820B4F84220B2F57C6FB0
:108F80001ED23F2A06D9920801333F2ADBB2FAD813
:108F90009B01DBB21344DBB200278DF80D3084F85F
:108FA0003C702346022203A902A8FFF701FC84F8C3
:108FB000447000287FF43EAE39E64FF0FF306DE795
:108FC000FF23E9E74FF0FF3057E64FF0FF3049E766
:108FD0004FF0FF3001E74FF0FF30B9E64FF0FF30C0
:108FE0007FE600BFCDCCCCCCD34D62101F85EB51BA
:108FF00010B40A46194992F839C092F83A3004463A
:1090000003C983B0083300900CF108000DEB000C8D
:109010006B44ADF804101CF8081C13F8083C0B4412
:1090200092F8381008316944204611F8081C0C4C9D
:10903000194440F2AB7C41F2B9230CFB0133A4FB91
:1090400003439B090133038092F83E1019B1B2F833
:1090500042201344038003B010BC704760D5010068
:10906000D34D62102DE9F04F87B0002900F09A81AE
:109070008B6C0C46002B00F09581CB6C002B00F024
:1090800091810B6D002B00F08D810026CDE90266E9
:1090900007460496ADF814608DF816600A2546B1AF
:1090A000013D15F0FF05FAD10226304607B0BDE8B4
:1090B000F08FA36C002B00F07881E36C002B00F0A4
:1090C0007481236D002B00F0708123460F2202A9CA
:1090D0001D20FFF73FFB06469DF808209DF816105F
:1090E0009DF80D909DF80EA09DF80F009DF810B012
:1090F0009DF811C09DF815E002F0800302F00F0208
:109100007A7001F0300243EA02089DF80920BA7033
:109110009DF80A2000929DF80B20019287F80080AC
:109120009DF80C201BB9236D0A209847B8E7E58A03
:109130000B460009019940EA0A10120940EA093079
:1091400042EA01126D00009994F91AA0C5EBD0050E
:10915000E81742EA0132690841EAC07101FB00F0F8
:10916000A1FB011909EB4009B4F9180080FB0505C2
:10917000090BC00A41EA095140EA45504FEAEA7535
:109180004FEA29394FEA0A1A01FB05F50AFB09558E
:10919000A1FB0A1A5544890B41EA8541014401EBC0
:1091A00081008030001221634910B880A1F57A4A0D
:1091B000B4F9249094F920104CEA0B2C4FEAAA053C
:1091C000B4F91EB005FB05F50AFB09F949010AFBD4
:1091D0000BFA4FEA653B0BFB01F1C91001EB6A0189
:1091E00094F926A0ED120AFB05F54FEA490909EBAF
:1091F000A509B4F922502D0405EBA905C2F580128A
:10920000A2EB25328914A58BB4F92A9001F500410F
:1092100001FB05F540F63541ED1302FB01F1B1FB11
:10922000F5F141F39C0202FB02F2B4F9285052130B
:1092300009FB02FA41F35D0205FB02F241F3D71983
:10924000521309FB09F502EB2A3294F82CA009FB12
:1092500005F50AFB05F502EB654294F9275002EB90
:10926000C512121102EB4102BA6094F90E10504D72
:1092700000FB01F1CA1785FB0191C2EB611294F961
:109280000D1000FB02F200FB01F14FEAA21985FB71
:1092900009A9D21785FB01BAC917C1EB6A11C2EB44
:1092A00069120A44618994F90C9002F5804201FB2D
:1092B00002F22189ACEB011C94F9101000FB09F9B2
:1092C00000FB01F185FB09A04FEAE979C9EB6019C0
:1092D000ACEB6900921200FB02F285FB0150C9174A
:1092E000C1EB6011E07B01EBC011901300FB00F0BB
:1092F0000911801201FB00F002EB60024FF47A7159
:10930000921201FB02F212132A4922EAE2728A4205
:10931000A8BF0A46FA6003F00F059A09264B53F8D6
:1093200025C094F9363042EA8E0240F23C514FF0AB
:10933000050E0020CEFB0310204B53F82550A1FB57
:109340000C130CFB0033D203090C41EA034112F168
:109350007F4260EB000052184FEA234C40EB23435E
:10936000A5FB010105FB0C11400A550845EAC37530
:1093700040EAC15040194FEA630545EB612107F00F
:10938000FFFB3861002E7FF490AE18F0800F18BFFD
:109390000123304614BF84F8453084F8456007B097
:1093A000BDE8F08F4FF0FF367FE64FF0FF3693E6D3
:1093B0001F85EB51A08601005C8EFF1F9C8EFF1F56
:1093C000164AC0F3036CC0F3035100B503464FEADD
:1093D000107E134812F80CC0515C80F801C08170F7
:1093E000C3F3034CC3F3033112F80CC0515C80F893
:1093F00003C00171C3F3032CC3F3031103F00F0384
:1094000012F80EE012F80CC0515CD35C80F800E05A
:1094100080F805C08171C3715DF804FB68D5010057
:1094200004A0FF1F024B4FF0FF321A60704700BFCD
:10943000DC8EFF1F014B1868C0437047DC8EFF1F96
:10944000002916DD10B50B4C00F1FF3C22680A48DC
:109450000CEB010E1CF8013F08215A4042F30003B7
:109460000340013983EA5202F8D1E645F2D1226085
:1094700010BD7047DC8EFF1F2083B8ED0378A3B1C9
:1094800010B40A4C8446226809485A40082142F325
:1094900000030340013983EA5202F8D11CF8013F6E
:1094A000002BF2D1226010BC70477047DC8EFF1F8A
:1094B0002083B8ED2DE9F04F04689C460B5D002B2E
:1094C0006DD0914D914E00275B2B00F0218100F271
:1094D000ED80093B5FFA83FEBEF1310F1CD8312BC2
:1094E0001AD8DFE803F0565619195619191919191F
:1094F0001919191919191919191919191956197444
:10950000191919191919191919561919191919198E
:109510001919191919191956D0F800E011F80E3057
:1095200001EB0E08002B00F085803A2B03F0DF09D9
:10953000A3F1200A00F29C801F2B00F2B0800A2BBE
:1095400076D8082B76D804606FF00100BDE8F08F64
:109550008B46714696464A46D94698F800B0D345A0
:1095600040F0C8800134C0F80890C8F8084002EB09
:109570000318744601E0D8F80440013404D0D8F848
:109580000840013400F01681013B5C1CA8F1100872
:10959000F1D10468013404600B5D002B94D1416863
:1095A0004B1E58BF02EB01120ED452F80C1C0131B5
:1095B00003F1FF3304D052F8081C013100F0078199
:1095C000591CA2F11002F0D10020BDE8F08F04F187
:1095D0000108C0F8008011F808E04346BEF1000F12
:1095E00021D09146724604E0036801330360CA5CEF
:1095F000CAB1222A00F0BA805C2AF5D10133036097
:10960000CA5CA2F15C0E5FFA8EFE752A26FA0EFE87
:1096100099D85B2A71D91EF0010F94D001330360F1
:10962000CA5C002AE5D104606FF00200BDE8F08F4B
:109630000D2B88D143689C452DD902EB03184FEAC6
:109640000319013343608368C8F80C7002F809708D
:10965000C8F804405C1CC8F808E000F0AF8002EBDA
:1096600003187446D8F80C300133C8F80C3092E770
:10967000B9F15D0FDED0BAF15E0F3FF664AF0EF1C7
:10968000010EC0F800E018F8013F002B7FF44DAF49
:1096900043689C45D1D804604FF0FF3056E7203B2B
:1096A000DBB225FA03F3DB07E9D5C3E77B2B2FD029
:1096B00003F0DF0EBEF15D0F7FF42EAF7D2B43680C
:1096C0000CBF4FF0010A4FF0020A013B7BD402EBC2
:1096D00003188E469146D8F80420511C05D0D8F8BE
:1096E0000810B1F1FF3F3FF433AF013B5A1CA8F122
:1096F0001008F0D16FF0010028E7222A3FF475AF7F
:109700002F2A3FF472AF1EE7011000044104440306
:10971000D0F804E0F44553D9D0F8088002EB0E19D4
:109720000EF1010AC0F804A0B8F1FF3F4FF0FF3A74
:10973000C9F808A0C9F80C704FEA0E1A07D002EB5E
:109740000818D8F80CB00BF1010BC8F80CB07B2B43
:1097500003680CBF4FF001084FF0020802F80A80BE
:10976000C9F80440C0F808E05C1C14E7D0F804E035
:10977000F4454A468FD909EB0E190EF101044FEA60
:109780000E1A44604FF00304C9F80C7002F80A4046
:10979000C9F808308368C9F804805C1C3FF4F9AE4E
:1097A00002EB031E0468DEF80C3001330134CEF8FE
:1097B0000C30F0E6046883600134ECE67446EAE6B7
:1097C0004FF0FF30C2E601337FF4E3AE92E76FF073
:1097D0000200BBE600234FF0FF320360436082606B
:1097E000704700BF2DE9F0433B4E83B08846814669
:1097F0000E213046174600F091FC0121304600F062
:10980000DFF84FF47A730093727B3169012330469D
:1098100000F08EFF4023013BFDD100250123009382
:109820000E220623717B3069019500F0A3FF306999
:109830003D60C8F80050C9F80050D0F83821D0F881
:1098400034319A4204D000F0AFFF030230691DB2F8
:10985000D0F83821D0F834319A4235D12B46002443
:10986000C9F80030D0F83821D0F834319A4204D009
:1098700000F09AFF030230691DB2D0F83821D0F809
:1098800034319A4203D000F08FFFC4B2306945EA08
:109890000403C8F80030D0F83821D0F834319A42A7
:1098A00004D000F081FF030230691DB2D0F83821E6
:1098B000D0F834319A4202D000F076FFC4B22C4383
:1098C0003C6003B0BDE8F08300F06EFFC4B245EA2F
:1098D00004033069C4E700BF10A0FF1FF0B583B0D8
:1098E0000D4E0023019301230D46174600930246B7
:1098F0000B463069717B00F03DFF55B1013D7C1E88
:1099000057FA85F5306900F04FFF04F8010FAC42BB
:10991000F8D103B0F0BD00BF10A0FF1FF0B50346A3
:109920000D4683B00D481946174600F0F7FB5DB1B0
:10993000013D0A4E7C1E57FA85F514F8011F30468A
:1099400000F03EF8AC42F8D104480023427B0169A4
:109950000093012300F0ECFE03B0F0BD10A0FF1F48
:10996000002070470369D3F83801D3F83431C01AA6
:10997000704700BF0369D3F83411D3F838219142FE
:1099800008D2D3F83421511C1A44C3F8341192F888
:10999000300070474FF0FF30704700BF0369D3F8C5
:1099A0003411D3F8382191423DBFD3F834219B18AC
:1099B00093F830004FF0FF30704700BF704700BF92
:1099C0000369D3F84422B2F5817F03D901234360B0
:1099D00000207047D3F84422012003EB020C02441C
:1099E000C3F844228CF83C11704700BF38B50369B6
:1099F0000A4A026093F84822022A044601D020460F
:109A000038BDD3F87452002DF9D0284602F0F0F991
:109A10002846082103F084F8204638BDA0D601006E
:109A2000036970B50446D3F84402B0F5817F04D9C8
:109A3000012300256360284670BDD3F84452D3F853
:109A40004462C5F581750135954228BF154603F579
:109A50009E703CBF012363602A46304402F016FF2B
:109A60002269D2F844322B44C2F84432284670BDF1
:109A700070B5154CD4F8A8321B7813F0200512D01D
:109A800094F8F8340133DBB2012B84F8F83403D8AE
:109A900094F8E534012B05D094F8E704BDE8704054
:109AA00003F006B970BD84F8F15494F8E70403F0AC
:109AB000FFF8D4F80435002BF4D0C4F8D053D4F810
:109AC000D403BDE870401847E08EFF1F70B5154CF9
:109AD000E3681B7813F0200512D094F85C32013350
:109AE000DBB2012B84F85C3203D894F84932012BA5
:109AF00005D094F84B02BDE8704003F0D9B870BDB2
:109B000084F8555294F84B0203F0D2F8D4F8683236
:109B1000002BF4D0C4F83451D4F83801BDE87040BB
:109B2000184700BFE08EFF1FF8B5C3681B789B067F
:109B300023D483680D4680211970C36812211970DF
:109B400090F84932012B044608D01AB980F848220F
:109B50000120F8BD531E012B11D813468DB1012DE4
:109B600005D14FF0E0224FF00071C2F80011022B36
:109B70000ED0012084F84802F8BD0020F8BD012075
:109B8000F8BD4FF0E0224FF08071C2F80011EEE70F
:109B9000D4F87462002E56D03379102B5DD075B393
:109BA000012D07D00022022384F85E2284F8483277
:109BB0000120F8BD31688B8B9BB243F008038B8387
:109BC00033792D4E5A1102F138224032920003F1BE
:109BD000100703F01F0005FA00F0284D46F8275043
:109BE00010608A8B03F1804392B203F5043342F094
:109BF00002028A830020972218701A70D2E7316817
:109C00008B8B9BB243F008038B8333791A4E5A1126
:109C100002F13822403203F01F07920003F1100CCA
:109C20000120B840164F46F82C7010608A8B03F163
:109C3000804392B203F5043342F002028A839622F3
:109C40001D701A70AEE7082002F068FF002106467A
:109C500002F070F8C4F874629EE7304602F0C8F86B
:109C60003046082102F05CFF01200023C4F8743262
:109C700084F84802F8BD00BF0084FF1F3DAE00001D
:109C800031AE00002B4B70B5A3FB014E2A4DA3FB58
:109C900002324FEA9E1E92094FEA0E2EAC46BEFBE0
:109CA000F2FE1423002204E00132372A38D05CF897
:109CB000043FBEEB032F4FEA0324F5DAAAB91423BD
:109CC0004468B1FBF3F322701C4AC0F85032914251
:109CD00003D3836904221A7070BD194B8269A3FBF8
:109CE0000131C1F30751117070BD02F1FF3CAEEBC1
:109CF000040455F82C502E02AEEB060EBEF1000FF8
:109D0000B8BFCEF1000E002CB8BF6442A64504DCFB
:109D10000C4A2B4612F80C20D2E70A4CA25CCFE783
:109D2000744600234FF470264FF470654FF0360CE4
:109D3000E2E700BFD34D621084D50100006CDC0265
:109D4000819F5E1660D601002DE9F0471D469DF803
:109D500024309DF820909DF8288004460E46174632
:109D600013B1B8F1000F1DD116B3012E15D11D2F5F
:109D700000F0BA801A2F00F0AE8094F84A324FF00B
:109D8000000A1E2D94F84B3232D01F2D00F09C801B
:109D90009D4228D00020BDE8F08794F84A3294F81C
:109DA0004B32F7E7C26812789206F3D4002EDCD16A
:109DB000102F49D0132F50D094F84A32B246A5F153
:109DC0001103012B94F84B32E2D89D4212D1B8F125
:109DD000000F00F093800223BAF1000FDAD0181EB2
:109DE00018BF0120D7E7B8F1000FD3D00023F3E765
:109DF0001E2BECD00226B8F1000F09D094F84C12BB
:109E000094F84B02003918BF0121490003F0B6F95C
:109E10003302B9F1000F14D143F064033B4A02EB63
:109E2000C502BAF10000526813604FF0010384F8D4
:109E30004B5284F8993218BF012084F84C92BDE847
:109E4000F08743F00303E9E794F84A22102A08D187
:109E5000002B57D04FF0020AB1E794F84A22132A98
:109E6000F6D04FF0020A4BB194F84C1294F84A0223
:109E7000003918BF0121490003F080F94FEA0A2296
:109E8000B9F1000F1DD142F06402204B03EBC70370
:109E90005B681A60012384F84A7284F84C9284F853
:109EA0009832002E8BD0012E3FF46BAF94F84B32DA
:109EB0009D427FF46FAFB8F1000F3FF46BAF00230A
:109EC0008DE742F00302E0E71F2B15D1B8F1000F38
:109ED00016D0062380E794F84A221A2A4FF0060A81
:109EE000C1D1002BCAD04CE794F84A221D2AB8D120
:109EF00043B14FF0020A44E706267CE7022687E7D3
:109F0000062685E74FF0020AB8E700BFBCD801007B
:109F10002DE9F04184B0044696469C469DF8287091
:109F20009DF82C209DF830309DF834009DF83C6061
:109F30000D4600295ED1DFF8EC80D8F8341041F0EE
:109F40004001C8F83410002184F849E284F8551221
:109F5000BEF1000F27D1616920270F7012B994F864
:109F60004A22D2B213B994F84B32DBB2009094F883
:109F70009912029194F89812019120462946FFF710
:109F8000E3FE0E9A28492046FFF77CFE324629461A
:109F9000FFF7CAFD94F84932ABB9A36880221A7062
:109FA00004B0BDE8F081A7B961694FF0200E81F8D7
:109FB00000E021684FEA4C0C5FFA8CFC81F800C08D
:109FC000E1690F70CAE7A368C0221A7004B0BDE847
:109FD000F08161694FF0280E674581F800E014D9DF
:109FE00021684FEA4C0C5FFA8CFC7F00FFB281F8CD
:109FF00000C0E5E70129A6D1DFF82880D8F83410A1
:10A0000041F08001C8F834109DE74FEA470E2168FF
:10A010005FFA8EFE4FEA4C0C5FFA8CF781F800E095
:10A02000CEE700BF00800440006CDC022DE9F04167
:10A03000144682B005460F46984603F0DBF80CB98B
:10A04000D5F8784203F0D6F8AB681A78920606463F
:10A0500009D5B4221A702F4B1B78002B35D0012064
:10A0600002B0BDE8F0812CBBEA6892F800C01CF099
:10A07000200CF8D1AB6885F849C2B0221A70AB68E1
:10A08000187810F02000E6D1062385F85532D5F86F
:10A090009032013304D0D5F890320133C5F89032B4
:10A0A000D5F87032002BDBD001909847019802B0B0
:10A0B000BDE8F08103F09EF8801B8442D4D8AB68E1
:10A0C000187810F02000C6D1DEE795F84832013B41
:10A0D000012BC4D802F000FD0F4B012F14BF1B7ED3
:10A0E0005B7E8342BBDB0F2809DD67B1012F0AD1FC
:10A0F000A0F11003084ADBB253763846B0E70120DE
:10A1000088F80000ACE7044AA0F11003DBB2137634
:10A11000A5E700BF38A0FF1F00E400E00369490085
:10A1200083F83C11036900220121C3F84412426004
:10A1300083F85522704700BF2DE9F043054683B0F0
:10A140001C46D5F8443200208DF80700002B74D04F
:10A1500017460CB9D5F87842EB6812221A702846D7
:10A160000DF107032246FFF761FF002865D095F83F
:10A1700048321BB19DF80720002A4BD003F03AF873
:10A18000082385F85532D5F8446285F85472804624
:10A190001EB305F23B1700264FF00209002C5FD1D9
:10A1A0002B6917F8012F1A70EB6801E0002C47D1DA
:10A1B00019788A07FAD583F80090002C49D1EA680B
:10A1C0001378D806D9B252D4CB0762D4D5F844322A
:10A1D0000136B342E2D895F85472AB68012F0CBF38
:10A1E0008022B0221A70D5F84432B34262D90123DA
:10A1F00085F85532D5F88032013304D0D5F8803255
:10A200000133C5F88032D5F87032B3B103B0BDE880
:10A21000F0431847591E01290FD80821022B85F851
:10A22000551285F85472C5F8402258D0AB68F02218
:10A230001A702B6995F83C211A7003B0BDE8F083C1
:10A2400002F0D8FFA0EB08008442ADD8EB6883F899
:10A25000009002F0CFFFA0EB08008442AFD8BAE72D
:10A2600002F0C8FFA0EB0800844299D8B3E710239E
:10A27000042185F855121370AB6880221A70D5F846
:10A280008C320133BFD0D5F88C320133C5F88C3213
:10A29000B9E7BEB1032385F85532D5F888320133CA
:10A2A00004D0D5F888320133C5F88832AB688022F3
:10A2B0001A70A8E7D5F86032002285F85522002BE5
:10A2C000A4D1BAE7022385F85532D5F88432013398
:10A2D000ECD0D5F884320133C5F88432E6E7D5F8FE
:10A2E0004432042BA2D9D5F87432012085F85E02DD
:10A2F000D5F844121B6805F59F7498809860C1F1E9
:10A30000030003391C6089B2D983DA71D982D8601D
:10A31000D5F8743229691B68B1F1804F19619A82AE
:10A320009A7101D39A680AB901229A6000229A614F
:10A330007CE700BF2DE9F04383B0044600209DF880
:10A3400028700B9D8DF8070003B3B3F5827F20D2F0
:10A35000C4F834019046C4F85832C4F838010DB935
:10A36000D4F87852E36812221A7020460DF10703E0
:10A370002A46FFF75BFE48B194F848327BB19DF85E
:10A38000072062B9591E012940F23E8103B0BDE8A1
:10A39000F083052384F8553203B0BDE8F08302F062
:10A3A00029FF4FEA4803226984F8547243F00103FD
:10A3B000DBB2092184F8551206461370E26802E008
:10A3C000002D40F0968013789F07F9D50223137073
:10A3D000002D40F09780E2681378D806D9B200F1DA
:10A3E0000181CA0700F12281D4F858320A22012BD8
:10A3F000A36884F855220CBFA822A0221A702369F2
:10A400001B7800274FF0B008D4F83831D4F8582220
:10A410009A42BBD94FF0200994F855320A2BB5D196
:10A42000E26801E0002D3AD113789B07FAD50223A8
:10A430001370002D3BD1D4F83831D4F858120233C0
:10A440008B4241D0D4F838310133994246D8A368C1
:10A4500084F85D7283F8008023691978D4F8383164
:10A46000E2180133C4F8383182F8301094F85432CD
:10A47000012B05D14B46013BFDD1A36880221A7008
:10A48000D4F8643284F85572002B00F0A880984705
:10A49000D4F85812D4F838318B42BDD376E702F0A5
:10A4A000A9FE801B8542BBD8E36802221A7002F025
:10A4B000A1FED4F83831801B854203F102033FD955
:10A4C000D4F858128B42BDD1A368A8221A70D4F8D0
:10A4D0003831D4F8581201339942B8D9D4F8383108
:10A4E0002269581CC4F838012344127883F83020BC
:10A4F000D0E702F07FFE831B9D423FF65FAFE3682B
:10A5000002221A7002F076FE831B9D423FF663AF73
:10A51000A26801238021117084F85532D4F880326A
:10A52000013304D0D4F880320133C4F88032D4F837
:10A530007032002B3FF42AAF03B0BDE8F043184758
:10A54000D4F85822934200F0828094F85D32BBB96F
:10A55000A368A8221A70D4F83831D4F858220133ED
:10A560009A420FD994F85D3263B9D4F83831226930
:10A57000591CC4F838112344127883F830202AE09B
:10A58000D4F83831A36884F85D7283F800802369B9
:10A590001978D4F83831E2180133C4F8383182F828
:10A5A000301094F85432012B05D12023013BFDD10A
:10A5B000A36880221A70012384F85532D4F88032BF
:10A5C000013304D0D4F880320133C4F88032D4F897
:10A5D000703203B19847012384F85D3214E7D4F850
:10A5E000581257E71023042184F855121370A368FA
:10A5F00080221A70D4F88C32013398D0D4F88C327F
:10A600000133C4F88C3292E70921022B84F854728A
:10A6100084F8551226D0A368F0221A704FEA480336
:10A62000226943F00103DBB21370AFE6A368022195
:10A63000802284F855121A70D4F8843201333FF422
:10A6400076AFD4F884320133C4F884326FE7A3685C
:10A65000A8221A70D4F83831D4F858220133934222
:10A6600080D38FE7D4F85832042BD4D9012184F851
:10A670005E12D4F8741220690968B0F1804F086046
:10A680008A80CA7101D38A680AB901228A60D4F823
:10A69000742200201268C86004F130011161C3F116
:10A6A0000101013B9BB2D383D3820123907191615D
:10A6B00093829360AFE700BF70B51546044602F081
:10A6C00099FD0DB9D4F8785202F094FD064600E0E9
:10A6D000A5B994F85532072BFAD8A5B994F8553294
:10A6E000072B84BF012384F855328023013BFDD121
:10A6F00094F85502B0FA80F0400970BD02F07AFD7E
:10A70000801B8542E5D802F075FD801B8542E5D8A7
:10A7100094F84832022BE1D194F85E32002BDDD060
:10A7200094F85532072BFBD8012384F85532D5E72E
:10A73000F8B5069F0C46154606461A4629463B467E
:10A740002046FFF7F9FC3A4629462046FFF7B4FFBA
:10A75000336993F85532013BDBB2052B02D8044A2A
:10A76000D05CF8BD7068003818BF0120F8BD00BF8C
:10A770007CD5010070B582B09DF8186013B9002037
:10A7800002B070BD0096079E019604460D46FFF785
:10A79000D1FD079A29462046FFF78EFF0028EED00C
:10A7A000D4F8380102B070BDD0F83421D0F8383177
:10A7B0009A4208D2D0F834315A1C0344C0F83421EC
:10A7C00093F8300070474FF0FF307047F0B5AD4F51
:10A7D000D0F80CC03B780133DBB2044680683B7094
:10A7E0009CF80050037813F0200683B0EDB2DAB283
:10A7F0005ED0D60694F85E3221D5022B00F0E680BA
:10A8000094F85E32032B00F0E18094F85532082B67
:10A8100000F0218294F85532092B00F0478294F819
:10A820005532012B00F0028280230370E36802227C
:10A830001A703B78013BDBB23B7003B0F0BD022BDA
:10A8400000F08F8094F85E32032B00F08A80D4F8F9
:10A850003831D4F858220233934200F0718194F8D1
:10A860005532012B00F06781D4F83831013393421F
:10A8700080F0118194F85532012B00F00781D4F853
:10A8800038312269591CC4F838112344127883F8EE
:10A890003020E36802221A7094F85532012BDAB2A4
:10A8A000C7D194F85D32002BC3D184F85D22C0E794
:10A8B000EB062CD510238CF800306B06B6D594F837
:10A8C00055320C2B00F0448115F0040500F00F8187
:10A8D0000B2284F85522A3680022C4F84422D02217
:10A8E0001A70226913785B0884F85632D4F86C32F7
:10A8F0000BB198472269D4F84432002B40F02581EF
:10A9000084F83C3101231670C4F840328EE715F00C
:10A910004003D4D112F0100219D015F0010540F017
:10A920000181D4F84022D4F844329A4207D2D4F8B4
:10A9300040325A1C2344C4F8402293F83C51236906
:10A940001D70A368D0221A70D4F80CC004E094F8EB
:10A9500055320C2B00F00A8102238CF8003003B032
:10A96000F0BDD4F874321A68928B120600F11E8181
:10A9700094F85E22032A00F02B81434A1979D06AA9
:10A9800001238B4003423FF454AF9177D4F87432E3
:10A990001B79D377A36880220020072184F85E0208
:10A9A00084F855121A70E36802221A70D4F89432AF
:10A9B000013304D0D4F894320133C4F89432D4F87B
:10A9C0007032002B3FF435AF984732E7D4F8742249
:10A9D00013689B8B180600F15D8194F85E32032B9F
:10A9E00036D029491279C86A0123934003423FF4C3
:10A9F00020AF8A77D4F874321B79CB7700220723F3
:10AA000084F85E2284F85532D4F89432013304D0AD
:10AA1000D4F894320133C4F89432EB0611D50423F0
:10AA200084F85532D4F88C32013304D0D4F88C3207
:10AA30000133C4F88C32E268102100231170C4F88D
:10AA40004032A36880221A70E36802221A70B6E7C7
:10AA50009CF800301906FBD50B4912790A770023C0
:10AA600084F85E32D4F844322169013BC4F84032A4
:10AA7000D4F840322344022293F83C310B70E3684F
:10AA80001A70D6E638A0FF1F0080004094F85D32AF
:10AA9000002B3FF4F4AEA3680021B02284F85D12CD
:10AAA0001A70D4F838312269591CC4F8381123447B
:10AAB000127883F8302094F85432012B05D12023EA
:10AAC000013BFDD1A36880221A70E36802221A704C
:10AAD00094F85532012B00F0FC80D4F86432002247
:10AAE00084F85522002B3FF4D7AE9847D4E6BC4BF0
:10AAF000BC4A94F84B0284F85C5200290CBF114602
:10AB00001946032202F060F8A3680C2284F855224B
:10AB1000C022C4F838511A7023691B785B0884F886
:10AB2000563283E6C02202702269D4F80CC0127833
:10AB300084F8553210E794F85D32002B7FF494AE20
:10AB4000E8230370D4F858228EE694F83C61D9E6E5
:10AB5000D4F86832002B3FF4B7AE0022C4F8342199
:10AB6000D4F83801019198470199ADE69C4B9D4D71
:10AB700084F85C2200290CBF29461946032294F868
:10AB80004B0202F021F823691B78D4F83821B2F582
:10AB9000817FDBB207D8D4F83821A1180132C4F87C
:10ABA000382181F83030D4F80CC0D5E694F85E2214
:10ABB000022AD1B27FF4DCAE8B4A1B79D377A3682B
:10ABC000E8221A70E368032284F85E22197030E6E6
:10ABD000854A1B791377A3680021B02284F85E129E
:10ABE0001A70D4F858322269013BC4F83831D4F8CD
:10ABF0003831591CC4F838112344127883F83020B6
:10AC000094F85432012B05D12023013BFDD1A368D8
:10AC100080221A70E36802221A70D4F8643200228B
:10AC200084F85522002B7FF4CFAE02E694F854321C
:10AC3000012B0CBF8023B0230370E36802221A703B
:10AC4000D4F8803201333FF4BAAED4F88032013305
:10AC5000C4F88032B3E615F0100349D00023042273
:10AC600084F85E3284F8552210228CF80020A26805
:10AC700080211170E268C4F8403202211170D4F8CA
:10AC80008C3201333FF49BAED4F88C320133C4F8DC
:10AC90008C3294E694F85E32022BD9B27FF49DAEEA
:10ACA000514B1279DA77A368F0228AE7EE0637D59E
:10ACB0000422102384F855228CF80030A3688022E7
:10ACC0001A70E36802221A70D4F88C320133DBD197
:10ACD00075E6D4F88032013304D0D4F880320133E1
:10ACE000C4F88032D4F87032002B7FF4FEAED3E586
:10ACF00015F0010528D084F85E32D4F84032002BDC
:10AD000052D1022384F85532D4F88432013304D06E
:10AD1000D4F884320133C4F884328023037093E67C
:10AD2000E9072CD50223802284F855320270E268AC
:10AD30001370D4F8843201333FF441AED4F8843236
:10AD40000133C4F884323AE6D4F840320133C4F80F
:10AD50004032D4F84422934233D394F8543284F8E6
:10AD60005552012B0CBF8023B0230370E3680222ED
:10AD70001A70D4F86032002B7FF426AE59E594F8AF
:10AD80005E32012B32D0D4F85832012B4FF00A0238
:10AD90000CBFE823E02384F8552203702169E3689F
:10ADA000097802221A7044E5032384F85532D4F856
:10ADB00088320133B1D0D4F888320133C4F88832F4
:10ADC000ABE794F85E32012B1FD0D4F840322169F2
:10ADD0002344022293F83C310B70E3681A7028E593
:10ADE000719A0000CD9A0000008000400223E12209
:10ADF00084F85E320270D4F874120C4A0979D17664
:10AE00002169E2680978137013E50223F12284F8BE
:10AE10005E320270D4F87412044A0979D17622693C
:10AE200094F83D111170E268137002E50080004053
:10AE300001480021FFF7CABCE08EFF1F0148012135
:10AE4000FFF7C4BC7C91FF1F2DE9F8431148DFF8E0
:10AE50004890DFF84880124E124D066000244FF4EF
:10AE60007A774A46414644608760047344730561BB
:10AE700004F062FE0C48012305F527750473437343
:10AE80004A4641468760066005614460BDE8F84374
:10AE900004F052BE10A0FF1F408EFF1FED9900006E
:10AEA000A0D60100E08EFF1F24A0FF1F90F81CC059
:10AEB0004160BCF1020FC26001D18368184700F005
:10AEC000B1BF00BF436810B41C685A6821681143C1
:10AED00002682160154C16491460D160154C164962
:10AEE00014611160417A154A5C180A3194F824C043
:10AEF00053F8214002EBCC0149680C60017A5C18E0
:10AF000003EB810194F818C0CC6902EBCC014968CD
:10AF10000C60817A10BC581803EB810390F8300064
:10AF2000596B02EBC00253681960704701401F0063
:10AF3000011000380110007800001F80BCD801000B
:10AF400010B4426890F809C0104B944400219CF85A
:10AF500024C003EBCC0CDCF80440216090F808C05E
:10AF600094449CF818C003EBCC0CDCF8044021603E
:10AF7000847A00682244064C92F8302003EBC20326
:10AF80005B681960046010BC704700BFBCD801004A
:10AF900001401F0070B4016B4A4A0979D177C16A38
:10AFA00009791177016B09791177826A03462AB30F
:10AFB0004168C9688A4243D9C46A006B521A216841
:10AFC0009A620D6803F12404A5424FF0010259D0A2
:10AFD0001C68E56815F0804F0D6829D12D780E6842
:10AFE00045F0004501360E60656336490079C87644
:10AFF00012B1DB6A1B79CB7670BC70470168324CAA
:10B00000406B0A63CC62CC6824F08044CC60046856
:10B010002E4924684FF0030C8C4283F825C039D1A7
:10B02000037F4260022BC26038D170BC836818472E
:10B030002D880E6845F0004502360E606563D4E742
:10B04000C16A0968CC8B260402F1FF3031D4C0F309
:10B050000E00C883CC8B186BA4B2CC820468E58B3D
:10B060002D041ED4C2F30E05E583E58BADB2E58257
:10B070000D680024013A9C6203F1240418BF0122E8
:10B08000A542A5D11968CC6893F8244044F0004447
:10B090004C63AAE72346114670BC184770BC00F009
:10B0A000C1BEE58BC2F3080605F47E453543E58352
:10B0B000DBE7CC8BC0F3080004F47E442043C88354
:10B0C000C8E700BF0080004000000FFFADAE0000E9
:10B0D00008B50248FFF75EFF08BD00BF3CA0FF1F98
:10B0E0000A4A0B49002310B40A4C936093841460FD
:10B0F000516010BCD36093619362D3621363536356
:10B1000013615361D3611362704700BF3CA0FF1FFE
:10B11000BCD6010000C0024010B40A4B0A491B68AB
:10B120000A4A0B4C1268206083B003440B60094B41
:10B13000019202211970019A074B1A6003B010BCEA
:10B14000704700BF1894FF1F78A0FF1F00A1FF1FCA
:10B1500080A0FF1F7CA0FF1F74A0FF1F2DE9F04FF0
:10B160000268524912688A4283B0834640F08E805A
:10B1700090F924506A1C13D04D494E4A51F825408D
:10B18000EDB2157064B1AD0094F82520204603217E
:10B1900012B12268126890472C446468002CF3D1E5
:10B1A00000F07CF9DBF80020434952688A420446EB
:10B1B0006FD19BF92420531C64D03D4951F8225093
:10B1C000002D5FD0D2B205EB820091004668002EC0
:10B1D00050D070184768002F44D07818D0F80480F9
:10B1E000B8F1000F3BD008EB0100D0F80490B9F1A2
:10B1F000000F2BD009EB0100D0F804A0BAF1000F2A
:10B200001BD00AEB0100436873B1194401935846FF
:10B2100003234968FBF732FD019890F825301BB1F4
:10B22000036803215B6898479AF825302BB1DAF858
:10B23000003050465B680321984799F825302BB1C0
:10B24000D9F8003048465B680321984798F82530C4
:10B250002BB1D8F8003040465B680321984797F837
:10B260002530EBB996F8253023B1336803215B68AC
:10B270003046984795F8253023B12B6803215B6849
:10B2800028469847204603B0BDE8F08F0321904739
:10B2900086E7584603219047204603B0BDE8F08F6B
:10B2A0003B6838465B6803219847DBE7516800003C
:10B2B00084A0FF1FA4A0FF1FBD6D00003F4B9A7923
:10B2C00012F00C0F02D19A79D20636D43B4A937908
:10B2D000C3F38103032B35D0384A9379C3F3810339
:10B2E000022B37D0354A9379C3F38103022B3CD02C
:10B2F000324A9379C3F38103022B41D02F4B9879C3
:10B30000C0F38100012843D02C4A9379C3F3810311
:10B31000012B47D0294A937913F00C0FC3F3810016
:10B3200009D19379DB0607D4907980F02000C0F32F
:10B33000401080007047002070479B799806C5D464
:10B34000032070479379D906C6D493799B06C3D559
:10B35000082070479379D806C4D493799906C1D54B
:10B3600053789B07BED4072070479379D806BFD483
:10B3700093799906BCD453789A07B9D405207047BD
:10B380009379DB06BAD453789807B7D5062070476F
:10B390009A79D106B8D59A799206B5D45B789B078D
:10B3A000CAD4B1E79379D806B4D593799906B1D4C4
:10B3B00053789A07AED40220704700BF0040064081
:10B3C000024A034B102111809B78704700200540F2
:10B3D00000D00740C268D107034638D4110722D4F1
:10B3E000D10638D4910634D4510636D4110638D457
:10B3F000D10534D4910536D4510536D4110536D44F
:10B40000D10436D4910436D4510436D4110436D440
:10B41000D10336D4910304D4D10234D412F4402F92
:10B4200033D0222000E021201B4900220A704A70FC
:10B430008A70CA701A705A709A70DA7093F804C0E1
:10B440005FFA8CFC81F804C01A71DA6070471A2028
:10B45000EAE71020E8E70420E6E71620E4E70A2000
:10B46000E2E70920E0E70D20DEE70B20DCE71E2005
:10B47000DAE70220D8E70720D6E70620D4E7152030
:10B48000D2E72420D0E72520CEE712F4001F0CBF1E
:10B490004FF0FF302320C7E700C0074010B501F090
:10B4A0001BFBA0F11103EE2B98BF10383C4A3D4B1B
:10B4B0003D4994BFC0B2802050755A683B4842F065
:10B4C00080625A601A6842F080421A60CC68384A3A
:10B4D00004600023CB601178364B374CC9B2197029
:10B4E0005178C9B259709178C9B29970D178C9B2FE
:10B4F000D9701279D2B21A712378063B042B19D86D
:10B50000DFE803F0033C434827002C4A0321517035
:10B5100052784FF0E0231A69042122F002021A61E6
:10B52000C3F8101D30BF0022C3F8102D1A6942F075
:10B5300002021A611B4B1C4C5A68214942F080627E
:10B540005A601A6822F080421A600368E360086853
:10B5500010BD1A4A4FF0E0230021917092781A69C9
:10B56000042422F002021A61C3F8104D30BFC3F860
:10B57000101D1A6942F002021A61DBE70F4A4FF010
:10B58000E023032191709278C5E70C4A4FF0E02345
:10B590000221F7E7094A4FF0E0230121F2E700BF5B
:10B5A00000E400E00070044000900440C8A0FF1FC9
:10B5B000D0A0FF1F00C007401C94FF1F00E0074001
:10B5C0000082FF1F30B583B00F49009104460F4B36
:10B5D0000F4A002100F03EFA04F140050D490091A8
:10B5E0000D4B0E4A0121284600F034FA0223204672
:10B5F00084F88030C4F88440C4F88850C4F88C4083
:10B60000C4F8905003B030BD00B0034034D70100FF
:10B610003CD7010000B00B4038D7010068D70100CB
:10B6200090F821308B421ED001291DD061B9154AF6
:10B63000154B517083F84010436B80F821105B016B
:10B6400003F18443C3F8001472B6436B5B0103F14A
:10B650008443012200214276C3F89C14C3F8982445
:10B66000C3F89C2462B67047064B074A4FF0600C43
:10B6700083F800C04FF0E10C83F801C082F840105D
:10B68000DAE700BF004007400000FA4290F823309C
:10B690008B420AD070B4092900F29380DFE801F0F0
:10B6A0002F2F61060671818E40547047436B4FEA1D
:10B6B000431C0CF1844C0CF580730CF5C07C002409
:10B6C0000122CCF808202646DC610025CCF80C507D
:10B6D0001E605D605C619A6180F8231072B6436BF6
:10B6E0005B0103F18443012200214276C3F89C14DC
:10B6F000C3F89824C3F89C2462B670BC7047436BAF
:10B700004FEA431C0CF1844C0CF580730CF5C07CA3
:10B710000022CCF808200122DA6114461646D4E74C
:10B72000436B00245A0102F1844202F58073C2F88F
:10B73000884102F5C072DC610124D46000225C60A3
:10B740001C609A615A61C7E7436B5A0102F1844257
:10B7500002F5807302F5C072012494600024DC615C
:10B76000EAE7436B4FEA431C0CF1844C0CF5807301
:10B770000CF5C07C00260122CCF808601446DE617E
:10B78000A3E7436B4FEA431C0CF1844C0CF5807328
:10B790000CF5C07C00220124CCF808401646DA6182
:10B7A00093E7436B5A0102F1844202F5807302F57C
:10B7B000C072002494600124DC61BDE7436B012466
:10B7C000B0E7C38A9BB243F00103C38295E700BF91
:10B7D000436B5B0103F1844310B5D3F89C2403F55C
:10B7E0009063044652B103F059FD636B5B0103F1B2
:10B7F000844303F59063DA69002AF4D19B6923B18D
:10B80000E38A9BB243F00203E38272B6637E03B322
:10B81000626B936BD16B0B44116C506C0B44916C4D
:10B8200003440B44D16C0B44C3F34E0343F4004375
:10B83000D362936DD16D0B44116E506E0B44916EBB
:10B8400003440B44D16E0B44C3F34E0343F4004353
:10B85000136362B6A37E0022627603B910BD022193
:10B860002046FFF713FF637E03BB636B590101F1B1
:10B87000844201200021C2F81001C2F88011C2F8F0
:10B880008401627E022184F8241092B95B0103F1E5
:10B890008443002201200421C3F88804C3F88424CF
:10B8A000C3F8802484F82010A27610BDFFF790FF23
:10B8B000DBE72046FFF78CFF636BE7E738B5C37E15
:10B8C0008B4212D0437E04460D460BBB092D0DD88A
:10B8D000636B5B0103F184430020C3F80C01FF217B
:10B8E0000822C3F80801E161E27638BD0B2D12D9B8
:10B8F0000D2D1ED8636B5B0103F1844300220120F0
:10B90000C3F8080140F6FF71C3F80C210C22EAE7E6
:10B91000FFF75EFFDAE7636B5B0103F1844301220B
:10B920000020C3F8080140F2FF31C3F80C210A22BD
:10B93000D9E7636B5B0103F184430120C3F80C0179
:10B940004FF6FF711022C3F80801CCE738B5037E2B
:10B950003D4A0446002B6AD1D36B43F00063D363A6
:10B96000626B3A483A4940F201455201658402F15E
:10B9700084420425002384F824500125E376E36102
:10B9800084F8203084F82C306376E3826375C2F843
:10B990009051437081F84030626B84F8213052013D
:10B9A00002F18442C2F8003472B6626B65765201CD
:10B9B00002F18442C2F89C34C2F89854C2F89C54F4
:10B9C00062B60A212046FFF779FF637EA5769BBB0E
:10B9D000636B5B0103F1844301212022C3F88814C7
:10B9E0002046C3F88414C3F8801484F82020FFF79D
:10B9F0004DFE637E23BB636B590101F18443012239
:10BA00000020C3F81021C3F88021C3F8840184F812
:10BA1000242072B6636B62765B0103F18443C3F842
:10BA20009C04C3F89824C3F89C2462B638BD136BF9
:10BA300043F00063136393E72046FFF7C9FEC7E7AF
:10BA4000FFF7C6FED7E700BF008004400040074074
:10BA50000000FA4210B500298262094A03630CBF54
:10BA600039233A23017680F83C300649029B436330
:10BA700018BF114604468163FFF768FF204610BDDA
:10BA8000386003401060034038B5437E05460C46DD
:10BA9000A3B9042C0FD8DFE804F01E2D3C031400DA
:10BAA0006B6B5A0102F184430121C3F81011C3F8F2
:10BAB0008411C3F8801185F8244038BDFFF788FE53
:10BAC000E7E76B6B5B0103F184430022C3F81021AD
:10BAD00085F8244038BD6B6B5A0102F18443012183
:10BAE000C3F810110021C3F88411C3F8801185F840
:10BAF000244038BD6B6B5A0102F1844301210022BE
:10BB0000C3F81011C3F88011C3F8842185F82440CC
:10BB100038BD6B6B5A0102F1844301210022C3F846
:10BB20001011C3F88021C3F8841185F8244038BD72
:10BB300038B5437E04460D462BBB012D636B18D9E7
:10BB40005B0103F1844303F590630121042D9960A7
:10BB500006D8002159600422196084F8202038BDDD
:10BB6000082D13D9102D18D800221A601022596000
:10BB7000F3E75B01002103F184430A46C3F888140C
:10BB800084F8202038BDFFF723FED6E700200822E6
:10BB90001960586084F8202038BD5960202219604F
:10BBA000DBE700BF2B290BD8836A5B5C13F04003F3
:10BBB00006D0036B1A788A4205D09A788A4201D05F
:10BBC0000020704702335B7803F01F021F2AF7D072
:10BBD000426B520102F1844202F52062D26D0AB139
:10BBE000D809704701207047036B1A788A4220D029
:10BBF0009A788A4218BF1F221AD0436B5B0103F167
:10BC0000844303F52063DB6D83B902F01F0372B632
:10BC1000416B4A0102F184429269003A18BF012245
:10BC200003EB821320330B6062B670470223EEE70A
:10BC300002335A78E1E700BF2DE9F04F83B00446A4
:10BC40009046FFF7AFFF00286AD0627D0E46617E06
:10BC50000132627500295FD1606B94F81BB042011C
:10BC600002F1844202F58062D269151E18BF0125D7
:10BC7000002A3CD1A946AA462F46019500954001CD
:10BC800000F184400023C0F88C34424631462046FF
:10BC9000FFF7AAFF01E003F001FB636B5B0103F117
:10BCA000844303F58063DB69002BF4D172B6626BC9
:10BCB000530103F18443DB693BB31069BBF1100FFF
:10BCC00000B200D1400062B65DB172B6636B019AFA
:10BCD000C3F808A0C3F80C901A62009A5F621A6059
:10BCE00062B6637D013B637503B0BDE8F08F72B649
:10BCF000626B13680093D2F808A0D2F80C90136A14
:10BD00000193576A62B6606BB9E7E38A08489BB251
:10BD100043F08003E382D6E72046FFF759FD9BE717
:10BD2000E38A03489BB243F00403E382DCE700BFED
:10BD300090EEFEFF10B472B621B9026812B1037919
:10BD40000F2B41D9284C2188002341FA03F212F02D
:10BD5000010208D00133102BF7D162B60022026035
:10BD6000037110BC70474FF0010C0CFA03FC41EA60
:10BD70000C01218062B61D495FFA83FC80F804C083
:10BD80000C6C44F002040C64CC6B44F00204CC63F1
:10BD900003F10073A1F58021822403F590630C6008
:10BDA0005B0181F81AC081F81EC081F818C081F8C3
:10BDB0001FC010BC0360C3E90022C3E90222C3E92B
:10BDC0000422C3E906227047074C218841FA03FC8C
:10BDD0001CF0010FB8D003F1007303F59063B2EBD0
:10BDE000431FB1D162B6BCE7E0A0FF1F0080044052
:10BDF00003790F2B11D8094A937672B6084990F847
:10BE000004C00B88012202FA0CF223EA02030B8021
:10BE100062B6102200230271036070470080004068
:10BE2000E0A0FF1FEFF3108272B6437F5BB9017F82
:10BE3000012930B40BD0032913D00123437702B971
:10BE400062B630BC70470AB962B670477047124C90
:10BE50002168B1B1114943610B6883610860586181
:10BE6000EBE70F4D0F492C688CB143610B68836180
:10BE700058614FF0E0234FF080540860C3F8044D40
:10BE8000DBE7064B4161816120601860D5E74461C2
:10BE900084612860EDE700BFE4A0FF1FF4A0FF1F4E
:10BEA000ECA0FF1FE8A0FF1F70B5EFF3108272B681
:10BEB0000C4C206880B10C4E00254369236073B19F
:10BEC0009D6102B962B6836845779847EFF31082A7
:10BED00072B620680028F0D102B962B670BD336036
:10BEE000EFE700BFECA0FF1FE8A0FF1FFFF7DCBFDC
:10BEF000024A136801331360704700BF00A1FF1F9F
:10BF00000368C9B21B6818470368C9B21B681847A1
:10BF10000368C9B21B6818470368C9B21B68184791
:10BF20004B0803F1376303F5D83310B50446B3FB70
:10BF3000F1F001F041FA044B1B7803B110BD20462B
:10BF4000BDE8104003F022BA6D95FF1F08B5084602
:10BF500001F024FC012008BD08B5084601F01EFCD4
:10BF6000012008BD38B508460D460AF029FA0446F6
:10BF70000146284601F01CFC204638BD10B5084695
:10BF80001446114601F014FC204610BD0846114627
:10BF900001F03CBE0846114601F01CBE01F034BD64
:10BFA00008B5084601F0D0FB003818BF012008BDD5
:10BFB00008B5084601F0A6FB003818BF012008BDEF
:10BFC0000846114601F036BB084601F071BB00BFC0
:10BFD000084601F013BB00BF01F0AABA10B54B0828
:10BFE00003F13763144603F5D833B3FBF1F001F0E6
:10BFF000E3F92046BDE8104001F04CBA01F0DEBC88
:10C0000001F096BC01F080BC01F05ABC01F064BCA8
:10C010004B0803F1376303F5D83310B50446B3FB7F
:10C02000F1F001F003FE044B1B7803B110BD204674
:10C03000BDE8104003F0AAB96E95FF1F08B5084689
:10C0400001F0E2FF012008BD08B5084601F0DCFF61
:10C05000012008BD38B508460D460AF0B1F904467E
:10C060000146284602F04CF8204638BD10B5084677
:10C070001446114602F044F8204610BD0846114609
:10C0800002F06CBA0846114602F04CBA02F064B9EC
:10C0900008B5084601F098FF003818BF012008BD18
:10C0A00008B5084601F06EFF003818BF012008BD32
:10C0B0000846114601F0FABE084601F035BF00BF40
:10C0C000084601F0D7BE00BF01F06CBE10B54B08AA
:10C0D00003F13763144603F5D833B3FBF1F001F0F5
:10C0E000A5FD2046BDE8104001F00EBE02F00EB9DD
:10C0F00002F0C6B802F0B0B802F08AB802F094B804
:10C100000368064A1B68934205D110B5C8B201F016
:10C110007BFF012010BDC9B2184700BF49C0000015
:10C120000368064A1B68934205D110B5C8B201F0F6
:10C130006BFF012010BDC9B2184700BF49C0000005
:10C140000368064A1B68934205D110B5C8B201F0D6
:10C150005BFF012010BDC9B2184700BF49C00000F5
:10C160000368064A1B68934205D110B5C8B201F0B6
:10C170004BFF012010BDC9B2184700BF49C00000E5
:10C18000704700BF036830B403B300249C600124EF
:10C19000DC601A601A4A1B4C1A444FEA221C44F80D
:10C1A0002C100CF144014A1103249C6002F1382246
:10C1B000154B00790CF8030040320120920001F089
:10C1C0001F0100FA01F130BC116070470F4CE36BA6
:10C1D00043F40003E36300BF0D4B0E4D01241C60CC
:10C1E00003F5807303609C68002CD2D01033AB42FF
:10C1F0000360F8D10023036030BC1846704700BFCD
:10C20000008FFCBF4894FF1F44E400E0008004401E
:10C210000070034040710340F0B40468CCB10E4993
:10C220000E4E0F4F2144091101F14402531103F145
:10C23000382360339B00012502F01F0205FA02F249
:10C2400046F8217000211A60A160E560C3F8002162
:10C250000160F0BC704700BF008FFCBF4894FF1F17
:10C2600081C10000034A044B01211B68C2F80C1174
:10C27000184700BF007003404894FF1F034A044B57
:10C2800001215B68C2F81C11184700BF0070034011
:10C290004894FF1F034A044B01219B68C2F82C11EC
:10C2A000184700BF007003404894FF1F034A044B27
:10C2B0000121DB68C2F83C11184700BF0070034041
:10C2C0004894FF1F70B5012A8AB008BF0A22A1B3A3
:10C2D0004FF0210E02E05FFA86FE2946B1FBF2F52F
:10C2E00002FB15145FFA84FC092C0CF1300498BF92
:10C2F0005FFA84FC0EF1280488BF0CF1370C6C4403
:10C3000088BF5FFA8CFC91420EF1FF3604F824CC12
:10C31000E1D24BB10EF1FF3E5FFA8EFE0EF1280323
:10C320006B442D2203F8242C036801A95B68CEF12D
:10C330002202714498470AB070BD30228DF8252042
:10C340004FF0210EE5E700BF0029BABF49422D2377
:10C3500000230A22FFF7B6BF034B022888BF03461B
:10C3600018461B685B6818477095FF1F0EB400B530
:10C3700082B003AA52F8041B019207F0CBFF02B06F
:10C380005DF804EB03B07047F8B588424FF0000544
:10C390000446056045608560057302D08E680F68AD
:10C3A0000EB92046F8BD701C07F0F8FF0028F8D041
:10C3B000C4E900060570A660394608F08FFD2046E6
:10C3C000F8BD00BF10B50446006807F0EFFF204637
:10C3D00010BD00BFF8B50446154632B9036803B175
:10C3E0001A700023A3602046F8BD43689A420E46A7
:10C3F0001CD90068511C09F0A1FB074660B1A36875
:10C40000206065600BB903702768A5603146384627
:10C4100008F064FD2046F8BD206810B107F0C6FFA3
:10C42000276000236360A3602046F8BD0768A5600D
:10C430003146384608F052FDECE700BF38B500231E
:10C440000446036043608360037341B108460D46B0
:10C4500009F0B6FF294602462046FFF7BBFF2046FB
:10C4600038BD00BF38B505460C4649B1084609F04D
:10C47000A7FF214602462846FFF7ACFF284638BDF5
:10C48000A960284638BD00BF2DE9F843044600687E
:10C49000A36888420D46164609D8C218914206D2B2
:10C4A0000F1A4FF0010936B92046BDE8F8834FF066
:10C4B0000009002EF8D0626803EB060890450CD9FD
:10C4C00008F1010109F03AFB0028EDD0A368C4E9A6
:10C4D000000813B903702068A368B9F1000F08D1F0
:10C4E0002946184408F0FAFCC4F808802046BDE844
:10C4F000F8833246C119184400F0C8F923680022B5
:10C5000003F80820F0E700BF38B5054641B10846FA
:10C510000C4609F055FF214602462846FFF7B4FFB6
:10C52000284638BD10B582B000238DF804100122D2
:10C5300001A904468DF80530FFF7A6FF204602B09A
:10C5400010BD00BF826808B50B463AB161B1006802
:10C5500008F05AFBB0FA80F0400908BD31B11878F4
:10C56000B0FA80F0400908BD0368F8E7012008BD73
:10C5700038B52A4C2A4D01E002F090FE636A1B0692
:10C58000FAD46B6A13F08003F6D172B625490A78A3
:10C59000002A40D0A26BE06B0244206C0244606C25
:10C5A0000244A06C0244E06C0244C2F34E0242F426
:10C5B0000042E262A26DE06D0244206E0244606EB1
:10C5C0000244A06E0244E06E0244C2F34E0242F402
:10C5D00000422263AA6BE86B0244286C0244686C38
:10C5E0000244A86C0244E86C0244C2F34E0242F4D6
:10C5F0000042EA62AA6DE86D0244286E0244686E49
:10C600000244A86E0244E86E0244C2F34E0242F4B1
:10C6100000422A630B7062B638BD00BF00B0034011
:10C6200000B00B40FCA0FF1F2A4B2B4A6020E121E9
:10C630001870597013782948082B34D00A2B20D051
:10C640000C2B274B0CBF35213D2112228160C2608B
:10C650009960DA60234B21491B78214ACBB1012331
:10C660000B621362204B1D491B781D4A012B13D905
:10C67000042B1BD884234B6253621C4B01221A707B
:10C680007047174B392113228160C2609960DA60CC
:10C69000E0E70B621362E5E780234B625362134BC2
:10C6A00001221A7070470E4B0121ECE7082B06D8C7
:10C6B00085234B6253620D4B01221A707047102B79
:10C6C00094BF862387234B625362084B01221A7062
:10C6D000704700BF004007405894FF1F00B0034060
:10C6E00000B00B40FAA0FF1F5994FF1FFCA0FF1FD2
:10C6F000282829D8304B2DE9F0411E5CFF2E53D05D
:10C700002E4B1B7813BB340624D472B62C4C2D4D03
:10C7100001272E60277062B672B62B68180609D4FE
:10C720002378002BF5D062B602F0B8FD72B62B6804
:10C730001906F5D5234A00231069237062B6224BEF
:10C740001B781841BDE8F08100207047FFF710FF0B
:10C750003406DAD572B61D4D1D4C06F0400801278F
:10C7600006F03F06E368B8F1000F20D023F0100375
:10C77000E36026602F7062B672B623681A0609D489
:10C780002B78002BEED062B602F088FD72B62368DB
:10C790001B06F5D50E4A002310692B7062B60A4BB2
:10C7A0001B781841BDE8F0810020BDE8F08143F01E
:10C7B0001003E360DDE700BF6CD80100FCA0FF1FA1
:10C7C000F8A0FF1F00B00340FBA0FF1FF9A0FF1F50
:10C7D00000B00B400B4A0C49D36A43F48053D36238
:10C7E0000B784BB1094B802283F82120074B80F353
:10C7F0000C0000B218807047044BC02283F821203F
:10C80000F4E700BF00800440FAA0FF1F00C00C4006
:10C8100010B5174B0FCB84B0EC468CE80F00154BCE
:10C820005A78910717D51A78124C12F0700218BF77
:10C830001A7080210023E171332223710323E272F5
:10C84000A37272B64CF001032046984762B6237873
:10C8500013F0700309D1084B064901E0013B02D0F7
:10C860004A78D207FAD504B010BD237004B010BDC9
:10C8700098D8010000000240410D030008B5F9F707
:10C880006FFBF9F701FB02F009FDFAE701B441EA99
:10C89000000313F003036FD1403A41D351F8043B36
:10C8A00040F8043B51F8043B40F8043B51F8043B8A
:10C8B00040F8043B51F8043B40F8043B51F8043B7A
:10C8C00040F8043B51F8043B40F8043B51F8043B6A
:10C8D00040F8043B51F8043B40F8043B51F8043B5A
:10C8E00040F8043B51F8043B40F8043B51F8043B4A
:10C8F00040F8043B51F8043B40F8043B51F8043B3A
:10C9000040F8043B51F8043B40F8043B51F8043B29
:10C9100040F8043B51F8043B40F8043B403ABDD298
:10C92000303211D351F8043B40F8043B51F8043B3A
:10C9300040F8043B51F8043B40F8043B51F8043BF9
:10C9400040F8043B103AEDD20C3205D351F8043BC9
:10C9500040F8043B043AF9D204320AD0D2071CBF93
:10C9600011F8013B00F8013B03D30B7803704B78BF
:10C97000437001BC704700BF0C2A4AD310F0030378
:10C9800011D0C3F10403D21ADB071CBF11F8013B1D
:10C9900000F8013B07D311F8013B00F8013B11F807
:10C9A000013B00F8013B11F003033FF475AF30B4D5
:10C9B000043AC91AC3F1040C51F8044B022B19D0E4
:10C9C000032B0BD0240A51F8043B1D0644EA05044E
:10C9D00040F8044B1C46043AF4D216E0240E51F8F9
:10C9E000043B1D0244EA050440F8044B1C46043A8B
:10C9F000F4D20AE0240C51F8043B1D0444EA050477
:10CA000040F8044B1C46043AF4D20432B1EB0C015A
:10CA100030BC043AA0D3013A11F8013B00F8013BC5
:10CA2000F9D20B7803704B7843708B78837001BC1C
:10CA3000704700BF08B50F4C636B58030DD4636B90
:10CA400059050FD4636B1A0511D4636BDB04F3D55E
:10CA500000F012F8636B5803F1D501F051FE636BDF
:10CA60005905EFD500F0F4FF636B1A05EDD501F021
:10CA700097FCEAE70080044008B5FFF7DBFF00BF42
:10CA8000704700BF094A08B50346106833B16946CC
:10CA90000344A1F580518B4201D2136008BD05F01B
:10CAA000E9FF0C2303604FF0FF3008BD5C94FF1FCB
:10CAB000002070474FF0FF30704700BF4FF4005325
:10CAC0004B600020704700BF012070474FF0FF30DF
:10CAD000704700BFFEE7FFFFEFF31383CBB9EFF31F
:10CAE0001080A0B9EFF3058343B94FF48070EFF3E2
:10CAF00011835BB1984228BF184670470F2BF6D9B7
:10CB0000054AD05CEFF31183002BF3D17047184630
:10CB100070474FF0FF307047F0E300E007F03EBC95
:10CB200007F044BC01F1FF3C70B56546002401E00C
:10CB300070460134B0FBF2FE02FB1E03092B03F129
:10CB400030068ABF3733F3B2DBB2904205F8013FBB
:10CB5000EED2631C0022CA54C8187CB162461CF88D
:10CB6000015F10F801ED8CF800E0A1EB0C0302323C
:10CB7000013B521A23449A420570EFDB084670BD10
:10CB8000704700BF10B40F4B53F8302092F880422A
:10CB90002CB1012391B182F8803010BC704703EBB7
:10CBA000C0035B681A6821B922F0020210BC1A6047
:10CBB000704742F0030210BC1A60704782F80031DF
:10CBC00010BC7047BCD80100212835D8042A33D8BE
:10CBD00030B42A4B2A4D53F8223005EBC0021B0417
:10CBE0005468226812F4E06239D0264A2648C2F816
:10CBF0009C012648C2F8A0012548C2F8A401254896
:10CC0000C2F8A8012448C2F8AC0104F14042A2F5E0
:10CC100092207C2811D8214872B6226822F4702212
:10CC200022601343C4F3840243F0807340F822105F
:10CC3000236062B630BC70477047A2F594207C2810
:10CC400015D9A2F596207C2813D9A2F598207C2826
:10CC500011D9A2F59A227C2AECD81148DCE755F8C4
:10CC6000300080F880224FF480722260BDE70D48CA
:10CC7000D2E70D48D0E70D48CEE700BFA8D80100A5
:10CC8000BCD801000084FF1FF98DFF1FC58DFF1F59
:10CC9000918DFF1F5D8DFF1F298DFF1F6494FF1F66
:10CCA0003C95FF1F9C94FF1FEC94FF1F1C95FF1FDA
:10CCB0001A4B03EBC0035A6802F14043A3F59221DB
:10CCC0007C2905D9A3F594217C2914D8144900E0C6
:10CCD000144910B472B61368134C23F08773C2F36F
:10CCE000840023F4803343F08073136041F82040C4
:10CCF00062B610BC7047A3F596217C2909D9A3F52B
:10CD000098217C2907D9A3F59A237C2B05D80749BC
:10CD1000DFE70749DDE70749DBE77047BCD80100DB
:10CD20009C94FF1F6494FF1F81CB00003C95FF1F64
:10CD3000EC94FF1F1C95FF1F014B1868704700BF44
:10CD400000D00340034B002210215A615A60186042
:10CD50005961704700D00340704700BFF0B54FF0F5
:10CD6000E0244FF400054FF0807CC4F80851C4F86B
:10CD700008C14FF0007CC4F808C11D4A1D481E4977
:10CD80004FF0806CC4F808C1282300274BF6FF76CB
:10CD900009254FF0006CC4F808C183B05760966055
:10CDA000D3605361D3615362D3625363D3635364DB
:10CDB000156047608660C360436105604F608E60A8
:10CDC000CB604B610D60FFF72FFCFFF7C5FF0B4CED
:10CDD00023680093009B132BFAD902F04BF82368C9
:10CDE0000193019BB3F5967FF9D303B0F0BD00BF6B
:10CDF000008003400090034000800B4000A1FF1F13
:10CE000028287F4B36D000291B783FDD012202FA0B
:10CE100003FC614510B554D2C21E012A70D92028E6
:10CE200067D0192865D0774A926802FB011222FA6E
:10CE300003F3421F1B2A7DD8DFE812F0C600BF00B3
:10CE40007C007C00B800B1007C007C007C007C0091
:10CE50007C007C007C007C007C00AA00A3009C007D
:10CE600095007C00CD007C007C007C007C007C0078
:10CE70007C00D40018780B2895BFC0F10C000C384A
:10CE800001FA00F041FA00F0FFF7A4BC212817D8FE
:10CE90005D4B53F8302092F8801203EBC003002959
:10CEA0003CD001215B6882F8001101204FF4A2718F
:10CEB00082F8800219601A6822F020021A60704716
:10CEC0007047212814D8504B53F8301091F8804205
:10CED00003EBC00344B35B6881F880204FF4A27277
:10CEE000012081F880021A601A6822F020021A607C
:10CEF00010BD464A926802FB011222FA03F398E73A
:10CF0000434CA268042802FB011222FA03F270D1FA
:10CF1000404BA2614FF45171596310BD5B681968B1
:10CF200021F002011960C0E75B681A6842F0030251
:10CF30001A60D3E72128DBD87F29D4BF0021012143
:10CF4000FFF720FE304B03EBC00253F8301053685C
:10CF500001244FF4A27281F880421A601A6822F00C
:10CF600020021A6010BD27482B4A836140F24441D9
:10CF7000916010BD2348284A036140F2444151604A
:10CF800010BD2048254A036440F24441916110BD20
:10CF90001C48224A836340F24441516110BD194844
:10CFA0001D4A836240F24441116110BD15481A4A7E
:10CFB000036240F24441D16010BD1248174A036336
:10CFC00040F24441116110BD0E48144A836440F29E
:10CFD0004441D16110BD0D48114A83614FF4517134
:10CFE000D16410BD09480E4A03614FF45171916438
:10CFF00010BD084B22614FF45171196310BD00BF81
:10D000006094FF1F00800340BCD8010000800B40EB
:10D01000009003400090044000B0044000C0044071
:10D0200000A004400346102B28BF1023034A012B05
:10D0300038BF012310781370704700BF6094FF1F42
:10D040002DE9F0470E4680462C49304603F02AFD74
:10D050002B4B002847F6122712BF4FF0020A4FF061
:10D06000010A1F4600244FF05E5927FA04F003F02E
:10D0700023FB4946054603F077FB0146304603F0A3
:10D0800025FD30B90134072CEFD1F80903F014FB6A
:10D0900005463146284603F01BFC4FF07C5103F057
:10D0A00059FA03F04DFD4FF6FF73984228BF18461A
:10D0B000A8F10303012B11D9A8F105085FFA88F83C
:10D0C000B8F11B0F08D80F4A012303FA08F31A40DE
:10D0D00010D113F0016F0BD1BDE8F0870A4B00228D
:10D0E00044EACA041A605A6098601C60BDE8F08780
:10D0F000064BF5E7064B0022F2E700BF001BB740E6
:10D10000006CDC02338007000090034000800B407D
:10D1100000800340212816D810B4104B53F830205B
:10D1200092F880422CB1012371B982F8003110BC11
:10D13000704703EBC0035B681A6849B142F0030211
:10D1400010BC1A607047704782F8803010BC70477E
:10D1500022F0020210BC1A60704700BFBCD8010068
:10D16000212806D8044B53F8303093F80002C0B29F
:10D1700070470020704700BFBCD80100212820D88C
:10D180001B4A02EBC00301295B680FD004291DD0A4
:10D1900052F83000002280F8802299B1022922D072
:10D1A00003290DD14FF481721A60704752F8300094
:10D1B0004FF4A27280F880121A601A6822F02002DE
:10D1C0001A6070474FF480721A60704752F830103E
:10D1D0004FF4A272012081F880021A601A6842F0AE
:10D1E00020021A60704740F203121A60704700BFB5
:10D1F000BCD8010072B60D494FF0E022936908686F
:10D20000D2F8042D62B6520102D5322B88BF01300C
:10D21000074AC3F5BB334FF47A71FF33A2FB0323F4
:10D2200001FB00F000EB9310704700BF00A1FF1F4F
:10D23000ABAAAAAA2DE9F843044672B6204F4FF0D4
:10D24000E02293693D68D2F8042D62B6520102D5FE
:10D25000322B88BF01350CB9BDE8F883DFF8649044
:10D26000DFF86480A9EB0303A8FB03234FF47A7271
:10D2700002FB05F505EB93154FF0E02672B6B16998
:10D280003A68D6F804CD62B6A9EB0103A8FB030304
:10D290001CF0806FC5EB93134FF47A7002D03229E3
:10D2A00088BF013200FB0233B3F57A7F04D3013C1F
:10D2B000D2D005F57A75E1E701F0F0FFDEE700BFB7
:10D2C00000A1FF1FFF760100ABAAAAAA2DE9F84F23
:10D2D000314B1B6807460BB101221A70DFF8BC9076
:10D2E000DFF8BC8099F80040D8F800302D4D0134AB
:10D2F0009C422B782AD303F0FF0A002B3ED15446E0
:10D30000294EDFF8A8B005E033791B0623D42B782B
:10D31000A3420AD1FFF7E0FB4028F5DDFF28F6DD48
:10D3200001F0BCFF2B78A342F4D03F2C29D9204B2D
:10D33000403C1B68FFB21F551E4A1B4B0121117058
:10D34000BC2289F800A0DA70BDE8F88F9C425FFA31
:10D3500084FAD5D0E9E72B78D8F800105A1C8A4215
:10D36000DBB203D23F2A10D8D1B201E000210A4635
:10D370001BF80230DBB2F3712970C8E74FF0000AE6
:10D3800054460A4BFFB21F55D6E7D1B2084A3F3B7D
:10D390001268D35CDBB2EEE754A1FF1F9CA1FF1F14
:10D3A0005095FF1FA4A1FF1F00A006405CA1FF1F16
:10D3B000A0A1FF1F58A1FF1F2A4A2B49536B70B42D
:10D3C00043F48063294D536300232B70284E0B7068
:10D3D000284C2949237032780B7028490B709AB376
:10D3E000152A03D1264B40F213329A61254B1B7844
:10D3F000012B31D0052B03D1214B4FF45172DA614F
:10D400002028214B214C38BF2020C0F3443C83F816
:10D4100000C0C0F3471C00F01F0083F801C00422C5
:10D42000987202209A70D87488205A754FF0E021C3
:10D43000187440223C20D87084F82D204FF40053FB
:10D4400070BCC1F804317047114B40F213321A64BA
:10D450000C4B1B78012BCDD10D4B4FF451725A64FC
:10D46000CEE700BF0080044050A1FF1F48A1FF1F6E
:10D4700051A1FF1F9CA1FF1FA4A1FF1F58A1FF1FC7
:10D4800000C004405495FF1F00A0064000E400E0E7
:10D4900000A00440214B21499B7800F0030203F0D7
:10D4A000EC031343420700F00F0248BF43F01003A0
:10D4B000042A8B7003D18B7943F040038B71174B97
:10D4C000164A5B79C10603F0EF0348BF43F010032F
:10D4D00053719379820603F0EF03104A48BF43F07B
:10D4E000100310F40070937110D093780C4943F03E
:10D4F000A003937009780B4B0B4A03EBC10340F276
:10D5000047305B680949186011607047064B074A4D
:10D510001968914208BF1860704700BF00A006401C
:10D520005495FF1FBCD8010054A1FF1FD400D44262
:10D53000284B5B6B5B054CD510B5274C237823B18A
:10D5400001F0ACFE2378002BFAD1244A244B4FF093
:10D55000E0204FF400540021C0F88441D1701B78C2
:10D5600063B3152B1BD01F4B1B7803F07F03012BDC
:10D570001FD0052B0ED01C4B184A1C4C1C48196898
:10D5800092F804C0D27900232370037009B10123FB
:10D590000B7010BD174B40F20312DA61EBE7154B2D
:10D5A00040F203129A610F4B1B7803F07F03012BAB
:10D5B000DFD1114B40F203125A64DCE70E4B40F20C
:10D5C00003121A64074B1B7803F07F03012BD0D1A1
:10D5D000EFE770470080044058A1FF1F00A00640FD
:10D5E00051A1FF1F5495FF1F04A1FF1F48A1FF1F5A
:10D5F00050A1FF1F00C0044000A004400A4A38B5F3
:10D600000546137803F0FF04002BFAD101212846C8
:10D61000FFF7B4FD21462846FFF77CFD034A044B83
:10D6200052F835201A6038BD58A1FF1FBCD8010040
:10D6300054A1FF1F09B140F08000194A13788342BA
:10D6400017D010B4174C646B64050FD503F07F033B
:10D65000012B21D0052B14D0002900F07F0314BF2B
:10D6600060214421012B10D0052B03D0107010BC79
:10D67000704770470C4B41F44071D961107010BC79
:10D680007047094B0024DC61E6E7084B41F4407128
:10D690005964107010BC7047044B00245C64DBE7D5
:10D6A0005495FF1F0080044000C0044000A00440C7
:10D6B000104A137883420AD00F49496B490505D5B2
:10D6C000ABB1152B09D068B1152801D01070704787
:10D6D0000A4B40F213319961F8E7084B0021996138
:10D6E0000028F1D1064B40F213311964EEE70449EA
:10D6F0000B64E8E751A1FF1F0080044000C0044014
:10D7000000A004400D4B5B6B13F4806313D0212801
:10D7100003D90B4B0020186070470A4B10B5084C1A
:10D7200053F8303023600121FFF728FD23680022E1
:10D730001A70012010BD1846704700BF00800440D9
:10D7400004A1FF1FBCD80100104B5B6B13F4806376
:10D7500012D012280BD0142810D10D4B40F20232F7
:10D760005A610C4A537B01200343537370470A4BA1
:10D7700040F20232DA60F4E718467047054A537BFC
:10D7800003F0FE0300205373704700BF0080044085
:10D7900000C0044000A0064000A00440034B5B6BA7
:10D7A0005B0501D5FFF792BD704700BF00800440C4
:10D7B0002DE9F84F394B5B6B5A053CD5384B1B684C
:10D7C0000BB101221A704718B84231D2354EDFF83A
:10D7D000D880364CDFF8D89000F1010A13E003F04E
:10D7E000FF0B53B34FF0000B5D46324A1AF8013C71
:10D7F0005355524630490123BA420B700AF1010ACF
:10D8000086F800B014D23578D8F800300135AB4234
:10D810002378E4D9AB425FFA85FB0FD03F2DE4D9E2
:10D82000264B1AF8012C1B68403D5A555246E1E739
:10D830001F4BBC22DA70BDE8F88F5D466FF04303E2
:10D8400089F8033006E099F804301B060BD42378DE
:10D85000AB42E3D1FFF740F94028F4DDFF28F6DDC5
:10D8600001F01CFDF3E72378D8F800105A1C914210
:10D87000DBB203D93F2A0AD8D1B201E000210A461F
:10D880000C4B9B5CDBB289F807302170DFE7D1B22B
:10D890000A4A3F3B1268D35CDBB2F4E700800440E5
:10D8A00054A1FF1F9CA1FF1F5095FF1FA4A1FF1FA4
:10D8B00000A006405CA1FF1F58A1FF1FA0A1FF1FF1
:10D8C00010B5044C237823B101F0E8FC2378002B39
:10D8D000FAD110BD58A1FF1F084A094B11781A78D8
:10D8E0009142C8B2D3B202D2013B181A7047054A1E
:10D8F0001268013A1344181A704700BF9CA1FF1F19
:10D90000A4A1FF1F5095FF1F064A074B11781A78F4
:10D910009142D0B23CBF054A1268CBB238BF9B18C7
:10D92000181A704748A1FF1F50A1FF1F4C95FF1FF9
:10D930001B4B1C491A780B789A422ED010B55FFA0F
:10D9400082FE194AD8B21268431C9A4219D93F2B59
:10D950001BD85FFA83FC1548C05CC0B281F800C0D8
:10D960001349096861B19E453CBF7244D31A114AFC
:10D97000126828BFAEEB03039A4201D300230B7059
:10D9800010BD4FF0000C6346E5E70B4C3F382468B0
:10D99000205C5FFA83FCC0B2E0E74FF0FF307047D5
:10D9A00048A1FF1F50A1FF1F4C95FF1F08A1FF1F9B
:10D9B00004A1FF1F4895FF1F4CA1FF1F0D4A0E4BEE
:10D9C00011781B789942DAB211D00C490968531CBE
:10D9D000994207D93F2B06D9094B3F3A1B68985CFF
:10D9E000C0B270470023074AD05CC0B270474FF006
:10D9F000FF30704748A1FF1F50A1FF1F4C95FF1F2C
:10DA00004CA1FF1F08A1FF1F0C4B5B6B5B0514D5DE
:10DA10000B4B0C48DA78402102F0CB02DA705974D3
:10DA2000DA78094942F03402DA70084A0378126859
:10DA3000DBB20B700AB10023137070470080044002
:10DA400000A0064050A1FF1F48A1FF1F04A1FF1F17
:10DA50002DE9F041504C237913F0300F47D072B6C6
:10DA6000A37D03F0FF01002B58D062B6DFF82C81B4
:10DA70004B4898F800304B4A057816684A4F5FFAD1
:10DA800083FC4A4BEDB2D3F800E008E01DB14FF043
:10DA9000000C07F80C304A1E12F0FF0112D0E37997
:10DAA0000CF101029642DBB2F0D99542ACF13F0095
:10DAB000F1D03F2A6DD994464A1E12F0FF010EF8AC
:10DAC0000030ECD15FFA8CF388F80030384B1968DD
:10DAD00069B1AC453CBF721B02EB0C03354A1268BE
:10DAE00028BFACEB05039A429CBF01230B702A4868
:10DAF000C3781E06DDB216D46A060DD5264B1B79F7
:10DB00005B0609D52C4B2D491B6800220A7003B116
:10DB10001A70214B3C22DA70BDE8F0814023E27993
:10DB2000637462B6E3E703791C06E5D5244B254A06
:10DB3000DFF894E01C7816689EF80030234A244FE2
:10DB4000D2F800C0E4B2DBB207E003790023FA5C4C
:10DB5000D2B2C271027D072A11D8A34203F101019A
:10DB60000ED08E42F1D93F290279A3F13F0301D8AB
:10DB70000B46ECE71CF803200B46D2B2E9E7DCB217
:10DB8000054B8EF800401A79110644BF7C22DA70EA
:10DB9000B2E794467DE700BF00A0064048A1FF1F02
:10DBA00050A1FF1F4C95FF1F08A1FF1F4CA1FF1F95
:10DBB00004A1FF1F4495FF1F54A1FF1F58A1FF1F81
:10DBC0009CA1FF1F5095FF1FA4A1FF1FA0A1FF1F35
:10DBD0005CA1FF1F094B10B4186060B101F1400453
:10DBE000074B084801F11A021A60074B04602831FC
:10DBF00010BC196070474024F2E700BF4CA1FF1F22
:10DC00004895FF1F4C95FF1F4495FF1F054B18605B
:10DC100018B1054B403119607047034B4021196022
:10DC2000704700BFA0A1FF1F5095FF1F2A4A2B4934
:10DC3000536B70B443F40063294D5363294E2A4C4F
:10DC4000327800232B700B70284923700B70284901
:10DC5000092A0B7033D01A2A03D1264B40F2133213
:10DC60005A60254B1B780A2B31D01F2B03D1214B37
:10DC70004FF451721A602028204B214C38BF2020CD
:10DC8000C0F3443C83F800C0C0F3471C00F01F0001
:10DC900083F801C00422987202209A70D8748820F8
:10DCA0005A754FF0E021187440223C20D87084F857
:10DCB0002F204FF4004370BCC1F804317047114B62
:10DCC00040F21332DA600C4B1B780A2BCDD10D4B8E
:10DCD0004FF451721A61CEE700800440F4A1FF1F97
:10DCE000ECA1FF1F6495FF1F28A2FF1F30A2FF1F9A
:10DCF000FCA1FF1F00D004406C95FF1F00B0064040
:10DD000000E400E000B00440214B21499B7800F082
:10DD1000030203F0EC031343420700F00F0248BF75
:10DD200043F01003042A8B7003D18B7943F0400336
:10DD30008B71174B164A5B79C10603F0EF0348BF9E
:10DD400043F0100353719379820603F0EF03104AF6
:10DD500048BF43F0100310F40070937110D0937813
:10DD60000C4943F0A003937009780B4B0B4A03EB6B
:10DD7000C10340F247305B68094918601160704781
:10DD8000064B074A1968914208BF1860704700BFE8
:10DD900000B006406C95FF1FBCD80100F8A1FF1F22
:10DDA000D400D642294B5B6B1B054DD510B5284CD2
:10DDB000237823B101F072FA2378002BFAD1254A97
:10DDC000254B4FF0E0204FF400440021C0F884417F
:10DDD000D1701B78092B2CD01A2B1BD01F4B1B7812
:10DDE00003F07F030A2B1FD01F2B0ED01C4B194AA8
:10DDF0001C4C1D48196892F804C0D2790023237086
:10DE0000037009B101230B7010BD184B40F20312CF
:10DE10001A60EBE7154B40F203125A600F4B1B7868
:10DE200003F07F030A2BDFD1114B40F203121A617A
:10DE3000DCE70F4B40F20312DA60084B1B7803F06B
:10DE40007F030A2BD0D1EFE7704700BF008004406A
:10DE5000FCA1FF1F00B006406495FF1F6C95FF1FDB
:10DE6000A8A1FF1FECA1FF1FF4A1FF1F00D00440D9
:10DE700000B004400A4A38B50546137803F0FF04A1
:10DE8000002BFAD101212846FFF778F921462846D0
:10DE9000FFF740F9034A044B52F835201A6038BDA9
:10DEA000FCA1FF1FBCD80100F8A1FF1F09B140F081
:10DEB0008000194A1378834217D010B4174C646B52
:10DEC00024050FD503F07F030A2B21D01F2B14D07C
:10DED000002900F07F0314BF602144210A2B10D0D9
:10DEE0001F2B03D0107010BC704770470C4B41F4CF
:10DEF00040711960107010BC7047094B00241C6001
:10DF0000E6E7084B41F440711961107010BC70478E
:10DF1000044B00241C61DBE76C95FF1F008004406C
:10DF200000D0044000B00440124B1A7882420CD05A
:10DF30001149496B090507D5092A16D01A2A0AD0B2
:10DF400009280DD01A2801D0187070470B4A40F2EA
:10DF500013315160F8E7094A002109285160F1D1D5
:10DF6000074A40F21331D160EEE7054A0021D16043
:10DF7000E6E700BF6495FF1F0080044000D0044026
:10DF800000B004400D4B5B6B13F4006313D02128E9
:10DF900003D90B4B0020186070470A4B10B5084C92
:10DFA00053F8303023600121FFF7E8F8236800229E
:10DFB0001A70012010BD1846704700BF0080044051
:10DFC000A8A1FF1FBCD801000C4B5B6B13F40063CE
:10DFD00012D0172809D10A4B0A4A40F2023199603F
:10DFE000537B0120034353737047064A537B03F06E
:10DFF000FE030020537370471846704700800440AA
:10E0000000B0044000B006402DE9F84F334B5B6B85
:10E010001A053AD5324B1B6806460BB101221A701D
:10E02000DFF8C090DFF8C08099F80040D8F80030E1
:10E030002E4D0134A3422B7829D99C425FFA84FAF1
:10E0400014D12B4FDFF8ACB005E03B791B0623D48D
:10E050002B78A3420AD1FEF73FFD4028F5DDFF28CB
:10E06000F6DD01F01BF92B78A342F4D0272C29D937
:10E07000214B283C1B68F6B21E55204A1C4B01213F
:10E080001170BC2289F800A0DA70BDE8F88F03F0A7
:10E09000FF0AA3B95446D4E72B78D8F800105A1CCD
:10E0A0009142DBB208D9272A10D8D1B21BF802302E
:10E0B000DBB2FB712970CBE700210A46F6E74FF08F
:10E0C000000A54460B4BF6B21E55D6E7D1B20A4AA7
:10E0D000273B1268D35CDBB2EBE700BF0080044053
:10E0E000F8A1FF1F28A2FF1F6895FF1F30A2FF1F86
:10E0F00000B0064000A2FF1F2CA2FF1FFCA1FF1FC3
:10E100002DE9F84F394B5B6B1A053CD5384B1B6832
:10E110000BB101221A704718B84231D2354EDFF8E0
:10E12000D880364CDFF8D89000F1010A13E003F0F4
:10E13000FF0B53B34FF0000B5D46324A1AF8013C17
:10E140005355524630490123BA420B700AF1010A75
:10E1500086F800B014D23578D8F800300135AB42DB
:10E160002378E4D9AB425FFA85FB0FD0272DE4D9A1
:10E17000264B1AF8012C1B68283D5A555246E1E7F8
:10E180001F4BBC22DA70BDE8F88F5D466FF0430389
:10E1900089F8033006E099F804301B060BD4237885
:10E1A000AB42E3D1FEF798FC4028F4DDFF28F6DD12
:10E1B00001F074F8F3E72378D8F800105A1C914264
:10E1C000DBB203D9272A0AD8D1B201E000210A46DE
:10E1D0000C4B9B5CDBB289F807302170DFE7D1B2D2
:10E1E0000A4A273B1268D35CDBB2F4E700800440A4
:10E1F000F8A1FF1F28A2FF1F6895FF1F30A2FF1F75
:10E2000000B0064000A2FF1FFCA1FF1F2CA2FF1FB1
:10E2100010B5044C237823B101F040F82378002B8B
:10E22000FAD110BDFCA1FF1F084A094B11781A78DA
:10E230009142C8B2D3B202D2013B181A7047054AC4
:10E240001268013A1344181A704700BF28A2FF1F32
:10E2500030A2FF1F6895FF1F064A074B11781A78F6
:10E260009142D0B23CBF054A1268CBB238BF9B186E
:10E27000181A7047ECA1FF1FF4A1FF1F6095FF1F44
:10E280001B4B1C491A780B789A422ED010B55FFAB6
:10E2900082FE194AD8B21268431C9A4219D93F2B00
:10E2A0001BD85FFA83FC1548C05CC0B281F800C07F
:10E2B0001349096861B19E453CBF7244D31A114AA3
:10E2C000126828BFAEEB03039A4201D300230B7000
:10E2D00010BD4FF0000C6346E5E70B4C3F38246857
:10E2E000205C5FFA83FCC0B2E0E74FF0FF3070477C
:10E2F000ECA1FF1FF4A1FF1F6095FF1FACA1FF1F42
:10E30000A8A1FF1F5C95FF1FF0A1FF1F0D4A0E4B38
:10E3100011781B789942DAB211D00C490968531C64
:10E32000994207D93F2B06D9094B3F3A1B68985CA5
:10E33000C0B270470023074AD05CC0B270474FF0AC
:10E34000FF307047ECA1FF1FF4A1FF1F6095FF1F76
:10E35000F0A1FF1FACA1FF1F0C4B5B6B1B0514D57D
:10E360000B4B0C48DA78402102F0CB02DA7059747A
:10E37000DA78094942F03402DA70084A0378126800
:10E38000DBB20B700AB100231370704700800440A9
:10E3900000B00640F4A1FF1FECA1FF1FA8A1FF1FC2
:10E3A0002DE9F041504C237913F0300F47D072B66D
:10E3B000A37D03F0FF01002B58D062B6DFF82C815B
:10E3C0004B4898F800304B4A057816684A4F5FFA78
:10E3D00083FC4A4BEDB2D3F800E008E01DB14FF0EA
:10E3E000000C07F80C304A1E12F0FF0112D0E3793E
:10E3F0000CF101029642DBB2F0D99542ACF13F003C
:10E40000F1D03F2A6DD994464A1E12F0FF010EF852
:10E410000030ECD15FFA8CF388F80030384B196883
:10E4200069B1AC453CBF721B02EB0C03354A126864
:10E4300028BFACEB05039A429CBF01230B702A480E
:10E44000C3781E06DDB216D46A060DD5264B1B799D
:10E450005B0609D52C4B2D491B6800220A7003B1BD
:10E460001A70214B3C22DA70BDE8F0814023E2793A
:10E47000637462B6E3E703791C06E5D5244B254AAD
:10E48000DFF894E01C7816689EF80030234A244F89
:10E49000D2F800C0E4B2DBB207E003790023FA5CF3
:10E4A000D2B2C271027D072A11D8A34203F1010141
:10E4B0000ED08E42F1D927290279A3F1270301D882
:10E4C0000B46ECE71CF803200B46D2B2E9E7DCB2BE
:10E4D000054B8EF800401A79110644BF7C22DA7091
:10E4E000B2E794467DE700BF00B00640ECA1FF1FF5
:10E4F000F4A1FF1F6095FF1FACA1FF1FF0A1FF1F3C
:10E50000A8A1FF1F5895FF1FF8A1FF1FFCA1FF1F27
:10E5100028A2FF1F6895FF1F30A2FF1F2CA2FF1F1C
:10E5200000A2FF1F094B10B4186060B101F1400454
:10E53000074B084801F11A021A60074B04602831A2
:10E5400010BC196070474024F2E700BFF0A1FF1F24
:10E550005C95FF1F6095FF1F5895FF1F054B1860C6
:10E5600018B1054B283119607047034B28211960F9
:10E57000704700BF2CA2FF1F6895FF1F704700BFA8
:10E58000704700BF431E032B17D872B60C4951F8D1
:10E59000230080B110B40B4CB0F800C034F8132045
:10E5A000A2EB0C02D0F804C041F823C024F81320D9
:10E5B00062B610BC704762B670470020704700BF5B
:10E5C000C4A2FF1F14A3FF1F013803280BD872B683
:10E5D000074B53F8203043B100205B680130002B1B
:10E5E000FBD162B67047002070471846F9E700BFBC
:10E5F000ECA2FF1F10B472B6194A1A4C042312F889
:10E60000011B090743F0010C05D554F8331061B123
:10E6100054F83C10B9B10433142BF0D162B6124B4C
:10E6200000221A7010BC00F09DBC0F4904EBC3021D
:10E63000083050600A780D4844F83300013A0A70F7
:10E6400062B610BC7047084A094904EBCC03083095
:10E650005860137844F83C10013B137062B6F0E741
:10E6600048DA01000080FF1F1CA3FF1F8800400044
:10E67000C8004000421E032A0ED81C4B400140F047
:10E68000100010B4034472B6194CA05C03281CD8C7
:10E69000DFE800F01315031870470520A05413F0AD
:10E6A000080F088814BFC8228822083142EA0042B5
:10E6B00059601A6062B610BC70470320EEE7083359
:10E6C0000220EBE708330420E8E70A4B53F8220066
:10E6D00038B1094B53F82200416043F8221062B66A
:10E6E000E9E743F82210044BF7E700BF0080FF1F63
:10E6F0000CA3FF1FECA2FF1FFCA2FF1F00BE00BF68
:10E700002DE9F04FDFF8CCA2DFF8CCB285B03DE0C8
:10E71000B24D9E0805EBC607013A796813F008036D
:10E72000D4B2A1F1080040F0B88055F836204FEA85
:10E73000124C120C21F808CC00F0A78021F8063CFE
:10E7400041F8043CA64B53F82420002A00F0018233
:10E75000A44B53F82420506043F82400A24B33F814
:10E760001420944423F814C000F0DCFB002800F0CF
:10E77000E98117F0080F9D4B00F1080018BF5B46B8
:10E78000786045F8363008238AF880309AF880306F
:10E790005907DCB21BD5964B1B78ABB195490A786B
:10E7A00002F0FF032AB1013BDBB20B70002B00F03B
:10E7B000468391490A7802F0FF032AB1013BDBB29C
:10E7C0000B70002B00F0EB8104238AF8803014F0EA
:10E7D000080200F0CC819AF89020D3B2120997D1A8
:10E7E000DFF8F8919B0809EBC30459F8330064681B
:10E7F000C0F3830009287CD00FD80138012808D83D
:10E800007E4A158842F22100854200F0FB8149F8DA
:10E8100033B001238AF89430B5E70D28F9D1D4E953
:10E820000007774D49F833B0744E764CC9F8102084
:10E8300083B240F2816CC9F818202A6063454FF01A
:10E840000102C6E90007227000F2FF80B3F5D06F25
:10E8500080F0CB82B3F5817F00F0268240F2DE802B
:10E8600040F2023293427BD107F07F07042F00F27F
:10E870000881020C40F00581634911F8273043F00C
:10E88000020301F82730134670E017F0080F574BCA
:10E8900018BF5B4645F8363075E700F063FB5B490F
:10E8A0005B4A51F82430002B00F05781586841F83A
:10E8B0002400115D03F108007860032905D8DFE822
:10E8C00001F0120F1502042111551A8817F0080FD4
:10E8D00014BFC823882343EA024345F8363052E781
:10E8E00002211155F1E703211155EEE705211155DC
:10E8F000EBE7434D2A683AB34649424C0F884648F5
:10E9000094F800E00678402F3B4628BF4023BEF134
:10E91000000F8EF0010E84F800E046F0020486F04D
:10E920000106067009EBC400426014BFC8208820AD
:10E9300040EA03401A44FB1A9BB249F834000B80AA
:10E94000002B00F036812A602C4B1A88B2F5A06F9C
:10E950007FF45FAF9A788AF8982000225A7058E7BF
:10E96000B3F5A06F40F08D8000221346B6F806C0C4
:10E970002948944528BF944667460278402F28BF0F
:10E98000402742F0020E3E0409EBCE0846F0C806CE
:10E99000C8F8043049F83E6000263B442670BCEBC2
:10E9A000070782F00106067040F01181BCF13F0FAD
:10E9B0004FF0010509D946F00206027009EBC602C4
:10E9C00025705360882349F8363001238AF8943043
:10E9D0001FE700BF00200740C80040000080FF1F65
:10E9E000C4A2FF1FD4A2FF1F14A3FF1F8800400072
:10E9F00010A3FF1F11A3FF1F3CA3FF1FE4A2FF1FD3
:10EA0000B8A2FF1FB5A2FF1FC0200740ECA2FF1F46
:10EA10000CA3FF1FB6A2FF1FB4A2FF1F802B00F0A4
:10EA20008B81822B2DD107F07F07042F29D8A74A8D
:10EA300000231380A64B13F827309F0740F1FC8179
:10EA400001231370A14B022290E742F2210C63458F
:10EA5000BBD01DD942F2212293420DD1BFB2002F6B
:10EA600082D19C4B1A689C4B1A609C4BC0F30740A8
:10EA700000221870134679E742F2213293423FF4A4
:10EA800073AF0F238AF8C03001238AF89430C0E6B0
:10EA9000B3F5086F00F04A81B3F5106FF1D1904BD8
:10EAA000C0F307400425187059F835301A0606D40B
:10EAB0000135142D0CD059F835301A06F8D509EB6C
:10EAC000C50301355868083800F04CFA142DF2D10E
:10EAD000844A854B0292854A0192854E854ADFF829
:10EAE00018820394009200251C4656F8047B2FB12F
:10EAF00038467F6800F036FA002FF9D1009BD8F82D
:10EB0000007043F8045B46F8045C00932FB138466C
:10EB10007F6800F027FA002FF9D1029B48F8045BC8
:10EB200043F8045B0293019B23F8025B0193237873
:10EB3000023B032B00F20981DFE813F03F010401DF
:10EB40003F0104016D4A45F8360013780133137014
:10EB500019E643F82400674BFEE5115D022926D033
:10EB60007FF611AE03291DD1012313550BE6E007F3
:10EB70006ED4210621D4A20708D5614B93F88820D2
:10EB80000221D2B283F8882083F88010E30603D5EF
:10EB90005B4B102283F8802005B0BDE8F08F00F0B9
:10EBA00059FB11E617F0080F14BF03230223135576
:10EBB000E9E53F2F98BF0022C5E6514B80220D2189
:10EBC00083F8C01083F88020A207DFD5D5E746F090
:10EBD00002060270402F09EBC6003A4628BF4022C9
:10EBE00043601004134440F088000121BA1A49F828
:10EBF0003600217055D02B60424B1A8001238AF8D1
:10EC0000943006E692885AB93F4AE51D14F8011B74
:10EC100002F8011FAC42F9D13C4A1268862A3CD066
:10EC20003B4C3C4825780278002D85F00105257085
:10EC300042F0020482F00102027009EBC4024FF0BC
:10EC40000000506014BFC822882249F83420DEE555
:10EC50002B4B30483049314C022583F894500270D8
:10EC60002F480C602F4D48608C600D24CD60FF2034
:10EC70000A618A6183F8C04001219F2483F88800DB
:10EC800083F8800083F8982083F88C0083F8844010
:10EC900083F8941005B0BDE8F08F234A0F20107060
:10ECA000BEE73F2FA7D890E607F07F07042F3FF677
:10ECB000E8AE000C7FF4E5AE054A12F8273023F0E9
:10ECC000020302F82730002213464FE6BCA2FF1FC2
:10ECD000C020074000A1FF1F38A3FF1F34A3FF1F60
:10ECE00010A3FF1FFCA2FF1F0CA3FF1F14A3FF1FF5
:10ECF000C4A2FF1FD4A2FF1FECA2FF1F1CA3FF1F73
:10ED000000200740B6A2FF1F2BA3FF1F2CA3FF1F4D
:10ED1000B5A2FF1FB4A2FF1F0080FF1F88004000A4
:10ED200034A2FF1F74A2FF1F11A3FF1F484B4949C4
:10ED30001B780B700B4619E6464A00231380454B9F
:10ED4000022213E64FF001032370434BB34204F158
:10ED500001047FF4CAAE414E039CDFF80481414FA9
:10ED600000233370042518F8013B3F4AAB541B07BE
:10ED700025D445F0020145F0030204350023142D8B
:10ED800049F8313049F83230EDD1384F25783A78AA
:10ED900042F0020009EBC00C85F00106CCF804300B
:10EDA000002D4DD1882382F0010226703A7049F877
:10EDB000303001238AF894302BE52570C5E700F048
:10EDC000B1F8002832D009EBC5030830586049F883
:10EDD000357000F0A7F808B345F0010309EBC30252
:10EDE0000830506049F833B0C3E7214A5368002B1C
:10EDF0003FF447AE000CBFB204E013690C32002BA5
:10EE00003FF43FAE11888142F7D15188B942F4D125
:10EE1000000A03280CBF1A781289A7E5337801335A
:10EE2000337045F0010349F83300A2E7337849F81D
:10EE3000350001333370CCE7064B022296E500BE65
:10EE40002670C82382F001063E7049F83030BCE5D8
:10EE500010A3FF1FBCA2FF1FD4A2FF1F1CA3FF1FF4
:10EE600048DA010088004000C0200740B4A2FF1F1C
:10EE7000F4D9010070B500F0B3FA00231A4A19461C
:10EE800042F8331002EBC3000133142B4160F7D179
:10EE9000164C174B606B174D40F480206063C2F333
:10EEA000072483F89C40144CFF204FF0010CC2F360
:10EEB0000746120E83F8B0604FF0E02E83F8B420BE
:10EEC00083F8800083F88800187483F894C0217058
:10EED00083F884C0702385F849304FF40072102302
:10EEE000CEF80821237270BD0080FF1F008004400F
:10EEF0000020074000E400E00021074000F0ACB82B
:10EF000000F07CB800F056B800F090B800F076B988
:10EF100000F050B90846114600F0BAB8084600F0B3
:10EF20003BB900BF72B60D490B68B3FA83F00B28EA
:10EF300010DC4FF00042C24023EA02030B6062B6CD
:10EF4000074A00EBC000C10002EBC0000023535091
:10EF50004360704762B60020704700BF8095FF1F76
:10EF6000BC85FF1F0E4BC31AB3F5587F10D20D4A54
:10EF7000127872B972B60C4A0C49A2FB03230868D6
:10EF80004FF000421B0922FA03F303430B6062B601
:10EF90007047074A1278002AECD0FFF72BBB00BF5E
:10EFA000BC85FF1F1CA3FF1F398EE3388095FF1F10
:10EFB00010A3FF1F38B50F4C206878B14388028832
:10EFC000C11801339A420D7A02D94380284638BDD0
:10EFD000FFF7C8FF00232360284638BD064B1B7887
:10EFE0002BB10320FFF7CEFA20600028E6D14FF0C6
:10EFF000FF35EBE720A3FF1F10A3FF1F10B5094C3F
:10F00000206818B143881844007A10BD064B1B785D
:10F010002BB10320FFF7B6FA20600028F2D14FF0A1
:10F02000FF3010BD20A3FF1F10A3FF1F084B094A8C
:10F030001B6810B594881BB11A885B88D31A1C44CE
:10F040000CB1204610BD00F029F9204610BD00BFCC
:10F0500020A3FF1F14A3FF1F0B4B1B789BB110B500
:10F060000A4C206848B1FFF77DFF0023032023608E
:10F07000FFF788FA30B1FFF775FF0320FFF782FA38
:10F080000028F8D110BD704710A3FF1F20A3FF1F59
:10F090002DE9F04FDFF8EC9083B0012289F80020D1
:10F0A000019179B3384FDFF8E480019D384EDFF8E5
:10F0B000E4A083463968A1B3B1F802E0CEF1400C78
:10F0C000AC4528BFAC460EEB0C040022A4B2327053
:10F0D000A5EB0C054C8001F10802BCF1000F0AD031
:10F0E0000EF1FF3E7244DC441BF8014B02F8014F65
:10F0F000DC45F9D14C883F2C0BD805228AF800203A
:10F10000002DD7D10198002389F8003003B0BDE865
:10F11000F08F40220A800420FFF7ACFA00223A6008
:10F12000EBE798F800202AB34AF2F92408E0013C02
:10F1300019D03278BAB900F0B1F898F80020CAB105
:10F140000420FFF741FA0728F1D84FF0010389F8AE
:10F150000030FFF7E7FE014638600028ACD1013CE3
:10F1600089F80000E5D101234FF0FF30337003B080
:10F17000BDE8F08F00234FF0FF3089F8003003B076
:10F18000BDE8F08F25A3FF1F28A3FF1F10A3FF1FBB
:10F1900024A3FF1F3CA3FF1F00B583B0034601213A
:10F1A0000DF107008DF80730FFF772FF03B05DF82F
:10F1B00004FB00BF38B50E4D0E4C286801232370A8
:10F1C00028B140880023C0F14000237038BD0A4BAD
:10F1D0001B7813B90020207038BD0420FFF7F4F924
:10F1E0000728F7D8FFF79EFE28600028E9D1F1E74D
:10F1F00028A3FF1F25A3FF1F10A3FF1FF8B5114B66
:10F200001B788BB1104E114D346801272F7064B1FB
:10F210000F4B00271F706388238021460420FFF7CF
:10F2200029FA376000232B70F8BDFFF77BFE084BEF
:10F23000014620B104201C70FFF71CFAF2E71F7092
:10F24000F0E700BF10A3FF1F28A3FF1F25A3FF1F88
:10F250003CA3FF1F38B50E4B1B7853B90D4C2168EA
:10F2600041B103F0FF054B880B800420FFF702FA41
:10F27000256038BDFFF756FE014620B1BDE8384095
:10F280000420FFF7F7B9044B01221A7038BD00BF04
:10F2900025A3FF1F28A3FF1F3CA3FF1F2DE9F84351
:10F2A000324E337863B1324F3A784AB90122D907E6
:10F2B0003A7043D49A0726D400225B073A7001D4EF
:10F2C000BDE8F8832B4B1A68002AF9D0EFF30582CA
:10F2D000002AF5D1EFF3108572B6186800283AD0ED
:10F2E000254C2178002936D142691A600123237008
:10F2F000002A37D0916105B962B600258368457749
:10F3000098472570DCE7DFF8748098F80020002A21
:10F31000D2D00025DFF868902B4659F823402368A7
:10F3200020461B690135984708B12369984798F82A
:10F330000020EBB29A42F0D83378BDE7FFF776FEB3
:10F3400068B9104B1B780BB93378B3E7337803F007
:10F35000FE033370AEE7002DB2D162B6B0E700F025
:10F360003DF8EEE7084B1A60C5E700BF8495FF1F24
:10F370003DA3FF1FE4A0FF1FF0A0FF1F4CA3FF1F32
:10F3800040A3FF1F94D70100F4A0FF1F70B4104EDC
:10F39000104D3478D4B1621ED2B2291D2B4601EB38
:10F3A000820101E08B4205D053F8042B8242F9D14F
:10F3B00070BC7047631CDBB2074A3370137845F8A2
:10F3C000240043F00203137070BC70470123F3E77D
:10F3D0004CA3FF1F40A3FF1F8495FF1F704700BF72
:10F3E00010B584B072B6174A702441200F218023D3
:10F3F0001470D0719171137013781B06FCD590684E
:10F4000062B6114B114C984238BF00EB800001A945
:10F4100038BF40000A22FDF785FB01A920460023E2
:10F4200011F8012B01333AB10A2B20F8022FF7D142
:10F430001623237004B010BD5B00DBB2237004B050
:10F4400010BD00BF00000240809698001496FF1F78
:10F4500008B5C0F3C7537F3B162B014615DC002BC4
:10F4600002460BDB0B481841014205D04FF48001E6
:10F470001941114421EA0001084608BD013300F09A
:10F480000041F9D141F07E51F6E7802BF4D101F033
:10F4900063F808BDFFFF7F00F8B504460D4600F095
:10F4A00023F8224606460F462B462046294600F002
:10F4B0009FFF30B9204629460022002300F070FF4C
:10F4C00010B930463946F8BD03F0D4FA00220023C3
:10F4D000212101601046194600F01AFE06460F462B
:10F4E00030463946F8BD00BF2DE9F84F714E8E43C6
:10F4F00005460C4600F0A580002902460B4651DD6A
:10F5000008155DD0C3F31301C307A0F2FF3641F421
:10F51000801103D4490001EBD2715200D30F0025B2
:10F5200003EB4103761052001620AC464FF4001155
:10F530000CEB01049C4203DC1B1B04EB010C0D448F
:10F540005B00013803EBD2734FEA51014FEA4202EC
:10F55000EED1074620244FF0004109E040D05B0087
:10F56000013C03EBD2734FEA51014FEA420241D012
:10F57000634501EB000EF1DDBEF1000F0EEB010063
:10F580000BDBE046A3EB0C03964588BF03F1FF338A
:10F59000A2EB0E020F44C446E1E70028F1DB0CF1B8
:10F5A0000108EFE721F00046064346D000296FD15D
:10F5B0000846D30A15385205002BFAD0DE0274D45F
:10F5C00000215B00DD020C4601F10101F9D5154671
:10F5D0008A40C1F1200125FA01F1001B0B4391E79C
:10F5E0009645BCD8BEF1000F0EEB0100D5DB984666
:10F5F0000023CDE7134312D0DFF8BCA0DFF8BCB086
:10F60000DAE90001DBE9002300F0A0FADAE9008979
:10F6100002460B464046494600F0CCFEF8B97C084D
:10F620006B1003F17F53EA0703F5001348BF44F062
:10F63000004403EB065125460C4628462146BDE80A
:10F64000F88F02460B4600F039FC2A46234600F0AC
:10F650007FFA05460C4628462146BDE8F88FB7F1EB
:10F66000FF3FDAE90001DBE900231AD000F070FA6D
:10F67000DAE9008902460B464046494600F090FE12
:10F6800088B1B91C07F1020408BF01356408C7E757
:10F6900000F05CFA02460B4600F03AFD05460C46C7
:10F6A000CBE70135BCE70137B9E7154620214FF01C
:10F6B000FF3490E70000F07F3096FF1F3896FF1F61
:10F6C000F8B504460D4600F037F8224606460F46C8
:10F6D0002B462046294600F08BFE98B900220023D5
:10F6E0002046294600F07AFE60B900220023204619
:10F6F000294600F04BFE40B103F0BCF9084F22232D
:10F700000360002630463946F8BD03F0B3F90346DE
:10F7100021221A600348BDE8F84000F005B800BF98
:10F720000000F0FFACC6010001490020704700BF97
:10F730000000F87FFFFFFFFF2DE9F04FB1F5801FBC
:10F7400087B002460B460F4658DA21F000440443C6
:10F7500000F0F8800029C0F23281D74B002200F07F
:10F76000ADFB0F460B46D5498F4202466FF0350080
:10F7700049DC3E15C7F3130707F51521A6F2FF363E
:10F7800001F66471064401F4801106EB115681F014
:10F790007F5181F4401141EA0703104619460022C7
:10F7A000C74B00F0D3F9BB1CC3F31303022B8246F3
:10F7B0008B462FDC0022002300F0E8FD002800F03B
:10F7C000CA80002E00F04B81304600F00DFBA6A34E
:10F7D000D3E9002306460F4600F070FBA4A3D3E94B
:10F7E000002304460D463046394600F067FB0246CA
:10F7F0000B462046294600F0ABF908E0AF498F429E
:10F800004FF00000B5DD1046194600F0A1F907B031
:10F81000BDE8F08FA7F5C223A3F27A43019300223B
:10F820004FF0804300F094F902460B46504659468B
:10F8300000F06EFC044630460D4600F0D5FA224634
:10F84000CDE904012B4620462946CDE9024500F0CA
:10F8500035FB02460B468046894600F02FFB86A307
:10F86000D3E9002304460D4600F028FB84A3D3E926
:10F87000002300F06DF922462B4600F01FFB82A307
:10F88000D3E9002300F064F922462B4600F016FB72
:10F890007FA3D3E9002300F05BF942464B4600F01A
:10F8A0000DFB7DA3D3E900238046894620462946E7
:10F8B00000F004FB7AA3D3E9002300F049F92246C3
:10F8C0002B4600F0FBFA78A3D3E9002300F040F9BF
:10F8D00022462B4600F0F2FA0B46024649464046C5
:10F8E00000F036F9C7F5D727019B51371F43002F8A
:10F8F0008046894655DD734B00225046594600F03C
:10F90000DDFA52465B4600F0D9FA04460D46002E59
:10F910005CD122462B464046494600F019F9DDE904
:10F92000022300F0CBFA02460B462046294600F09F
:10F930000DF902460B465046594600F007F907B04C
:10F94000BDE8F08F002200235F49002000F0E0FBBB
:10F9500007B0BDE8F08F56A3D3E9002350465946BF
:10F9600000F0ACFA02460B460020564900F0EEF8D3
:10F97000524604460D465B465046594600F09EFAF4
:10F9800002460B462046294600F098FA04460D46EA
:10F99000002E50D102460B465046594600F0D6F88C
:10F9A00035E7002E40F0928002460B4650465946FD
:10F9B00000F0CCF8DDE9022300F080FAB9E700F0AE
:10F9C000C5F80022002300F0A3FB20E726A3D3E91B
:10F9D0000023DDE9040100F071FA22462B460646B9
:10F9E0000F464046494600F0B3F8DDE9022300F037
:10F9F00065FA1FA3D3E9002380468946DDE90401A7
:10FA000000F05CFA02460B464046494600F0A0F87A
:10FA100002460B462046294600F098F852465B46BF
:10FA200000F094F802460B463046394600F08EF856
:10FA300007B0BDE8F08F304600F0D6F90AA3D3E94D
:10FA400000238046894600F039FA09A3D3E9002350
:10FA500006460F464046494600F030FAD8E70020F7
:10FA60000021D4E6AFF300800000E0FE422EE63F26
:10FA7000763C7935EF39EA3D44523EDF12F1C23F20
:10FA8000DE03CB966446C73F599322942449D23F64
:10FA9000935555555555E53F9FC678D0099AC33FB4
:10FAA000AF788E1DC571CC3F04FA97999999D93FCB
:10FAB000555555555555D53F00005043FFFFEF7F35
:10FAC0000000F03F0000E03F000050C316A3D3E960
:10FAD0000023DDE9040100F0F1F942464B460446FB
:10FAE0000D465046594600F031F8DDE9022300F09A
:10FAF000E5F90FA3D3E9002306460F46DDE904012B
:10FB000000F0DCF902460B463046394600F01EF89C
:10FB100052465B4600F01AF802460B46204629463C
:10FB200000F014F873E600BF0000E0FE422EE63F4E
:10FB3000763C7935EF39EA3D03460846194605F02B
:10FB40000FB800BF81F0004102E000BF83F0004326
:10FB500030B54FEA41044FEA430594EA050F08BF68
:10FB600090EA020F1FBF54EA000C55EA020C7FEA2C
:10FB7000645C7FEA655C00F0E2804FEA5454D4EBA9
:10FB80005555B8BF6D420CDD2C4480EA020281EA73
:10FB9000030382EA000083EA010180EA020281EAAB
:10FBA0000303362D88BF30BD11F0004F4FEA0131FD
:10FBB0004FF4801C4CEA113102D0404261EB41010C
:10FBC00013F0004F4FEA03334CEA133302D0524292
:10FBD00063EB430394EA050F00F0A780A4F101044E
:10FBE000D5F1200E0DDB02FA0EFC22FA05F2801888
:10FBF00041F1000103FA0EF2801843FA05F359416E
:10FC00000EE0A5F120050EF1200E012A03FA0EFCEC
:10FC100028BF4CF0020C43FA05F3C01851EBE37116
:10FC200001F0004507D54FF0000EDCF1000C7EEB33
:10FC300000006EEB0101B1F5801F1BD3B1F5001F71
:10FC40000CD349085FEA30004FEA3C0C04F1010490
:10FC50004FEA445212F5800F80F09A80BCF1004FB9
:10FC600008BF5FEA500C50F1000041EB045141EA3B
:10FC7000050130BD5FEA4C0C404141EB0101013C04
:10FC800028BFB1F5801FE9D291F0000F04BF0146F3
:10FC90000020B1FA81F308BF2033A3F10B03B3F1C5
:10FCA00020020CDA0C3208DD02F1140CC2F10C0255
:10FCB00001FA0CF021FA02F10CE002F11402D8BFB3
:10FCC000C2F1200C01FA02F120FA0CFCDCBF41EA7F
:10FCD0000C019040E41AA2BF01EB0451294330BD4E
:10FCE0006FEA04041F3C1CDA0C340EDC04F114042B
:10FCF000C4F1200220FA04F001FA02F340EA030002
:10FD000021FA04F345EA030130BDC4F10C04C4F147
:10FD1000200220FA02F001FA04F340EA0300294627
:10FD200030BD21FA04F0294630BD94F0000F83F471
:10FD3000801306BF81F480110134013D4EE77FEA54
:10FD4000645C18BF7FEA655C29D094EA050F08BFA0
:10FD500090EA020F05D054EA000C04BF1946104681
:10FD600030BD91EA030F1EBF0021002030BD5FEAC5
:10FD7000545C05D14000494128BF41F0004130BDED
:10FD800014F580043CBF01F5801130BD01F0004541
:10FD900045F0FE4141F470014FF0000030BD7FEAB4
:10FDA000645C1ABF194610467FEA655C1CBF0B46AF
:10FDB000024650EA013406BF52EA033591EA030FC6
:10FDC00041F4002130BD00BF90F0000F04BF0021BE
:10FDD000704730B54FF4806404F132044FF00005F1
:10FDE0004FF0000150E700BF90F0000F04BF00216A
:10FDF000704730B54FF4806404F1320410F00045D0
:10FE000048BF40424FF000013EE700BF42004FEACA
:10FE1000E2014FEA31014FEA02701FBF12F07F4347
:10FE200093F07F4F81F06051704732F07F4208BFFE
:10FE3000704793F07F4F04BF41F40021704730B505
:10FE40004FF4607401F0004521F000411CE700BF51
:10FE500050EA010208BF704730B54FF000050AE0D4
:10FE600050EA010208BF704730B511F0004502D5D5
:10FE7000404261EB41014FF4806404F132045FEAD7
:10FE8000915C3FF4D8AE4FF003025FEADC0C18BF80
:10FE900003325FEADC0C18BF033202EBDC02C2F172
:10FEA000200300FA03FC20FA02F001FA03FE40EA04
:10FEB0000E0021FA02F11444BDE600BF70B54FF008
:10FEC000FF0C4CF4E06C1CEA11541DBF1CEA1355E6
:10FED00094EA0C0F95EA0C0F00F0DEF82C4481EA4E
:10FEE000030621EA4C5123EA4C5350EA013518BF6E
:10FEF00052EA033541F4801143F4801338D0A0FB5B
:10FF000002CE4FF00005E1FB02E506F00042E0FB07
:10FF100003E54FF00006E1FB03569CF0000F18BF0D
:10FF20004EF0010EA4F1FF04B6F5007F64F54074B5
:10FF300004D25FEA4E0E6D4146EB060642EAC62148
:10FF400041EA55514FEAC52040EA5E504FEACE2EB5
:10FF5000B4F1FD0C88BFBCF5E06F1ED8BEF1004FB8
:10FF600008BF5FEA500E50F1000041EB045170BD34
:10FF700006F0004646EA010140EA020081EA030178
:10FF8000B4EB5C04C2BFD4EB0C0541EA045170BD74
:10FF900041F480114FF0000E013C00F3AB8014F1EE
:10FFA000360FDEBF002001F0004170BDC4F1000437
:10FFB000203C35DA0C341BDC04F11404C4F12005B8
:10FFC00000FA05F320FA04F001FA05F240EA020013
:10FFD00001F0004221F0004110EBD37021FA04F649
:10FFE00042EB06015EEA430E08BF20EAD37070BD03
:10FFF000C4F10C04C4F1200500FA04F320FA05F062
:020000021000EC
:1000000001FA04F240EA020001F0004110EBD37063
:1000100041F100015EEA430E08BF20EAD37070BDD3
:10002000C4F1200500FA05F24EEA020E20FA04F3AC
:1000300001FA05F243EA020321FA04F001F000415B
:1000400021FA04F220EA020000EBD3705EEA430ECC
:1000500008BF20EAD37070BD94F0000F0FD101F0FB
:100060000046400041EB010111F4801F08BF013C34
:10007000F7D041EA060195F0000F18BF704703F072
:100080000046520043EB030313F4801F08BF013DF9
:10009000F7D043EA0603704794EA0C0F0CEA1355B5
:1000A00018BF95EA0C0F0CD050EA410618BF52EA6F
:1000B0004306D1D181EA030101F000414FF0000075
:1000C00070BD50EA410606BF1046194652EA430683
:1000D00019D094EA0C0F02D150EA013613D195EAF7
:1000E0000C0F05D152EA03361CBF104619460AD13F
:1000F00081EA030101F0004141F0FE4141F4700149
:100100004FF0000070BD41F0FE4141F4780170BD38
:1001100070B54FF0FF0C4CF4E06C1CEA11541DBF9D
:100120001CEA135594EA0C0F95EA0C0F00F0A7F89F
:10013000A4EB050481EA030E52EA03354FEA0131CC
:1001400000F088804FEA03334FF0805545EA1313DF
:1001500043EA12634FEA022245EA111545EA1065A7
:100160004FEA00260EF000419D4208BF964244F13E
:10017000FD0404F5407402D25B084FEA3202B61A5D
:1001800065EB03055B084FEA32024FF480104FF431
:10019000002CB6EB020E75EB030E22BFB61A7546A5
:1001A00040EA0C005B084FEA3202B6EB020E75EB38
:1001B000030E22BFB61A754640EA5C005B084FEAA0
:1001C0003202B6EB020E75EB030E22BFB61A75466D
:1001D00040EA9C005B084FEA3202B6EB020E75EB78
:1001E000030E22BFB61A754640EADC0055EA060E39
:1001F00018D04FEA051545EA16754FEA06164FEA7C
:10020000C30343EA52734FEAC2025FEA1C1CC0D127
:1002100011F4801F0BD141EA00014FF000004FF0B4
:10022000004CB6E711F4801F04BF01430020B4F175
:10023000FD0C88BFBCF5E06F3FF6AFAEB5EB030C2D
:1002400004BFB6EB020C5FEA500C50F1000041EB2A
:10025000045170BD0EF0004E4EEA113114EB5C04F7
:10026000C2BFD4EB0C0541EA045170BD41F48011CA
:100270004FF0000E013C90E645EA060E8DE60CEAD2
:10028000135594EA0C0F08BF95EA0C0F3FF43BAFEF
:1002900094EA0C0F0AD150EA01347FF434AF95EAA6
:1002A0000C0F7FF425AF104619462CE795EA0C0F8A
:1002B00006D152EA03353FF4FDAE1046194622E757
:1002C00050EA410618BF52EA43067FF4C5AE50EA31
:1002D00041047FF40DAF52EA43057FF4EBAE12E721
:1002E0004FF0FF3C06E000BF4FF0010C02E000BF02
:1002F0004FF0010C4DF804CD4FEA410C7FEA6C5CE5
:100300004FEA430C18BF7FEA6C5C1BD001B050EA87
:10031000410C0CBF52EA430C91EA030F02BF90EA72
:10032000020F0020704710F1000F91EA030F58BF31
:10033000994208BF90422CBFD8176FEAE37040F093
:10034000010070474FEA410C7FEA6C5C02D150EA31
:10035000013C07D14FEA430C7FEA6C5CD6D152EAEC
:10036000033CD3D05DF8040B704700BF84461046B1
:1003700062468C461946634600E000BF01B5FFF7B0
:10038000B7FF002848BF10F1000F01BD4DF808ED80
:10039000FFF7F4FF0CBF012000205DF808FB00BF51
:1003A0004DF808EDFFF7EAFF34BF012000205DF8AB
:1003B00008FB00BF4DF808EDFFF7E0FF94BF0120F8
:1003C00000205DF808FB00BF4DF808EDFFF7CEFFF9
:1003D00094BF012000205DF808FB00BF4DF808ED38
:1003E000FFF7C4FF34BF012000205DF808FB00BF09
:1003F0004FEA410C7FEA6C5C02D150EA013C0AD121
:100400004FEA430C7FEA6C5C02D152EA033C02D112
:100410004FF0000070474FF0010070474FEA410273
:1004200012F5001215D211D56FF47873B3EB625246
:1004300012D94FEAC12343F0004343EA505311F06D
:10044000004F23FA02F018BF404270474FF00000FF
:10045000704750EA013005D111F0004008BF6FF03D
:10046000004070474FF00000704700BF4A0011D2B3
:1004700012F5001211D20DD56FF47873B3EB6252FE
:100480000ED44FEAC12343F0004343EA505323FA0A
:1004900002F070474FF00000704750EA013002D17F
:1004A0004FF0FF3070474FF0000070474FEA4102B5
:1004B000B2F1E04324BFB3F5001CDCF1FE5C0DD9C2
:1004C00001F0004C4FEAC0024CEA5070B2F1004F0C
:1004D00040EB830008BF20F00100704711F0804F0F
:1004E00021D113F13872BCBF01F00040704741F4D4
:1004F00080114FEA5252C2F11802C2F1200C10FAD8
:100500000CF320FA02F018BF40F001004FEAC123BB
:100510004FEAD32303FA0CFC40EA0C0023FA02F35F
:100520004FEA4303CCE77FEA625307D150EA013335
:100530001EBF4FF0FE4040F44000704701F0004005
:1005400040F0FE4040F40000704700BF80F00040E3
:1005500002E000BF81F0004142001FBF5FEA41039B
:1005600092EA030F7FEA226C7FEA236C6AD04FEA9B
:100570001262D2EB1363C1BFD218414048404140E0
:10058000B8BF5B42192B88BF704710F0004F40F492
:10059000000020F07F4018BF404211F0004F41F4AE
:1005A000000121F07F4118BF494292EA030F3FD07A
:1005B000A2F1010241FA03FC10EB0C00C3F120038D
:1005C00001FA03F100F0004302D5494260EB40001C
:1005D000B0F5000F13D3B0F1807F06D340084FEA87
:1005E000310102F10102FE2A51D2B1F1004F40EB7C
:1005F000C25008BF20F0010040EA030070474900E4
:1006000040EB0000013A28BFB0F5000FEDD2B0FA80
:1006100080FCACF1080CB2EB0C0200FA0CF0AABFA3
:1006200000EBC25052421843BCBFD0401843704741
:1006300092F0000F81F4000106BF80F40000013247
:10064000013BB5E74FEA41037FEA226C18BF7FEA1E
:10065000236C21D092EA030F04D092F0000F08BF60
:100660000846704790EA010F1CBF0020704712F047
:100670007F4F04D1400028BF40F00040704712F186
:1006800000723CBF00F50000704700F0004343F0EB
:10069000FE4040F4000070477FEA226216BF084621
:1006A0007FEA23630146420206BF5FEA412390EAE4
:1006B000010F40F4800070474FF0000304E000BFDA
:1006C00010F0004348BF40425FEA000C08BF70478B
:1006D00043F0964301464FF000001CE050EA01024F
:1006E00008BF70474FF000030AE000BF50EA010264
:1006F00008BF704711F0004302D5404261EB410151
:100700005FEA010C02BF84460146002043F0B64375
:1007100008BFA3F18053A3F50003BCFA8CF2083A9A
:10072000A3EBC25310DB01FA02FC634400FA02FCA3
:10073000C2F12002BCF1004F20FA02F243EB0200AA
:1007400008BF20F00100704702F1200201FA02FC0C
:10075000C2F1200250EA4C0021FA02F243EB0200FF
:1007600008BF20EADC7070474FF0FF0C1CEAD05243
:100770001EBF1CEAD15392EA0C0F93EA0C0F6FD004
:100780001A4480EA010C400218BF5FEA41211ED0E2
:100790004FF0006343EA501043EA5111A0FB0131CE
:1007A0000CF00040B1F5000F3EBF490041EAD371A3
:1007B0005B0040EA010062F17F02FD2A1DD8B3F11F
:1007C000004F40EBC25008BF20F00100704790F08E
:1007D000000F0CF0004C08BF49024CEA502040EAE0
:1007E00051207F3AC2BFD2F1FF0340EAC2507047A6
:1007F00040F400004FF00003013A5DDC12F1190FE4
:10080000DCBF00F000407047C2F10002410021FA55
:1008100002F1C2F1200200FA02FC5FEA310040F16D
:10082000000053EA4C0308BF20EADC70704792F0E6
:10083000000F00F0004C02BF400010F4000F013A1E
:10084000F9D040EA0C0093F0000F01F0004C02BF19
:10085000490011F4000F013BF9D041EA0C018FE788
:100860000CEAD15392EA0C0F18BF93EA0C0F0AD08E
:1008700030F0004C18BF31F0004CD8D180EA0100B4
:1008800000F00040704790F0000F17BF90F0004F4D
:10089000084691F0000F91F0004F14D092EA0C0F2F
:1008A00001D142020FD193EA0C0F03D14B0218BFC2
:1008B000084608D180EA010000F0004040F0FE4008
:1008C00040F40000704740F0FE4040F440007047A4
:1008D0004FF0FF0C1CEAD0521EBF1CEAD15392EA23
:1008E0000C0F93EA0C0F69D0A2EB030280EA010C13
:1008F00049024FEA402037D04FF0805343EA1111AC
:1009000043EA10130CF000408B4238BF5B0042F109
:100910007D024FF4000C8B4224BF5B1A40EA0C00AE
:10092000B3EB510F24BFA3EB510340EA5C00B3EBE0
:10093000910F24BFA3EB910340EA9C00B3EBD10FCE
:1009400024BFA3EBD10340EADC001B0118BF5FEA20
:100950001C1CE0D1FD2A3FF650AF8B4240EBC25049
:1009600008BF20F0010070470CF0004C4CEA50200A
:100970007F32C2BFD2F1FF0340EAC250704740F459
:1009800000004FF00003013A37E792F0000F00F04B
:10099000004C02BF400010F4000F013AF9D040EAC9
:1009A0000C0093F0000F01F0004C02BF490011F45D
:1009B000000F013BF9D041EA0C0195E70CEAD15355
:1009C00092EA0C0F08D142027FF47DAF93EA0C0F3C
:1009D0007FF470AF084676E793EA0C0F04D14B0220
:1009E0003FF44CAF08466EE730F0004C18BF31F0D2
:1009F000004CCAD130F000427FF45CAF31F00043CC
:100A00007FF43CAF5FE700BF4FF0FF3C06E000BF64
:100A10004FF0010C02E000BF4FF0010C4DF804CD87
:100A20004FEA40024FEA41037FEA226C18BF7FEA97
:100A3000236C11D001B052EA530C18BF90EA010F99
:100A400058BFB2EB030088BFC81738BF6FEAE17028
:100A500018BF40F0010070477FEA226C02D15FEAC4
:100A6000402C05D17FEA236CE4D15FEA412CE1D030
:100A70005DF8040B704700BF844608466146FFE7F7
:100A80000FB5FFF7C9FF002848BF10F1000F0FBDD9
:100A90004DF808EDFFF7F4FF0CBF012000205DF8D2
:100AA00008FB00BF4DF808EDFFF7EAFF34BF012057
:100AB00000205DF808FB00BF4DF808EDFFF7E0FFF0
:100AC00094BF012000205DF808FB00BF4DF808ED41
:100AD000FFF7D2FF94BF012000205DF808FB00BFA4
:100AE0004DF808EDFFF7C8FF34BF012000205DF886
:100AF00008FB00BF4FEA4002B2F1FE4F0FD34FF0A8
:100B00009E03B3EB12620DD94FEA002343F000437A
:100B100010F0004F23FA02F018BF404270474FF028
:100B20000000704712F1610F01D1420205D110F0AF
:100B3000004008BF6FF0004070474FF00000704762
:100B400042000ED2B2F1FE4F0BD34FF09E03B3EB37
:100B5000126209D44FEA002343F0004323FA02F063
:100B600070474FF00000704712F1610F01D142024F
:100B700002D14FF0FF3070474FF00000704700BFC8
:100B80007BB972B90029BEBF00204FF0004106E0DA
:100B900008BF00281CBF6FF000414FF0FF3000F08D
:100BA000BBB9ADF1080C6DE904CE002909DB002BBF
:100BB0001ADB00F04DF8DDF804E0DDE9022304B0B3
:100BC0007047404261EB4101002B1BDB00F040F815
:100BD000DDF804E0DDE9022304B0404261EB4101AD
:100BE000524263EB43037047524263EB430300F00E
:100BF0002FF8DDF804E0DDE9022304B0404261EBA8
:100C000041017047524263EB430300F021F8DDF8E5
:100C100004E0DDE9022304B0524263EB4303704772
:100C200053B94AB9002908BF00281CBF4FF0FF3153
:100C30004FF0FF3000F070B9ADF1080C6DE904CE53
:100C400000F006F8DDF804E0DDE9022304B07047A7
:100C50002DE9F047089E0D4604460F46002B4AD169
:100C60008A42944665D9B2FA82F343B102FA03FC90
:100C7000C3F120029F4020FA02F217439C404FEA42
:100C80001C4E1FFA8CF5B7FBFEF1220C0EFB117700
:100C900042EA074201FB05F090420AD91CEB02022E
:100CA00001F1FF3780F01B81904240F21881023938
:100CB0006244121AA4B2B2FBFEF00EFB102244EA08
:100CC000024400FB05F5A5420AD91CEB040400F11F
:100CD000FF3280F00681A54240F20381644402386D
:100CE00040EA0140641B00211EB1DC400023C6E93C
:100CF0000043BDE8F0878B4208D9002E00F0EC805D
:100D00000021C6E900050846BDE8F087B3FA83F183
:100D1000002949D1AB4202D3824200F2F780841A03
:100D200065EB030201201746002EE2D0C6E900471A
:100D3000DFE702B9FFDEB2FA82F3002B40F08F80CA
:100D40008A1A4FEA1C471FFA8CFE0121B2FBF7F505
:100D500007FB1520220C42EA00420EFB05F09042F0
:100D600008D91CEB020205F1FF3802D2904200F2D2
:100D7000CA804546121AA4B2B2FBF7F007FB102254
:100D800044EA02440EFB00FEA64508D91CEB04040D
:100D900000F1FF3202D2A64500F2BA801046A4EB61
:100DA0000E0440EA05409FE7C1F120078B4022FA7C
:100DB00007FC4CEA030C05FA01F420FA07F3FD40A6
:100DC000234300FA01F94FEA1C401FFA8CFEB5FBE1
:100DD000F0F81C0C00FB185544EA054408FB0EF51E
:100DE000A54202FA01F20BD91CEB040408F1FF3A08
:100DF00080F08780A54240F28480A8F10208644414
:100E0000641B9DB2B4FBF0F300FB134445EA0444B9
:100E100003FB0EFEA64508D91CEB040403F1FF30CA
:100E20006BD2A64569D9023B644443EA0840A0FB63
:100E30000283A4EB0E049C42C6461D4655D352D0F5
:100E400056B1B9EB0E0364EB050404FA07F7CB4087
:100E5000CC401F43C6E900740021BDE8F087C3F110
:100E6000200102FA03FC20FA01F225FA01F19D406B
:100E70002A434FEA1C471FFA8CFEB1FBF7F007FB31
:100E80001015110C41EA054100FB0EF58D4204FAE4
:100E900003F408D91CEB010100F1FF382FD28D4279
:100EA0002DD902386144491B92B2B1FBF7F507FB1B
:100EB000151142EA014205FB0EF1914208D91CEBE3
:100EC000020205F1FF3816D2914214D9023D624464
:100ED000521A45EA004139E73146304609E73946BA
:100EE000E7E61046FCE6C145AAD2B8EB020E63EB7A
:100EF0000C050138A4E74546EAE7034695E7404676
:100F0000D1E7D0467CE7023D624433E708460BE771
:100F10006444023843E700BF704700BFFFFFFFFF94
:100F20002DE9F04FA1B08946002107921C910022C3
:100F30000021CDE90412804649461B910F4611F865
:100F4000012B2D2A5ED801A050F822F0E7100100F5
:100F50000510010005100100051001000510010039
:100F60000510010005100100051001000510010029
:100F70003B0F01003B0F01003B0F01003B0F010045
:100F80003B0F0100051001000510010005100100D4
:100F900005100100051001000510010005100100F9
:100FA00005100100051001000510010005100100E9
:100FB00005100100051001000510010005100100D9
:100FC0000510010005100100051001003B0F010094
:100FD00005100100051001000510010005100100B9
:100FE00005100100051001000510010005100100A9
:100FF00005100100051001008F1701000510010008
:101000007B17010000210991302A79D00023089331
:101010002F2A144640F229854FF0000A38465646DA
:10102000554612E00130082D1B90C8BF0AEB8A0A12
:101030000478C6BF02EB4A02A2F1300AA3F13006DF
:101040002F2C05F1010522466BDD06EB8603392CBA
:1010500002EB4303E6DDA249012201F0E5FB002893
:1010600034D11B9B1A4601331B935478002D40F05A
:101070009C85302C40F04785C3F10102981801335C
:101080001B931C78302CF9D0A4F13103082B00F20B
:1010900024831B9F431CA4F1300E0A9301253C4678
:1010A0004FF0000B06EB86060EEB46060020631C95
:1010B0001B936478A4F13001092900F2DC8201302D
:1010C0008E46002940F0AD841B9CF0E70020652C83
:1010D000AB460A90864601D0452C2FD1002D74D105
:1010E000089B034370D1079B13B1079BC3F8009083
:1010F0004FF0000BD9465846494621B0BDE8F08F65
:101100007A7802F0DF02582A00F06E8401371B97CC
:101110003A78302AFAD0002A00F0C78001230893D9
:1011200076E76F49012201F07FFB002800F0D080B4
:10113000AB464FF0000ECDF828E0704600230B932D
:10114000002D00F08E803046FEF73EFE02460B4634
:10115000CDE90423DDE90A23BBF1000F08BFAB464C
:10116000102DA3EB02032C46A8BF1024092D0C93CD
:1011700013DD5C4B03EBC40353E91223FEF79EFE21
:10118000CDE904015046FEF71FFE02460B46DDE99D
:101190000401FEF7DDFCCDE904010F2D00F3A8806A
:1011A0000C9B002B00F013840C9B40F36B83162BDD
:1011B00040F3E4840C9AC5F12503934280F20C8538
:1011C0000C9B2C1B1C4499E00025DDF86C9009F168
:1011D00001031B9399F801402B2C00F07B822D2CEE
:1011E00000F0198200230C93A4F13003092B00F2C4
:1011F0000D82302C05D11B9B01331B931C78302CA6
:10120000FAD0A4F13103082B98D81B9A0B92531CE7
:101210001B93A4F1300154782F2C09DC00F033BC6F
:1012200001331B939CF801402F2CA2F1300106DD05
:1012300001EB8102392C9C4604EB4202F0DD0B9A53
:101240009B1A082B40F31F8444F61F630B930C9BDF
:10125000002B3FF475AF0B9B5B420B93002D7FF48B
:1012600072AF089B034320D1BEF1000F7FF43BAF68
:10127000692C00F0268400F31E83492C00F02184A1
:101280004E2C7FF430AF18491BA801F0CBF9002891
:101290003FF429AF1B9B1B78282B00F0788513485F
:1012A000FEF742FA8346894602E04FF0000BD9462A
:1012B000079A0AB11B9B1360099B002B3FF41BAFDD
:1012C00009F1004399465846494621B0BDE8F08FE0
:1012D0001B9B0A905A1C1B925C78AB46EAE600BF47
:1012E0007CD0010060DD010058DA0100ACC60100CD
:1012F0000C9B2C1B1C44002C40F3008314F00F00AB
:101300000AD0BB4901EBC001DDE90423D1E90001AA
:10131000FEF7D4FDCDE9040134F00F0340F0638201
:1013200000230893394600962B465A46404603F060
:10133000C5FE15900746002800F04E83DDE90A320D
:101340009B1A0C9A002AA8BF00230D9322EAE2728E
:1013500000239B4614929A467968404603F02EFE7D
:101360008146002800F022813A690232920007F19A
:101370000C010C30FBF78AFADDE904010A910B46F7
:101380001EA901911DA90B9002460091404604F050
:1013900043FA1C90002800F0F8800121404603F039
:1013A00035FF8246002800F001811D9B002BC0F212
:1013B000F0800D9A149D9E18089A1E9C9B1A234437
:1013C0008C4A013B9342C4F1360480F2A380D21AC6
:1013D0001F2AA4EB020400F3FF80012393400F9324
:1013E00000231093089B25443444A6421D443346F1
:1013F000A8BF2346AB42A8BF2B46002B02DDE41A50
:10140000ED1AF61A0D9B002B00F39F80002C00F3C1
:10141000B3800C9B002B00F3D580002D00F3BD8022
:10142000002E08DD51463246404604F02BF8824635
:10143000002800F0BB801C994A46404604F0BAF8E8
:101440008346002800F0B2800026C368C66051467B
:101450000E9304F08FF8B042C0F24E8400F0D383B4
:101460005146584604F038FA00224FF080430446B3
:101470000D46FEF79FFF002851D00E9B002B00F079
:10148000D7805D4B11935C4D059B10960F93002404
:101490000F9A5A4E5A4B16409E4200F0F280089B1B
:1014A0007BB1B6F1D46F0CD8DDE910014EA3D3E9BE
:1014B0000023FEF77FFF002840F07D8105F1D66311
:1014C0009D1BDDE90A1004F01FF902460B46204679
:1014D0002946FEF7F3FCDDE90A32FEF739FBCDE9D8
:1014E00004010C46089B23B9444B23409E4200F064
:1014F000FD801C99404603F087FD4946404603F0B5
:1015000083FD5146404603F07FFD5946404603F0B7
:101510007BFD21E701230020CDE90F3062E7394B45
:10152000002220462946FEF7C9FCCDE910010B46F2
:101530000E990246002976D103F1004312921393CB
:10154000059B0F93DDE91245A2E751461A46404636
:1015500003F038FF824648B301461C9A404603F028
:1015600083FE18B30E901C99404603F04DFD0E9B70
:101570001C93002C7FF74DAF1C992246404603F088
:1015800081FF1C9000287FF444AFCDF830905E4678
:1015900010E0149A0D9ED51A0EE749462A46404699
:1015A00003F070FF814600287FF43AAFCDF8309009
:1015B0005E461C98DFF844902223C8F800304FF0B4
:1015C000000BC5E04946149A404603F0FBFE8146F5
:1015D00000287FF422AFE9E70B4AD31A012202FA6E
:1015E00003F3CDE90F23FDE60000C0FFFFFFDF415D
:1015F00060DD010002FCFFFF0000F03F0000F07F13
:101600000000E07F0000E03FE2FBFFFF0023CDF899
:101610006C900B9394E501230C9309F102031B9347
:1016200099F80240E0E5DDE91023CDE9122387E7D0
:10163000DDE90412002940F0AD80C2F313030F92DC
:10164000002B40F0AD80A44B002220462946FEF737
:10165000A7FE002840F0A082A04B20462946002289
:10166000FEF72CFCCDE9100101F10043189019930D
:10167000DDE918450CE7652C4FF0010E3FF4A5ADF0
:101680002AE5A2F154730593DDE9042310461946B7
:1016900004F03AF802460B4620462946FEF70EFCB7
:1016A000DDE90423FEF754FA8D4A8E4B0A409A4234
:1016B000CDE904017BD90A9A03F154739A4203D10C
:1016C0000B9B01333FF472AF874A4FF0FF33CDE9F4
:1016D00004320EE700230C939FE7652C00F0E480B2
:1016E000452C00F0E1804FF0010EBAE5109E119DEF
:1016F000304629460AF03CFCFEF7B2FB0B46024698
:1017000029463046FEF722FA0E9D049E45EA060C55
:10171000C4F313065CEA060304460D4600F0A980F4
:1017200067A3D3E90023FEF73BFE48B966A3D3E9DC
:10173000002320462946FEF751FE00283FF4D9AE8B
:10174000DDE904341C98CDF830905E46A1469B46F6
:101750000146404603F058FC0C99404603F054FC07
:101760005146404603F050FC1599404603F04CFCAE
:101770003146404603F048FC9AE501220992791C63
:101780001B917A78002A3FF4AEAC0F463CE400226D
:101790000992F4E7DDE90412012900F07C810F923F
:1017A0004D49524D0023CDE91031002470E601F17E
:1017B0005474059496E6DDE91001FEF757FE012802
:1017C00038BF0120FEF700FBCDE910010B460E9952
:1017D0000246002940F0708103F1004316921793EE
:1017E000DDE916456AE6B3F59A7F00F3F580102B24
:1017F0004FEA23143E4B40F3E082DDE904019A46B0
:1018000008930023994614F0010F09F101094FEAEA
:10181000640404D0DAE90023FEF750FB0123012C15
:101820000AF1080AEFD10BB1CDE90401089B03EBE3
:10183000C90A059BA3F154730593DDE90423DAE992
:101840000001FEF73BFB264BCDE904010B400A46A5
:1018500028498B4200F2C080A1F580118B4240F2F2
:10186000448221494FF0FF33CDE90431002308932E
:1018700058E517A3D3E90023FEF792FD00283FF4B3
:1018800038AE5DE71633FFF633ADDDE90A329A1A5A
:10189000194B03EBC203DDE90401D3E90023FEF792
:1018A00037FC8346894603E54FF0000BCDF828B09E
:1018B0004FF0010E14E46E2C3FF4E5AC13E400BFCE
:1018C0009535A094FFFFDF3F35E5AF350000E03FE1
:1018D0009535A094FFFFCF3F0000F03F0000E03FB0
:1018E0000000F07FFFFF9F7CFFFFEF7F0000F0BF55
:1018F00038DD01000000A07C60DD01003FF410AD88
:10190000644214F00F020AD0AA4B03EBC203DDE9D4
:101910000401D3E90023FEF7FBFBCDE90401241108
:101920003FF4FEAC1F2C35DC14F01003DDE904019C
:1019300018BF6A23DFF8809208930023E20704D5DA
:10194000D9E90023FEF7BAFA0123641009F1080966
:10195000F4D10BB1CDE90401089B93B1DDE9040199
:10196000C1F30A52C2F16B03002B0ADD1F2B40F3B7
:101970004C820020342B049040F360824FF05C7363
:101980000593DDE9040100220023FEF7FFFC002897
:101990003FF4C8AC22234FF0000BC8F80030D94602
:1019A00086E41E9A049203F233421F9B23F48013B1
:1019B00043EA02530593E00502D543F00043059343
:1019C0007E4A1A401AB901F055F822230360DDE976
:1019D00004349B46A1466BE42223DFF8E091C8F86B
:1019E00000304FF0000B63E40293099B01931CABA2
:1019F0000093734A1DAB1BA9404600F059FB10F041
:101A00000F0504463FF451AC062D7FD1079B0137EB
:101A1000002B3FF46DAB4FF0000B1F60D946FFF772
:101A20006ABB0A9B1B9C03440A93012805F101032E
:101A30001A4615D0284400F1FF3C03E046009C45BF
:101A40000DD001332A46082A1D4606EB8600F5D93B
:101A5000102BDCBF0AEB8A0A4FEA4A0AEFE7023290
:101A6000082D46DC1546FFF71DBB564901223846B6
:101A700000F0DAFE002878D04FF0000BDA465E4620
:101A80005D46FFF756BB44F61F639942A8BF19464F
:101A90000B91FFF7DCBBDDE904340F94002C7FF4DD
:101AA0007FAECDF830905E4622234FF0000B1C989D
:101AB000C8F80030D9464BE6DDE91023CDE91623FE
:101AC0008EE641491BA800F0ADFD00283FF40BABAA
:101AD0001B9B3E49013B1BA81B9300F0A3FD10B9C3
:101AE0001B9B01331B93DFF8D4904FF0000BFFF7E3
:101AF000DFBB102ADCBF0AEB8A0A01EB4A0A154653
:101B00000020FFF7D4BA0020FFF7BEBA1C9A3AB102
:101B100035211EA803F00AFF1C99404603F074FA11
:101B2000013D1D9B042D00F2A18101A252F825F078
:101B3000A3190100611B01005B1B0100451B010093
:101B4000A31901004FF0FF336FF00045CDE90435D4
:101B5000E3057FF53CAF059B2FE7184B0593F7E7AF
:101B60001E9B04931F9B059325E71B9B1A4601337D
:101B70001B93547806468246FFF77BBA0C980D49B2
:101B800001EBC001DDE90423D1E90001FEF796F97C
:101B900083468946FFF78CBB0D4B0E4C11930E9B71
:101BA00010930023CDE9183462E5AB460A90FFF7A5
:101BB00081BA00BF60DD010088DA01000000F07F1B
:101BC0005CDA01007CD001004CDA010050DA01003F
:101BD0000000E03F0000E0BFA54CC5F10F0504EB9D
:101BE000C501DDE90423D1E90001FEF767F90C9B8B
:101BF0005D1B04EBC504D4E90023FEF75FF98346BF
:101C00008946FFF755BB0E9BCDF830905E46109F7E
